:0405000082EF8EF008
:08050800046ED8CF05F0E0CF2E
:1005100006F00001E9CF0CF0EACF07F0E1CF08F0D8
:10052000E2CF09F0D9CF0AF0DACF0BF0F3CF12F017
:10053000F4CF13F0FACF14F0F5CF15F0F6CF16F094
:10054000F7CF17F0F8CF18F0FBCF19F000C00EF07E
:1005500001C00FF002C010F003C011F0A3AAB4EF65
:1005600002F0A4BAD8EF05F09DAABAEF02F09EBA45
:1005700068EF05F09DA0C0EF02F09EB0CEEF06F050
:10058000F0A6C6EF02F0F0B0B1EF06F0A3A8CCEFF2
:1005900002F0A4B874EF06F00EC000F00FC001F036
:1005A00010C002F011C003F00CC0E9FF07C0EAFF61
:1005B000078E08C0E1FF09C0E2FF0AC0D9FF0BC0E7
:1005C000DAFF12C0F3FF13C0F4FF14C0FAFF15C026
:1005D000F5FF16C0F6FF17C0F7FF18C0F8FF19C0E7
:1005E000FBFF045006C0E0FF05C0D8FF1000F76A0B
:1005F000020FF66E060EF722000EF86E0900F55097
:1006000012003A574643424246450000F76A200F1F
:10061000F66E060EF722000EF86E0900F550120075
:100620003A574643424239390000F76A3E0FF66EA8
:10063000060EF722000EF86E0900F55012003A5728
:100640004643424239420000F76A5C0FF66E060EDE
:10065000F722000EF86E0900F55012003A57464393
:10066000424241390000F76A7A0FF66E060EF72211
:10067000000EF86E0900F55012003A574643424208
:10068000414100002563256325732043433A2573C8
:10069000202573204D433A20257320257320434D98
:1006A0003A254C58256300004E657720526573202B
:1006B000313038306935392E39340A0D00004E6535
:1006C000772052657320313038307033300A0D0096
:1006D0004E657720526573203732307035300A0D01
:1006E00000004E657720526573203130383069350F
:1006F000300A0D004E657720526573203130383056
:100700007032350A0D004E657720526573203732FE
:10071000307036300A0D00004E6577205265732028
:10072000313038306936300A0D004E657720526519
:1007300073203732307036300A0D00005570646116
:1007400074652043616D657261205265730A0D0006
:10075000456E636F6465722028302937323070200F
:1007600035392E3934487A0A0D00456E636F646559
:10077000722028312931303830692035392E39340A
:10078000487A0A0D0000456E636F64657220283256
:10079000293130383050203330487A0A0D00456E08
:1007A000636F64657220283329373230702035300A
:1007B000487A0A0D0000456E636F64657220283424
:1007C000293130383069203530487A0A0D00456EBD
:1007D000636F6465722028352931303830502032FB
:1007E00035487A0A0D00456E636F646572202836BD
:1007F0002937323070203630487A0A0D0000456EB5
:10080000636F6465722028372931303830692036AB
:1008100030487A0A0D00436C6F636B3A2028302908
:1008200037323070203630487A0A0D00436C6F63DF
:100830006B3A203130383069203630487A0A0D0062
:10084000436C6F636B3A20283229313038305020A6
:100850003330487A0A0D0000436C6F636B3A2028EE
:10086000332937323070203530487A0A0D00436C16
:100870006F636B3A202834293130383069203530A5
:10088000487A0A0D0000436C6F636B3A20283529C3
:100890003130383050203235487A0A0D0000436C30
:1008A0006F636B3A20283029373230702036304859
:1008B0007A0A0D00436C6F636B3A2031303830692F
:1008C000203630487A0A0D00566964656F205469F5
:1008D0006D6D696E6720436C6F636B3A2028302919
:1008E000373230702035392E3935487A0A0D0000FC
:1008F000566964656F2054696D6D696E6720436C3D
:100900006F636B3A2028312931303830692035390E
:100910002E3934487A0A0D00566964656F2054698F
:100920006D6D696E6720436C6F636B3A20283229C6
:100930003130383050203330487A0A0D0000566983
:1009400064656F2054696D6D696E6720436C6F63D9
:100950006B3A2028332937323070203530487A0AF4
:100960000D00566964656F2054696D6D696E67206E
:10097000436C6F636B3A202834293130383069205A
:100980003530487A0A0D0000566964656F20546955
:100990006D6D696E6720436C6F636B3A2028352953
:1009A0003130383050203235487A0A0D000056690F
:1009B00064656F2054696D6D696E6720436C6F6369
:1009C0006B3A2028302937323070203630487A0A86
:1009D0000D00566964656F2054696D6D696E6720FE
:1009E000436C6F636B3A20283129313038306920ED
:1009F0003630487A0A0D0000496E69745F48444DEC
:100A0000490A0D00496E69745F48444D493A2037E0
:100A10003230502F35392E39340A0D00496E697441
:100A20005F48444D493A2031303830502F35392E07
:100A300039340A0D0000496E69745F48444D493AE3
:100A40002031303830692F33300A0D00496E697417
:100A50005F48444D493A20373230502F35300A0D27
:100A60000000496E69745F48444D493A203130387E
:100A700030692F35300A0D00496E69745F48444D66
:100A8000493A2031303830502F32350A0D00496E46
:100A900069745F48444D493A20373230502F363020
:100AA0000A0D0000496E69745F48444D493A20318F
:100AB000303830502F36300A0D0048444D4920451B
:100AC0006E636F646572204C6F616465720A0D001D
:100AD0000C01C06B000E9EBA010E010834E1ABA4FC
:100AE00008D0AECFC0FC000E9EBA010E000A01E194
:100AF0002BD0ABA20AD0E10EAB160000AB88000EE3
:100B00009EBA010E000A01E11FD09EAAFED7AECF09
:100B1000C0FC036A010100519C0FE96E000E032026
:100B2000EA6EC0CCEFFF01C1BFFC010E00256308D7
:100B300002E2006B01D0002B0051015D02E1BFCC4D
:100B400000F10C01C7D74C849E9A0001CCEF02F053
:100B50000C01C96BC86B06017C517A5D0C01CA6F30
:100B600006017D517B590C01CB6FCA51CBCCC9FC1E
:100B7000CACCC8FC06017D517B5D0AE303E17A51D2
:100B80007C5D06E2BC0ED8800C01C857020EC95726
:100B90000C01C95303E1C8510F0804E2010E016EB4
:100BA00004D003D0000E016E00D0000166EF06F005
:100BB000810E0C01BF6F090EC06FC16B020EC26FB8
:100BC000C369C46BC76B000EA4BA010E0108D8A498
:100BD00083D06BA408D06ECFC7FC000EA4BA010E60
:100BE000000A01E179D06BA20AD0E10E6B16000079
:100BF0006B88000EA4BA010E000A01E16DD0A4AA10
:100C0000FED76ECFC7FCD89006017A35026E7B35D1
:100C1000036E0250020FE96E010E0320EA6EEC6AC9
:100C2000ED52C7CCEFFF4C867BC6C6FC7AC6C5FC2E
:100C3000010E7A250C01C86F000E06017B210C0104
:100C4000C96F010809E2FF0A03E1C851BB0804E2C9
:100C500006017B6B7A6B04D006017A2BD8B47B2B10
:100C60007C517A5D08E17D517B5D05E1C6CC7BF668
:100C7000C5CC7AF62FD00C01C7BF0ED0462AD8B407
:100C8000472ABF0E4624E96E0C0E4720EA6EEF504D
:100C9000C75D01E04A901ED0080139510C01C75DC3
:100CA00003E0C751880804E14A80476A466A12D0C7
:100CB000C73D10D006017E2B4AA006D04AB402D010
:100CC000496A486A4A86A388000142D7015201E175
:100CD0004C8E0C010C0177D7A49A0001CCEF02F0E6
:100CE000A4A8FED76D6E12003C0E4824E96E080ED3
:100CF0004920EA6EEF3C08D0A398A4984AA603D0F6
:100D0000496A486A01D04A9448520DE149520BE1C0
:100D10004A964A8408013939006EF00E00160050D8
:100D200080093C6F00013C0E4824E96E080E492002
:100D3000EA6EEFCFBFFC0C01BF510001D1DF3C0ECA
:100D40004824E96E080E4920EA6EEF3C03D0496A58
:100D5000486A04D0482AD8B4492AA498A498CCEF69
:100D600002F0036A08012EC802F0D890023603365A
:100D70000250C60FE96E060E0320EA6EB250EF6E07
:100D8000B3CFECFFB36AB26A2E51B30802E32E2B45
:100D900001D02E6BF0900001CCEF02F04DAE36D0BA
:100DA00008012F512E5D10E14CA208D04C924C90BE
:100DB0004CB002D08C9801D08C889598456A446AD2
:100DC000436A426A29D020D04CB202D04C824C8077
:100DD000010E4226D8B0432AD8B4442AD8B4452AB2
:100DE000455207E1445205E1435203E142500708EE
:100DF0000BE24C704CB002D08C9801D08C88959846
:100E0000456A446A436A426A07D000014CA203D093
:100E10004C928C88959808019E900001CCEF02F0CE
:100E20005265616420526F746172793D2532780A8F
:100E30000D00536C6F7420636172640A0D00080129
:100E40006B6B2F6B2FC82EF86B6B6B51B30811E3D4
:100E5000036A6BC802F0D890023603360250C60F00
:100E6000E96E060E0320EA6EEC6AED52EF6A6B2B18
:100E7000ECD700011200016603D0026602D007D051
:100E8000022A00C0EEFF012EFCD7022EFAD7120074
:100E90000101006B06017B6B7A6B0101016B06019E
:100EA0007D6B7C6B4C944C967E6B4B6A4A6AEA6A0B
:100EB0009C0EE96E006A026A640E016E0001DBDFBF
:100EC000010EEA6E020EE96E006A026EBC0E016E41
:100ED000D2DFC8EF8FF00C0EEA6EB60EE96EEF505F
:100EE0000DE00A0E016E006A002EFED7012EFBD720
:100EF0005F0E006E002EFED7EF2EF3D712000A0110
:100F00001D5302E11E5342E019CAE9FF1ACAEAFF63
:100F1000EFCF1FFA1CCA03F01BCAE9FF1CCAEAFF85
:100F2000EF501F5D17E01ACA03F019CAE9FF1ACA89
:100F3000EAFFEFCF1FFA1CCA03F01BCAE9FF1CCA65
:100F4000EAFFEF501F5D02E2FF0E01D0010E016EBD
:100F50001FD00BD01ACA03F019CAE9FF1ACAEAFF58
:100F6000EF5203E1000E016E13D01ACA03F01951BB
:100F7000192BD8B41A2B1CCA03F01B511B2BD8B445
:100F80001C2B1D51D8B41E071D07BAD7000E016EC9
:100F90000001120008016C6B6B6B6D6B6E6B200EA9
:100FA0006F6F706F716F726F736F746F756F766F35
:100FB000776F786F796F7A6F7B6F7C6F7D6F7E6FE5
:100FC0007F6F806F816B030E6C6FE70E6B6F6D6BC5
:100FD0006D51080823E3F2CF82F8F29E6CC8AAFF95
:100FE0006BC8A9FFA69CA69EA680A85082BFF28EC1
:100FF0006E6F050E0C01B66F00016DDF036A08010C
:101000006D516F0FE96E080E0320EA6E6EC8EFFF98
:10101000010E6B27000E6C236D2BDAD7786B080E50
:101020000A011A6F6F0E196F1C6B2E0E1B6F1E6B51
:10103000090E1D6F000163DF015204E1010E016E14
:1010400004D003D0FF0E016E00D0CAEF8FF05A6AB1
:101050005B6A5C6A5D6A5E6A626B616B070E606FF9
:101060005F6ABCEF08F008017C6B7B6B7E6B7D6B6D
:10107000806B7F6B806B400E7F6F7C6B7B6B7C53D8
:101080005DE17B510F085AE38051036E7F517F2B46
:10109000D8B4802B816F03C082F882C8AAFF81C8B0
:1010A000A9FFA868A69CA69EA684F250006EF29E98
:1010B0000F01550EA76EAA0EA76EA682A6B2FED786
:1010C000A6940050F212050E0C01B66F000103DF6A
:1010D00008017E6B010E7D6F7E532CE17D511F0850
:1010E00029E38051036E7F517F2BD8B4802B816F11
:1010F00003C082F882C8AAFF81C8A9FFA86AA69C7B
:10110000A69EA684F250006EF29E0F01550EA76EA9
:10111000AA0EA76EA682A6B2FED7A6940050F2121F
:10112000050E0C01B66F0001D6DE08017D2BD8B488
:101130007E2BD2D77B2BD8B47C2BA1D70001BDEF5F
:1011400008F008016C6B6B6B6E6B6D6B6F6B706B8B
:10115000310E716F330E726F2D0E736F530E746FED
:10116000650E756F700E766F2D0E776F310E786F7E
:10117000796F7A6B00016BD776D7AA6AA96A5AC0D1
:10118000A8FFA69CA69EA684F250006EF29E0F01B8
:10119000550EA76EAA0EA76EA682A6B2FED7A6947B
:1011A0000050F212AA6A010EA96E5BC0A8FFA69CAD
:1011B000A69EA684F2CF00F0F29E550EA76EAA0E50
:1011C000A76EA682A6B2FED7A6940050F212AA6A13
:1011D000020EA96E5CC0A8FFA69CA69EA684F2CFB4
:1011E00000F0F29E550EA76EAA0EA76EA682A6B2BA
:1011F000FED7A6940050F212AA6A030EA96E5DC033
:10120000A8FFA69CA69EA684F2CF00F0F29E550EE3
:10121000A76EAA0EA76EA682A6B2FED7A69400500D
:10122000F212AA6A040EA96EA86AA69CA69EA684BB
:10123000F2CF00F0F29E550EA76EAA0EA76EA68200
:10124000A6B2FED7A6940050F212AA6A050EA96EA5
:10125000A86AA69CA69EA684F2CF00F0F29E550E28
:10126000A76EAA0EA76EA682A6B2FED7A6940050BD
:10127000F212AA6A070EA96E010EA86EA69CA69E7F
:10128000A684F2CF00F0F29E550EA76EAA0EA76EAE
:10129000A682A6B2FED7A6940050F212AA6A080E41
:1012A000A96E050EA86EA69CA69EA684F2CF00F09D
:1012B000F29E550EA76EAA0EA76EA682A6B2FED704
:1012C000A6940050F212AA6A090EA96E040EA86E26
:1012D000A69CA69EA684F2CF00F0F29E550EA76EA5
:1012E000AA0EA76EA682A6B2FED7A6940050F2124E
:1012F000AA6A060EA96E070EA86EA69CA69EA684D4
:10130000F2CF00F0F29E550EA76EAA0EA76EA6822F
:10131000A6B2FED7A6940050F212030E08016C6F1D
:10132000E70E6B6F6F6B6F51080827E3036A6F510D
:101330002E0FE96E000E0320EA6EEFCF70F86CC836
:10134000AAFF6BC8A9FF70C8A8FFA69CA69EA6848A
:10135000F250006EF29E0F01550EA76EAA0EA76EF8
:10136000A682A6B2FED7A6940050F212010E080182
:101370006B27000E6C236F2BD6D7030E6C6FF00E0D
:101380006B6F6E6B6D6B6F6B6F51090848E3036A8F
:101390006F51240FE96E000E0320EA6EEFCF7BF849
:1013A0007B512F0803E27B51390802E2000E01D085
:1013B000010E010832E16E5330E16D5105082DE355
:1013C000036A6F51240FE96E000E0320EA6EEFCF1F
:1013D00070F86CC8AAFF6BC8A9FF70C8A8FFA69CCC
:1013E000A69EA684F250006EF29E0F01550EA76EC7
:1013F000AA0EA76EA682A6B2FED7A6940050F2123D
:10140000050E0C01B66F000166DD08016D2BD8B426
:101410006E2B010E6B27000E6C236F2BB5D7030EBE
:101420006C6FF60E6B6F6F6B6F51080835E3036AD4
:101430006F51710FE96E080E0320EA6EEFCF70F85E
:101440006CC8AAFF6BC8A9FF70C8A8FFA69CA69E7F
:10145000A684F250006EF29E0F01550EA76EAA0EE2
:10146000A76EA682A6B2FED7A6940050F212F2CFC3
:101470007BF8F29E6CC8AAFF6BC8A9FFA69CA69E2B
:10148000A680A85008017BBFF28E706F010E6B27FB
:10149000000E6C236F2BC8D70001D1EF8FF0F2CF75
:1014A0006EF8F29EAA6AA96AA69CA69EA680A8507B
:1014B00008016EBFF28E5A6EF2CF6EF8F29EAA6AE3
:1014C000010EA96EA69CA69EA680A8506EBFF28EA5
:1014D0005B6EF2CF6EF8F29EAA6A020EA96EA69C0F
:1014E000A69EA680A8506EBFF28E5C6EF2CF6EF8FC
:1014F000F29EAA6A030EA96EA69CA69EA680A8507C
:101500006EBFF28E5D6EF2CF6EF8F29EAA6A040E86
:10151000A96EA69CA69EA680A8506EBFF28E6C6F88
:10152000F2CF6EF8F29EAA6A050EA96EA69CA69E40
:10153000A680A8506EBFF28E6B6F6CC862F06BC84D
:1015400061F0F2CF6EF8F29EAA6A070EA96EA69C11
:10155000A69EA680A8506EBFF28E6B6FF2CF6EF87B
:10156000F29EAA6A080EA96EA69CA69EA680A85006
:101570006EBFF28E6C6FF2CF6EF8F29EAA6A090E01
:10158000A96EA69CA69EA680A8506EBFF28E6D6F17
:101590006BBF0CD06C51F00B09E16D51F00B06E103
:1015A0006BC83FF86CC840F86DC841F8F2CF6EF8D0
:1015B000F29EAA6A060EA96EA69CA69EA680A850B8
:1015C0006EBFF28E0001606F6051070802E2070EE5
:1015D000606F5E6A5B9201081BE15BC06BF80801FB
:1015E0006B93AA6A010EA96E6BC8A8FFA69CA69E63
:1015F000A684F250006EF29E0F01550EA76EAA0E41
:10160000A76EA682A6B2FED7A6940050F2124C8C0A
:101610000001D3EF8FF04D8E8C989598D7EF8FF017
:101620001ACA1CFA19CA1BFA1CCA03F00A011BCAFF
:10163000E9FF1CCAEAFFEF5206E01B2BD8B41C2BB3
:101640000001F2D70A0119511B5D006E1A511C5995
:10165000036E00C001F0000112004C940101006B08
:10166000016B00011200080E016E0A011F6B1ECAF9
:1016700000F000501F1B0032012EFBD79EA8FED7A2
:10168000ACA2FED7FE0EAC161FB1AC801ECAADFFD9
:10169000000112000A011C6B1B5320E01C6B1B5144
:1016A0001C5D15E2036A1C511925E96E1A510320CD
:1016B000EA6EEFCF1DFA1DCA1EFA0001D4DF010E3B
:1016C0000C01B66F000107DC0A011C2BE8D70A0EDB
:1016D0000C01B66F00016BEC07F00A01000112006B
:1016E000016A026A006A036A0A01215102E120517B
:1016F00018E0100E226FD8901E371F3700360336C1
:101700002151035C02E12051005C07E32051005E9F
:10171000D8A003062151035ED88001360236222F5D
:10172000EAD70001ACEF0BF0036A010101519C0FF5
:10173000E96E000E0320EA6EEFCF1BFA0A01010EDC
:10174000010101250A011D6F1F6B1E6F020E216F23
:10175000BC0E206F0001C4D700C001F1010100518F
:10176000015D01E14C940A011BCA01F00001120065
:101770000A0124512619800B286F24AF05D0231F9E
:10178000241F232BD8B4242B26AF05D0251F261FBA
:10179000252BD8B4262B23512503F3CF01F0F4CF0A
:1017A00000F02603F350002624512503F3500020B7
:1017B000026E28AF05D0011E021E012AD8B4022AEB
:1017C000000156EF0CF00A01216B1F6B0A0E206F0F
:1017D0001E6B1D6B1B511C1104E1000E016E026E8D
:1017E000E8D02151212B036A1B25E96E1C510320EF
:1017F000EA6EEFCF22FA22512D080DE1010E1F6F84
:101800002151212B036A1B25E96E1C510320EA6E2E
:10181000EFCF22FA0DD022512B080AE12151212BC2
:10182000036A1B25E96E1C510320EA6EEFCF22FAF2
:1018300022512F08D8B0AFD022513908D8A0ABD050
:101840002251300821E1036A21511B25E96E1C5108
:101850000320EA6EEF5078080AE0036A21511B2545
:10186000E96E1C510320EA6EEF5058080DE1100E8E
:10187000206F212B2151212B036A1B25E96E1C515E
:101880000320EA6EEFCF22FA20510A0823E1225109
:101890002F081FE2225139081CE3246B0A0E236F24
:1018A0001ECA26FA1DCA25FA000162D7300E0A01A7
:1018B000225D01241D6F000E02201E6F2151212B7D
:1018C000036A1B25E96E1C510320EA6EEFCF22FA52
:1018D000DED761D0205110085EE12251600806E297
:1018E00022517A0803E32251DF0B01D02251226FEB
:1018F00022512F0803E22251390806E22251400802
:101900004AE22251460847E322512F0819E22251A8
:10191000390816E31D35236F1E35246F233724370E
:101920002337243723372437F00E2317300E225D58
:101930002325016E000E242101C01DFA1E6F16D052
:101940001D35236F1E35246F233724372337243763
:1019500023372437F00E2317410E225D0A0F23256B
:10196000016E000E242101C01DFA1E6F2151212B92
:10197000036A1B25E96E1C510320EA6EEF50226FAB
:10198000600806E222517A0803E32251DF0B01D0FE
:101990002251226FADD720510A0807E11F2D05D033
:1019A0001D1F1E1F1D2BD8B41E2B1DCA01F01ECAE1
:1019B00002F00001A2EF0DF0300E0A010C6F780E5C
:1019C0000D6F300E0E6F0F6F106F116F126F136B64
:1019D000156B146B176B166B020E186F1853D8B477
:1019E000C7D0156B146B176B166B090EEA6EF40EED
:1019F000E96E006A026A0C0E016E00013BEC07F012
:101A00000A0EEA6EE96A006A026A0C0E016E3BEC8D
:101A100007F0090EEA6EF40EE96EF1C9E2FFF0C9B3
:101A2000E1FFE752E6CFEEFFFCE1090E0A011A6F73
:101A3000F40E196F0001F4DD0A01176B01C016FAEC
:101A400000010BDE090E0A011A6FF40E196F16CA97
:101A50001BFA00011FDE230E0C01B66F00016BECB8
:101A600007F00A01156B146B4CA424D014CA01F0C2
:101A70000A0E1525036E14CA19FA1A6F000154DEF6
:101A80001ACAEAFF19CAE9FF01C0EFFF0A01142BC5
:101A9000D8B4152B1751155D05E303E11451165DFC
:101AA00001E208D0010E0C01B66F00016BEC07F0EB
:101AB0000A01DAD714CAE9FF0A0E1525EA6EEF6AA1
:101AC000090E1A6FF40E196F0A0E1C6F1B6B1E6B3A
:101AD000060E1D6F00017FEC07F001523FE10A0E78
:101AE0000A011A6F196B00019BDD0A011651015C96
:101AF000D8B402D0000132D01753D8B402D00001BC
:101B00002DD016510A0802E1175306E006CA11FA51
:101B100007CA12FA136B09D006CA0FFA07CA10FADD
:101B200008CA11FA09CA12FA136BF3C903F0F2C911
:101B300019FA0A01F3C91AFA0A0E1C6F0C0E1B6F70
:101B4000000141D61ACAEAFF19CAE9FF02C0ECFF38
:101B5000ED5201C0EFFF010E016E0DD00A01180712
:101B60001E0E0C01B66F00016BEC07F00A0136D7B0
:101B7000FF0E016E000112000901076BD8900601EB
:101B80007C35026E7D35036E0250020FE96E010E48
:101B90000320EA6EEFCF07F90901010E06017C254B
:101BA0000901086F000E06017D210901096F010876
:101BB00009E2FF0A03E10851BB0804E206017D6B5C
:101BC0007C6B04D006017C2BD8B47D2B9D9A9DBAEA
:101BD000FED77A517C5D04E17B517D5D01E14C963D
:101BE0009D8A090107C901F0000120EF0EF0810E66
:101BF0000801FD6F090EFE6FFF6B020E0901006FF9
:101C00000169026B036B049106017E53D8B41AD1AB
:101C10007C517A5D04E17D517B5DD8B413D19D9AEE
:101C20009DBAFED7036A090103510801FA25016E26
:101C3000FB51032201C005F903C006F900019CD73E
:101C400006C9EAFF05C9E9FF01C0EFFF9D8A036AE3
:101C5000090103510801FA25E96EFB510320EA6EE0
:101C6000EFCF05F9000E090105BF010E0108D8A448
:101C7000C2D0036A03510801FA25E96EFB51032023
:101C8000EA6EEF3C15D006017E07090104B105D0CC
:101C9000035303E0010E016ED8D006017E5304E128
:101CA000FF0E016E0901D1D00901036BA1D008011B
:101CB00009010491036A03510801FA25E96EFB51F9
:101CC0000320EA6EEF5080080CE2036A0901035119
:101CD0000801FA25E96EFB510320EA6EEF508908EE
:101CE00054E2036A090103510801FA25E96EFB5128
:101CF0000320EA6EEF50900848E0036A090103519F
:101D00000801FA25E96EFB510320EA6EEF50A008A6
:101D10003CE0036A090103510801FA25E96EFB5111
:101D20000320EA6EEF50B00830E0036A0901035166
:101D30000801FA25E96EFB510320EA6EEF50C00856
:101D400024E0036A090103510801FA25E96EFB51F9
:101D50000320EA6EEF50D00818E0036A090103512E
:101D60000801FA25E96EFB510320EA6EEF50E00806
:101D70000CE0036A090103510801FA25E96EFB51E1
:101D80000320EA6EEF50F00834E1036A09010351C1
:101D90000801FA25E96EFB510320EA6E3951EF5C28
:101DA0000CE0036A090103510801FA25E96EFB51B1
:101DB0000320EA6E3A51EF5C02E109010481090156
:101DC000035314E0FBC803F00901036A035108013F
:101DD000FA25E96EFB510320EA6EEFCF07F90901FE
:101DE000FBC8EAFFFAC8E9FF07C9EFFF010E036F5E
:101DF000080126D00901035322E004A119D0036A87
:101E000003510801FA25E96EFB510320EA6EEFCF7A
:101E100005F9036A09010351FD0FE96E080E03205D
:101E2000EA6EEF50055D03E10351030801E20491FE
:101E3000032B03510801FC5D03E20901036B080158
:101E40000601E6D6FF0E016E0901000177EF0FF0E3
:101E50000901E66BE55302E1E45326E1E45303E1B3
:101E6000E55301E1E569036AE651E225E96EE351D4
:101E70000320EA6EE551EF5C10E0036AE651E225CB
:101E8000E96EE3510320EA6EEFCFE7F9E751000175
:101E900070EC06F00901E62BE6D7E551000170EC85
:101EA00006F019D018D00901E45314E0E66BE451B0
:101EB000E65D10E2036AE651E225E96EE351032094
:101EC000EA6EEFCFE7F9E751000170EC06F0090187
:101ED000E62BEDD70001120006017E5349E0F8C859
:101EE000FBF8F7C8FAF8F9C8FCF8000180D6012C15
:101EF0003DD04AA407D0010E0C01B66F00016BEC77
:101F000007F0F7D70801F7C8E9FFF8C8EAFF395129
:101F1000EF5C15E0F7C8E9FFF8C8EAFF3A51EF5C5B
:101F20000EE0F7C8E9FFF8C8EAFFEF50880807E0BD
:101F3000F7C8E9FFF8C8EAFFEF50890804E1010E8D
:101F4000016E19D014D04AA408D0010E0C01B66F4E
:101F500000016BEC07F00801F6D7F8C8E3F9F7C801
:101F6000E2F90901E46BE569000172DF080106018D
:101F7000000E016E080100011200020E0801FF258B
:101F8000E96E000E09010021EA6EEF508009080198
:101F9000396F020EFF25E96E000E09010021EA6E7D
:101FA000EF2A00C9E3F9FFC8E2F9E46BE569000133
:101FB0004FDFC9EF69F000C9E3F9FFC8E2F9090191
:101FC000E46BE569000144DFF3EF69F0C69E9E967D
:101FD000BBCCC9FF020EC6BE05D09EA6FED7000E22
:101FE000C5BC010E016E12000901E56BC582C5B2C8
:101FF000FED7500E0C01BB6F0001E8DF0901E56B55
:10200000E451E55D10E2036AE551E225E96EE35132
:102010000320EA6EEFCFE6F9E6C9BBFC0001D6DF8C
:102020000901E52BEDD70C01BB690001CFDFC584A9
:10203000C5B4FED71200C69CC586C5B6FED700B093
:10204000C59A00A0C58AC588C5B8FED7C9CF01F01A
:1020500012000901E66BE5C903F0E4C9E9FFE5C92F
:10206000EAFFEFCFE7F9E3C9EAFFE2C9E9FF006A57
:10207000026AE7C901F000013BEC07F085A409D032
:102080000901E4C9E9FFE5C9EAFFEF6A000E016E44
:1020900089D1E5C903F00901E4C9E9FFE5C9EAFF0F
:1020A000EF50100808E3E4C9E9FFE5C9EAFFEF6A69
:1020B000FF0E016E77D1C582C5B2FED7510E0C015D
:1020C000BB6F000183DF0901E2C9E9FFE3C9EAFF51
:1020D000010E006E0001AFDF01C0EFFF010E09012C
:1020E000E225E96E000EE321EA6E010E006E0001AA
:1020F000A2DF01C0EFFF020E0901E225E96E000E2A
:10210000E321EA6E010E006E000195DF01C0EFFFD2
:10211000010E0901E225E96E000EE321EA6EEF529D
:1021200008E1020EE225E96E000EE321EA6EEF52AD
:1021300018E0030EE225E96E000EE321EA6E006A64
:10214000000179DF01C0EFFFC584C5B4FED70901E6
:10215000E4C9E9FFE5C9EAFF040EEF6EFF0E016E68
:1021600021D1E2C9E9FFE3C9EAFFEF507F0BE3C9E0
:10217000EAFFE2C9E9FFEF6EE251E96EE351EA6E70
:10218000EF50400A000130E0010A2EE0030A2CE083
:10219000010A2AE0070A28E0010A26E0030A24E0EF
:1021A000010A22E00E0A20E0030A1EE0010A1CE0F8
:1021B000070A1AE0040A18E01B0A16E0060A14E0EF
:1021C000050A2CE0040A2AE01B0A4FE0020A4DE04F
:1021D0001C0A4BE01F0AD8B479D0180AD8B476D0BC
:1021E000040AD8B4A2D0D1D0030E0901E225E96EC9
:1021F000000EE321EA6E006A00011DDF01C0EFFF5F
:10220000C584C5B4FED70901E4C9E9FFE5C9EAFF01
:10221000040EEF6E010E016EC5D0C2D0030E09018F
:10222000E225E96E000EE321EA6E010E006E000168
:1022300002DF01C0EFFF040E0901E225E96E000E86
:10224000E321EA6E006A0001F6DE01C0EFFFC584FB
:10225000C5B4FED70901E4C9E9FFE5C9EAFF050EE7
:10226000EF6E010E016E9ED09BD0030E0901E22598
:10227000E96E000EE321EA6E010E006E0001DBDE66
:1022800001C0EFFF040E0901E225E96E000EE32113
:10229000EA6E010E006E0001CEDE01C0EFFF050EFA
:1022A0000901E225E96E000EE321EA6E006A0001F1
:1022B000C2DE01C0EFFF0901E4C9E9FFE5C9EAFF99
:1022C000060EEF6E010E016E6DD06AD0030E09018D
:1022D000E66FE6510A0810E3036AE651E225E96E6B
:1022E000E3510320EA6E010E006E0001A4DE01C07E
:1022F000EFFF0901E62BEDD70B0EE225E96E000E8C
:10230000E321EA6E006A000196DE01C0EFFFC5849A
:10231000C5B4FED70901E4C9E9FFE5C9EAFF0C0E1F
:10232000EF6E010E016E3ED03BD0030E0901E66F49
:10233000E6510F0810E3036AE651E225E96EE35126
:102340000320EA6E010E006E000175DE01C0EFFF92
:102350000901E62BEDD7100EE225E96E000EE32110
:10236000EA6E006A000167DE01C0EFFFC584C5B4F4
:10237000FED70901E4C9E9FFE5C9EAFF110EEF6ED6
:10238000010E016E0FD00CD00001C584C5B4FED77C
:102390000901E4C9E9FFE5C9EAFF030EEF6E00D0C9
:1023A000FF0E016E000112004DC8EAFF4CC8E9FFA4
:1023B0000901E6C9EFFFE92AD8B4EA2AEF6A080161
:1023C0004C2BD8B44D2B000112003A0E0901E46FDA
:1023D000720EE56F450EE66F310EE76F450EE86F42
:1023E000440EE96F300EEA6FEB6FEC6FED6FEE6B42
:1023F000090EF16FE40EF06FE3C9F3F9E2C9F2F9E7
:102400000001DCEC0CF0015042EF13F0EF520FE052
:10241000EACFE3F9E9CFE2F9EFCFE6F9C5DFE3C9A7
:10242000EAFFE2C9E9FFE92AD8B4EA2AEFD71200A5
:102430000900F6CFE3F9F7CFE4F9F8CFE5F9F5CFE6
:10244000E6F9B2DFE3C9F6FFE4C9F7FFE5C9F8FF33
:102450000901E22F01D002D00001EAD700011200E9
:102460000901E3BF11D00F0E006EE23900160A0E0B
:10247000005C03E2300E002602D0E351002600C0CB
:10248000E6F9000191DF09010F0EE2170A0EE25D85
:1024900002E2300E02D0E39FE351E227E2C9E6F9FF
:1024A000000182DF12000901496B486B900E4A6FF0
:1024B000500E4B6F4C6B010E4D6F050E4E6F040EA0
:1024C0004F6F0E0E506F516F020E526F5369546B67
:1024D000120E556F566B576B560EC16F780EC26F4A
:1024E000C36F2E0EC46F780EC56FC66F2E0EC76FEA
:1024F000780EC86FC96FCA6B390ED16FD26F2D0EAF
:10250000D36F580ED46FD56FD66F2D0ED76F390E8F
:10251000D86FD96FDA6BE16B4739006EF00E001699
:10252000005080094A6F08013A510901475D04E0F3
:1025300047518908D8A41DD14751890802E1890E65
:102540004A6F85B699D0090EE36F550EE26F010E02
:10255000E46F000149DD978485A407D00A0E0C01C1
:10256000B66F00016BEC07F0F6D7090EEA6E580E55
:10257000E96E006A026A190E016E3BEC07F0090E63
:10258000EA6E710EE96E006A026A500E016E3BEC53
:1025900007F0090EEA6EC10EE96E006A026A100EBB
:1025A000016E3BEC07F0090EEA6ED10EE96E006A8F
:1025B000026A100E016E3BEC07F0120E0901E16F8A
:1025C000090EE36F580EE26F090EE56FE10EE46F3E
:1025D00000013FDD012C4FD00901E15111084CE110
:1025E000090E08014D6FC10E4C6F560E0901E66FC2
:1025F0000001DADE5BC9E6F9D7DE5CC9E6F9D4DEB4
:102600002E0E0901E66F0001CFDE5DC9E6F9CCDED2
:102610005EC9E6F9C9DE2E0E0901E66F0001C4DECF
:102620005FC9E6F9C1DE60C9E6F9BEDE090E080140
:102630004D6FD10E4C6F61C9E6F90001B5DE62C97C
:10264000E6F9B2DE2D0E0901E66F0001ADDE63C9C9
:10265000E6F9AADE64C9E6F9A7DE65C9E6F9A4DEF3
:102660002D0E0901E66F00019FDE66C9E6F99CDECA
:1026700067C9E6F999DE0901090EE36F480EE26FBA
:102680000001A3D6090EEA6E710EE96E006A026AB5
:10269000500E016E3BEC07F0090E08014D6F710EF4
:1026A0004C6F4AC9E6F900017FDE500E0901E66F62
:1026B00000017ADEEA6A2E0EE96EA8DE8A0EF66E58
:1026C000060EF76E000EF86E040E0901E26F0001AF
:1026D000AFDEEA6A240EE96E99DE200E0901E66F8C
:1026E000000162DEEA6A380EE96E90DE930EF66E45
:1026F000060EF76E000EF86E050E0901E26F00017E
:1027000097DE090EEA6EC10EE96E80DE200E090129
:10271000E66F000149DE090EEA6ED10EE96E76DE43
:102720009D0EF66E060EF76E000EF86E040E090191
:10273000E26F00017DDE49C9E2F9370E0901E36F5E
:1027400000018EDE48C9E2F9370E0901E36F00018E
:1027500087DE0901E669000127DE090E0901E36F42
:10276000710EE26FE46BE569000128EC0FF00AD00E
:102770000901090EE36F4A0EE26FE46BE56900019F
:1027800028EC0FF01200900E0901486F600E496F9F
:10279000020E4A6F4B694739006EF00E001600506A
:1027A0008009486F090EE36F480EE26FE46BE5693C
:1027B000000128EC0FF01200900E0901496F600E25
:1027C0004A6F410E4B6F4C694839006EF00E00168F
:1027D00000508009496F4751010802E24A8301D045
:1027E0004A81090EE36F490EE26FE46BE56900016F
:1027F00028EC0FF01200900E0901326F400E336F7B
:1028000034693139006EF00E001600508009326FC5
:102810003051010802E2338301D03381090EE36FA6
:10282000320EE26FE46BE569000128EC0FF0120054
:10283000900E0901326F500E336F34693139006EDA
:10284000F00E001600508009326F3051010802E28C
:10285000338301D03381090EE36F320EE26FE46BF4
:10286000E569000128EC0FF01200090166516803C8
:10287000F3CF01F0F4CF00F06903F3500026675165
:102880006803F3500020026E000112000901656B1D
:10289000646B656B646B978485A423D0642BD8B478
:1028A000652B65C967F964C966F9696B050E686FC0
:1028B0000001DBDF02C067F901C066F9090163515D
:1028C000025C07E303E16251665D03E3FF0E016E04
:1028D0000AD0050E0C01B66F00016BEC07F0090180
:1028E000DAD7010E016E0001120009014D6B040ED2
:1028F0002F6F306B090EE36F2F0EE26F010EE46F46
:102900000001F4EC0FF0120E09014D6F85A408D000
:102910000A0E0C01B66F00016BEC07F00901F6D747
:10292000090EE36F390EE26F090EE56F4D0EE46F8D
:10293000000129EC10F0015012000901586B596B8D
:10294000050E306F316B090EE36F300EE26F010E32
:10295000E46F0001F4EC0FF0270E0901636F100E15
:10296000626F000193DF012C20D0090EEA6E440E45
:10297000E96E006A026A140E016E3BEC07F0120E5B
:102980000901586F090EE36F440EE26F090EE56FFF
:10299000580EE46F000129EC10F001C059F909014B
:1029A00059C901F006D005D00001FF0E016E0901E2
:1029B00000D0000112000901D26BD16BD46BD36B34
:1029C000020E0A010D6F0D53D8B4A4D00901D26BC9
:1029D000D16BD46BD36B090EEA6ED50EE96E006A2B
:1029E000026A1C0E016E00013BEC07F0090EEA6E54
:1029F000F10EE96E006A026A1C0E016E3BEC07F0F4
:102A0000090EEA6ED50EE96ED0C9E2FFCFC9E1FF2B
:102A1000E752E6CFEEFFFCE1090E0A011A6FD50E70
:102A2000196F000110EC0BF00901D46B01C0D3F950
:102A300000012DEC0BF0090E0A011A6FD50E196F6B
:102A4000D3C91BFA00014AEC0BF0230E0C01B66F40
:102A500000016BEC07F00901D26BD16B090EEA6E35
:102A6000F10EE96E006A026A1C0E016E00013BEC79
:102A700007F04CA428D0F10E0901D125016E090EF2
:102A8000D221036E01C00EFA0A010F6F000194EC0F
:102A90000BF00FCAEAFF0ECAE9FF01C0EFFF090100
:102AA000D12BD8B4D22BD451D25D06E303E1D1515E
:102AB000D35D02E2000107D0010E0C01B66F0001E8
:102AC0006BEC07F0D6D7F10E0901D125E96E090E9E
:102AD000D221EA6EEF6A090E0A011A6FD50E196F3C
:102AE000090E1C6FF10E1B6FD4C91EFAD3C91DFA53
:102AF00000017FEC07F0015203E1010E016E0DD0E1
:102B00000A010D071E0E0C01B66F00016BEC07F0F9
:102B10000A0159D7FF0E016E000112000901496B2D
:102B2000486B3A0E4A6F720E4B6F460E4C6F380E62
:102B30004D6F350E4E6F300E4F6F506F516F526F9D
:102B4000536F546B090EF16F4A0EF06F090EF36F5D
:102B5000480EF26F0001DCEC0CF0012C0DD00901E5
:102B600046C9E9FF47C9EAFF49C9ECFFED5248C928
:102B7000EFFF010E016E0AD0090146C9E9FF47C9FE
:102B8000EAFFEC6AED52EF6AFF0E016E00011200DF
:102B90000901426B416B436B090E476F410E466F53
:102BA0000001BCDF01C043F90901432D21D142518D
:102BB000630807E23FC9E9FF40C9EAFF140EEF6E60
:102BC00014D1425162080CE2FF0A03E14151870827
:102BD00007E23FC9E9FF40C9EAFF130EEF6E05D1D6
:102BE000425162080CE2FF0A03E14151100807E27A
:102BF0003FC9E9FF40C9EAFF120EEF6EF6D042511D
:102C000061080CE2FF0A03E141516F0807E23FC986
:102C1000E9FF40C9EAFF110EEF6EE7D042516008AC
:102C20000CE2FF0A03E14151A70807E23FC9E9FFAF
:102C300040C9EAFF100EEF6ED8D042515F080CE297
:102C4000FF0A03E14151B80807E23FC9E9FF40C963
:102C5000EAFF0F0EEF6EC9D042515E080CE2FF0A88
:102C600003E14151780807E23FC9E9FF40C9EAFFA3
:102C70000E0EEF6EBAD042515D080CE2FF0A03E17E
:102C80004151390807E23FC9E9FF40C9EAFF0D0E8B
:102C9000EF6EABD042515B080CE2FF0A03E14151F9
:102CA000A90807E23FC9E9FF40C9EAFF0C0EEF6E31
:102CB0009CD0425159080CE2FF0A03E14151CA0875
:102CC00007E23FC9E9FF40C9EAFF0B0EEF6E8DD066
:102CD000425157080CE2FF0A03E141519B0807E209
:102CE0003FC9E9FF40C9EAFF0A0EEF6E7ED04251AC
:102CF00055080CE2FF0A03E141511C0807E23FC9F5
:102D0000E9FF40C9EAFF090EEF6E6FD04251520849
:102D10000CE2FF0A03E141514D0807E23FC9E9FF18
:102D200040C9EAFF080EEF6E60D042514E080CE237
:102D3000FF0A03E14151DF0807E23FC9E9FF40C94B
:102D4000EAFF070EEF6E51D042514A080CE2FF0A2B
:102D500003E14151D00807E23FC9E9FF40C9EAFF5A
:102D6000060EEF6E42D0425145080CE2FF0A03E125
:102D70004151AA0807E23FC9E9FF40C9EAFF050E31
:102D8000EF6E33D042513E080CE2FF0A03E141519D
:102D9000F50807E23FC9E9FF40C9EAFF040EEF6EFC
:102DA00024D0425135080CE2FF0A03E141514908A1
:102DB00007E23FC9E9FF40C9EAFF030EEF6E15D0F5
:102DC000425124080CE2FF0A03E14151E80807E2FE
:102DD0003FC9E9FF40C9EAFF020EEF6E06D03FC9C6
:102DE000E9FF40C9EAFF010EEF6E010E016E02D04D
:102DF000FF0E016E000105EF17F009013E6B090E91
:102E0000406F3E0E3F6F0001C3D6012C05D03EC976
:102E10003BF8010E016E02D0FF0E016EC3EF19F0F8
:102E20000901F16BF26B010EF36FDA6AD96A090ED0
:102E3000F66FE90EF56F090EEA6EED0EE96EF6C952
:102E4000E2FFF5C9E1FFF3C9F4F9D890E550EE02CD
:102E5000F350F123F450F223F42FF7D7F1C9DEFF3A
:102E6000F2C9F1F9F26BD8B0F22BF52BD8B4F62BEE
:102E7000F32BF3510508DFE10001CFEF17F0D8B2D3
:102E800004D0090EEA6EF90EE96E0901F451F81941
:102E9000800BFE6FF4AF0BD0F11FF21FF31FF41F76
:102EA000F12BD8B4F22BD8B4F32BD8B4F42BF8AF61
:102EB0000BD0F51FF61FF71FF81FF52BD8B4F62B14
:102EC000D8B4F72BD8B4F82B006A016A026A036AF7
:102ED000F96BFA6BFB6BFC6BF851F711F611F511FE
:102EE0002CE0200EFD6FD890F137F237F337F4372E
:102EF000F937FA37FB37FC37F851FC5D08E1F75139
:102F0000FB5D05E1F651FA5D02E1F551F95D0FE374
:102F1000F551F95FF651D8A0F63DFA5FF751D8A008
:102F2000F73DFB5FF851D8A0F83DFC5FD880003634
:102F3000013602360336FD2FD6D7FEAF0BD0001E6A
:102F4000011E021E031E002AD8B4012AD8B4022A88
:102F5000D8B4032AF9C9EFFFFAC9ECFFFBC9ECFFAB
:102F6000FCC9ECFF000112000901E46BE36BE26BAA
:102F7000010EE16FE66BE76BDDBF01D019D0010EEA
:102F8000E66FDDC9ECF9DCC9EBF9DBC9EAF9DAC9AE
:102F9000E9F9F069EF69EE69ED69000141D703C015
:102FA000DDF902C0DCF901C0DBF900C0DAF9090182
:102FB000E15306E1E25304E1E35302E1E4536DE03F
:102FC000D892DDC9F4F9DCC9F3F9DBC9F2F9DAC941
:102FD000F1F9F86BF76BF66BDEC9F5F900014FDF1D
:102FE00003C0E4F902C0E3F901C0E2F900C0E1F96D
:102FF000036A0901E751DF25016EE051032201C098
:10300000E9F903C0EAF9EACFECF9E9CFEBF9D882A4
:10301000090EEA6EED0EE96EDDC9F4F9DCC9F3F9CB
:10302000DBC9F2F9DAC9F1F9F86BF76BF66BDEC9B7
:10303000F5F9000124DFECC9EAFFEBC9E9FF300E26
:103040000901ED25006E000EEE21000EEF21000EAD
:10305000F021EAC9EAFFE9C9E9FF00C0EFFF036A0E
:10306000E751DF25E96EE0510320EA6EEF503908A1
:103070000AE2036AE751DF25E96EE0510320EA6EB8
:10308000070EEF24EF6EE72BE4C9DDF9E3C9DCF9A5
:10309000E2C9DBF9E1C9DAF98BD7E62D0AD0036A78
:1030A000E751DF25E96EE0510320EA6E2D0EEF6E49
:1030B000E72BE56BD890E731E55D2FE2036AE55138
:1030C000DF25E96EE0510320EA6EEFCFE8F9036AED
:1030D000E551DF25016EE051032203C0EAF9E55115
:1030E000E75DFF0F036ADF25E96EE0510320EA6E1A
:1030F000EFCFEBF9EAC9EAFF01C0E9FFEBC9EFFF47
:10310000E551E75DFF0F036ADF25E96EE05103201B
:10311000EA6EE8C9EFFFE52BCDD7036AE751DF255B
:10312000E96EE0510320EA6EEF6ADFC901F0E0C901
:1031300002F000011200300E0901D26FD36FD46B80
:10314000DD6BDC6BDB6BCFC9DAF9100EDE6F090EBD
:10315000E06FD20EDF6F000107DF090E0A011A6F60
:10316000D20E196F000110EC0BF00150020811E1B2
:103170000901D0C9E9FFD1C9EAFFD2C9EFFF010EA9
:10318000D025E96E000ED121EA6ED3C9EFFF10D031
:1031900000010901D0C9E9FFD1C9EAFF300EEF6E85
:1031A000010ED025E96E000ED121EA6ED2C9EFFFE3
:1031B000000112003A0E0901636F570E646F460E4C
:1031C000656F440E666F460E676F430E686F300E74
:1031D000696F6A6F6B6B3A0E6D6F570E6E6F460EAE
:1031E0006F6F440E706F460E716F420E726F300E2D
:1031F000736F746F756B0F0E776F0B0E786F090E10
:10320000796F070E7A6F050E7B6F030E7C6F010ED0
:103210007D6F7E6B7F6B806B816B826B846B836B4E
:1032200062C981F98151070802E2070E816F036AC2
:103230008151770FE96E090E0320EA6EEFCF80F916
:1032400081510801485DD8B46FD009018151070848
:1032500005E00801485107084EE10901520E646F6C
:10326000090EF16F630EF06F84C9F3F983C9F2F9A7
:103270000001DCEC0CF0012C39D0090183C982F982
:1032800082878151070803E1829582970BD082855E
:10329000828780C9CFF9090ED16F730ED06F0001FC
:1032A0004ADF090182C9CFF9090ED16F690ED06FCB
:1032B000000141DF570E0901646F090ED06F630EE4
:1032C000CF6F0001DBEC14F0012C0CD0090E0901CA
:1032D000D06F6D0ECF6F0001DBEC14F0012C02D02B
:1032E00081C948F8010E016E22D003D0000E016E94
:1032F0001ED019D0080180C9CFF9090E0901D16F7C
:10330000730ED06F000117DF090E0901D06F6D0E2B
:10331000CF6F0001DBEC14F0012C05D081C948F817
:10332000010E016E04D00801000E016E00011200B2
:103330000901316B326B3D91090EEA6E330EE96E75
:10334000006A026A0A0E016E00013BEC07F00901F7
:10335000305325E1090EEA6E330EE96E000E0001CE
:10336000F7EC02F00A000900F550EE6E0009FBE1EF
:10337000090E0901D06F330ECF6F0001DBEC14F0A2
:1033800001C031F93AD50901312D05D00801479125
:1033900047934795090131C901F07BD078D030AB14
:1033A00007D03051070B326F303B0F0E301702D071
:1033B000010E326F32C962F90001FCDE09013D9154
:1033C00001B03D813051020830E13DB104D0080127
:1033D00047B326D00901090EEA6E330EE96E000EDE
:1033E000000106EC03F00A000900F550EE6E00093A
:1033F000FBE1090E0901D06F330ECF6F0001DBEC4A
:1034000014F001C031F90901312D05D008014781BF
:1034100047834795090131C901F03BD005D0080128
:10342000010E016E090135D032D0305103082FE171
:103430003DB104D0080147B526D00901090EEA6E56
:10344000330EE96E000E000115EC03F00A000900CE
:10345000F550EE6E0009FBE1090E0901D06F330E45
:10346000CF6F0001DBEC14F001C031F90901312DFF
:1034700005D00801478147934785090131C901F00B
:1034800008D005D00801010E016E090102D0FF0E1F
:10349000016E00011200300E0901D56FD66FD76F93
:1034A000D86FD96BDD6BDC6BD2C9DBF9D1C9DAF926
:1034B000100EDE6F090EE06FD50EDF6F000154DDD8
:1034C000090E0A011A6FD50E196F000110EC0BF0EE
:1034D000010E015CFC0FD8B087D0040FF5EF1AF095
:1034E000030E0901D325E96E000ED421EA6ED8C976
:1034F000EFFF020ED325E96E000ED421EA6ED7C984
:10350000EFFF010ED325E96E000ED421EA6ED6C975
:10351000EFFFD3C9E9FFD4C9EAFFD5C9EFFF000126
:1035200063D0030E0901D325E96E000ED421EA6EA3
:10353000D7C9EFFF020ED325E96E000ED421EA6E43
:10354000D6C9EFFF010ED325E96E000ED421EA6E35
:10355000D5C9EFFFD3C9E9FFD4C9EAFF300EEF6E3A
:10356000000142D0030E0901D325E96E000ED421DB
:10357000EA6ED6C9EFFF020ED325E96E000ED42104
:10358000EA6ED5C9EFFF010ED325E96E000ED421F6
:10359000EA6E300EEF6ED3C9E9FFD4C9EAFF300EF0
:1035A000EF6E000121D0030E0901D325E96E000E54
:1035B000D421EA6ED5C9EFFF020ED325E96E000EC5
:1035C000D421EA6E300EEF6E010ED325E96E000EA7
:1035D000D421EA6E300EEF6ED3C9E9FFD4C9EAFFF9
:1035E000300EEF6E000100D01200E824F76AF736C3
:1035F0000B0FF66E360EF722000EF86EFB6E0A0009
:10360000F550FA6E0800F550F96EA635643522358E
:10361000E0343A0E0901336F520E346F460E356FA7
:10362000380E366F360E376F300E386F396F3A6F8F
:103630003B6B3A0E3D6F570E3E6F460E3F6F380E96
:10364000406F350E416F430E426F300E436F310EA7
:10365000446F456B3A0E476F770E486F460E496FC1
:10366000380E4A6F350E4B6F380E4C6F300E4D6F63
:103670004E6F4F6F506F516B546B536B5591090EDA
:10368000F16F330EF06F090EF36F530EF26F0001FE
:10369000DCEC0CF0012CA9D00901532D4CD0545373
:1036A0004AE1090ED06F3D0ECF6F0001DBEC14F044
:1036B000012C42D00801476B0901546B536B55B183
:1036C0003AD00A0E0C01B66F00016BEC07F0090E40
:1036D0000901F16F330EF06F090EF36F530EF26FA5
:1036E0000001DCEC0CF0012C24D009015351006ED8
:1036F0005451036E035005E1010E005C00010FE020
:103700000901035005E1020E005C00010AE0090115
:10371000035004E10052000109E009010AD0090147
:1037200008D0FF0E016E63D0090103D00901558155
:1037300000D00901C4D7000132C962F93BDD31C9AB
:10374000D2F930C9D1F9090E0901D46F4D0ED36FEA
:103750000001A1DE090E0901D06F470ECF6F0001F5
:10376000DBEC14F0012C41D00901546B536B5591E3
:1037700055B13AD00A0E0C01B66F00016BEC07F0A0
:10378000090E0901F16F330EF06F090EF36F530E3E
:10379000F26F0001DCEC0CF0012C24D00901535134
:1037A000006E5451036E035005E1010E005C0001F0
:1037B0000FE00901035005E1020E005C00010AE080
:1037C0000901035004E10052000107E009010AD099
:1037D000090108D00901558105D0010E016E07D0FD
:1037E000090100D00901C4D70001FF0E016E1200CB
:1037F0003A0E0901316F570E326F460E336F410E8C
:10380000346F320E356F310E366F300E376F386FC2
:10381000396B3051030803E1310E386F02D0300E9E
:10382000386F090ED06F310ECF6F0001DBEC14F052
:10383000015012000901586B080E306F316B090EF0
:10384000E36F300EE26F010EE46F0001F4EC0FF055
:10385000978485A407D00A0E0C01B66F00016BECAB
:1038600007F0F6D7090EEA6E440EE96E006A026AA6
:10387000140E016E3BEC07F0120E0901586F090E91
:10388000E36F440EE26F090EE56F580EE46F00011E
:1038900029EC10F0015088EF1CF009012F532EE1A4
:1038A0004DBE23D04D8E030E306F0001A1DF012CE1
:1038B00001D00BD0640E0C01B66F00016BEC07F069
:1038C000030E0901306F000193DF9DEC14F08C981A
:1038D0009598040E0901306FFA0E0C01B66F0001C5
:1038E0006BEC07F00901302FF7D7020E306F0001A3
:1038F0007FDF010E016E14D013D009014DAE0CD044
:103900004D9E030E306F000173DF8C88959892D71F
:10391000015006D005D00901010E016E000100D052
:1039200012003A0E0901306F570E316F460E326F9A
:10393000336F450E346F360E356F300E366F376F7E
:10394000386B2F51020803E1380E366F09D02F5122
:10395000030803E1430E366F03D0FF0E016E09D05A
:10396000090ED06F300ECF6F0001DBEC14F0015068
:103970000901000112003A0E0901306F770E316F14
:10398000460E326F336F330E346F300E356F366F35
:10399000376F386F396F3A6B2F51020804E1310EDF
:1039A000376F396F02D0300E376F090ED06F300E7F
:1039B000CF6F0001DBEC14F0012C0BD009012F516B
:1039C000020802E14F8001D04F90010E016E04D039
:1039D0000001FF0E016E09010001120009016D6B6B
:1039E0006C6B6F6B6E6B706B6B51100803E2FF0EAC
:1039F000016E8DD06D6B400E6C6F726B6B35026E0D
:103A00007235036E0236033602360336023603364B
:103A100002360336E00E021602506C2703506D2367
:103A2000F2CF71F9F29E6DC9AAFF6CC9A9FFA69CDD
:103A3000A69EA680A85071BFF28E00017C6F09017E
:103A40006B5100017C5D05E0FF0E016E09015FD046
:103A500000017CC070F909016C2BD8B46D2B6F6B21
:103A6000010E6E6F6F532DE16E5118082AE37C0E24
:103A70006E25E96E000E6F21EA6EF2CF73F9F29EA9
:103A80006DC9AAFF6CC9A9FFA69CA69EA680A850D6
:103A900073BFF28EEF6E7C0E6E25E96E000E6F2105
:103AA000EA6EEF5070276C2BD8B46D2B0A0E0C0108
:103AB000B66F00016BEC07F009016E2BD8B46F2BC9
:103AC000D1D7FF0E701B010E70277C0E6E25E96E9C
:103AD000000E6F21EA6EF2CF73F9F29E6DC9AAFF54
:103AE0006CC9A9FFA69CA69EA680A85073BFF28EA3
:103AF000EF6E7C0E6E25E96E000E6F21EA6E70513E
:103B0000EF5C03E0FF0E016E02D0010E016E0001BA
:103B100012003A0E09016B6F570E6C6F460E6D6FF7
:103B20006E6F300E6F6F450E706F300E716F726F6B
:103B3000736B6A51020802E1729701D07287090E15
:103B4000D06F6B0ECF6F0001DBEC14F0012C0BD0AB
:103B500009016A51020802E14D9001D04D80010E29
:103B6000016E04D00001FF0E016E09010001120078
:103B70003A0E0901636F770E646F460E656F380E5B
:103B8000666F420E676F300E686F696F6A6F6B6F9A
:103B90006C6F6D6B3A0E6F6F570E706F460E716FD4
:103BA000380E726F420E736F320E746F300E756F77
:103BB000766F776B3A0E796F770E7A6F460E7B6F62
:103BC000380E7C6F420E7D6F300E7E6F7F6F320E2F
:103BD000806F300E816F826F836B866B856B090EF1
:103BE000D06F630ECF6F0001DBEC14F0012C69D0B5
:103BF000090E0901D06F6F0ECF6F0001DBEC14F0DE
:103C0000012C5FD062C9CFF9090E0901D16F810E75
:103C1000D06F00019BEC18F0090E0901D06F790EEE
:103C2000CF6F0001DBEC14F0012C4BD0520E0901D8
:103C3000706F866B856B855343E1865341E11E0EA1
:103C40000C01B66F00016BEC07F0090E0901F16F72
:103C50006F0EF06F090EF36F850EF26F0001DCEC52
:103C60000CF0012C28D009018551006E8651036E9D
:103C7000035005E1010E005C00010FE00901035053
:103C800005E1020E005C00010DE00901035004E1B2
:103C9000005200010CE009010CD0FF0E016E13D0A0
:103CA000090107D0010E016E0ED0090102D00901F1
:103CB00000D005D00001FF0E016E05D00901BBD771
:103CC0000001FF0E016E12003A0E0901636F770EBC
:103CD000646F460E656F380E666F420E676F300E6A
:103CE000686F696F6A6F6B6F6C6F6D6B3A0E6F6F99
:103CF000570E706F460E716F380E726F420E736FF3
:103D0000320E746F300E756F766F776B3A0E796F77
:103D1000770E7A6F460E7B6F380E7C6F420E7D6F8A
:103D2000300E7E6F320E7F6F330E806F300E816FDC
:103D3000826F836B866B856B090ED06F630ECF6FBE
:103D40000001DBEC14F0090E0901D06F6F0ECF6F8C
:103D50000001DBEC14F062C9CFF9090E0901D16F43
:103D6000810ED06F00019BEC18F0090E0901D06F95
:103D7000790ECF6F0001DBEC14F0012C01D003D0E1
:103D8000FF0E016E30D0520E0901706F866B856B8D
:103D9000855329E1865327E1090EF16F6F0EF06F0D
:103DA000090EF36F850EF26F0001DCEC0CF0012CB4
:103DB00001D003D0FF0E016E16D009018551020813
:103DC00008E1865306E1010E016E00010CD009D016
:103DD0000901852D07D0865305E1FF0E016E000114
:103DE00002D00901D5D7000174EF36F00901656BE7
:103DF000646B6351100803E2FF0E016E32D0656BF5
:103E0000400E646F010E635D676B666F6635026E10
:103E10006735036E02360336023603360236033642
:103E200002360336E00E0216025064270350652363
:103E300065C9AAFF64C9A9FFA868A69CA69EA68416
:103E4000F250006EF29E0F01550EA76EAA0EA76EDD
:103E5000A682A6B2FED7A6940050F212010E016E01
:103E600009010901CFEF36F03A0E0901636F770EB1
:103E7000646F460E656F380E666F420E676F300EC8
:103E8000686F696F6A6F6B6F6C6F6D6B3A0E6F6FF7
:103E9000570E706F460E716F380E726F420E736F51
:103EA000320E746F300E756F766F776B3A0E796FD6
:103EB000770E7A6F460E7B6F380E7C6F420E7D6FE9
:103EC000300E7E6F340E7F6F330E806F300E816F39
:103ED000826F836B866B856B090ED06F630ECF6F1D
:103EE0000001DBEC14F0012C69D0090E0901D06F40
:103EF0006F0ECF6F0001DBEC14F0012C5FD062C9B4
:103F0000CFF9090E0901D16F810ED06F00019BEC32
:103F100018F0090E0901D06F790ECF6F0001DBECAC
:103F200014F0012C4BD0520E0901706F866B856B1B
:103F3000855343E1865341E11E0E0C01B66F00012B
:103F40006BEC07F0090E0901F16F6F0EF06F090EAF
:103F5000F36F850EF26F0001DCEC0CF0012C28D021
:103F600009018551006E8651036E035005E1010E73
:103F7000005C00010FE00901035005E1020E005C46
:103F800000010DE00901035004E1005200010CE0C2
:103F900009010CD0FF0E016E13D0090107D0010EEC
:103FA000016E0ED0090102D0090100D005D0000138
:103FB000FF0E016E05D00901BBD70001010E016E95
:103FC00012003A0E09016C6F520E6D6F460E6E6F45
:103FD000430E6F6F706F380E716F300E726F736FAC
:103FE000746B776B766B6AC9E9FF6BC9EAFFEF6A9E
:103FF000090EF16F6C0EF06F090EF36F760EF26F13
:104000000001DCEC0CF0012C46D04D9409017651F6
:10401000006E7751036E035005E1070E005C00014E
:1040200016E00901035005E1080E005C000117E0ED
:104030000901035005E10A0E005C000118E00901C6
:10404000035004E1005200011BE009011AD00901EC
:104050006AC9E9FF6BC9EAFF0A0EEF6E18D00901C1
:104060006AC9E9FF6BC9EAFF0B0EEF6E10D04D84F1
:1040700009016AC9E9FF6BC9EAFF030EEF6E07D0B9
:1040800009016AC9E9FF6BC9EAFFEF6A00D0010EB6
:10409000016E04D00001FF0E016E09010001120043
:1040A0003A0E09016C6F520E6D6F460E6E6F420E26
:1040B0006F6F460E706F716F300E726F736F746B2F
:1040C000776B766B6AC9E9FF6BC9EAFFEF6A090E85
:1040D000F16F6C0EF06F090EF36F760EF26F000148
:1040E000DCEC0CF0012C15D0090176A708D04D822C
:1040F0006AC9E9FF6BC9EAFF050EEF6E06D04D9263
:104100006AC9E9FF6BC9EAFFEF6A010E016E04D0CC
:104110000001FF0E016E0901000112003A0E0901B3
:104120006C6F520E6D6F460E6E6F6F6F300E706F4C
:10413000450E716F300E726F736F746B776B766BA9
:104140006AC9E9FF6BC9EAFFEF6A090EF16F6C0EED
:10415000F06F090EF36F760EF26F0001DCEC0CF0DD
:10416000012C16D0090176A708D04D806AC9E9FF55
:104170006BC9EAFF030EEF6E07D04D906AC9E9FFE5
:104180006BC9EAFF020EEF6E010E016E04D0000152
:10419000FF0E016E0901000112003A0E09016C6F59
:1041A000520E6D6F460E6E6F450E6F6F430E706F41
:1041B000450E716F300E726F736F746B776B766B29
:1041C0006AC9E9FF6BC9EAFFEF6A090EF16F6C0E6D
:1041D000F06F090EF36F760EF26F0001DCEC0CF05D
:1041E000012C19D00901765102080AE1775308E140
:1041F0004D866AC9E9FF6BC9EAFF020EEF6E07D070
:104200004D966AC9E9FF6BC9EAFF030EEF6E010E16
:10421000016E04D00001FF0E016E090100011200C1
:104220003A0E09016C6F520E6D6F460E6E6F430EA3
:104230006F6F706F380E716F300E726F736F746BBB
:104240003A0E766F720E776F460E786F796F440E66
:104250007A6F430E7B6F300E7C6F7D6F7E6F7F6F4A
:10426000806B3A0E826F520E836F460E846F430E40
:10427000856F866F390E876F300E886F896F8A6BF6
:104280008D6B8C6B8F6B8E6B6AC9E9FF6BC9EAFF14
:10429000EF6A090EF16F6C0EF06F090EF36F8C0E62
:1042A000F26F0001DCEC0CF0012C01D209018C5101
:1042B0000A0802E18D5306E08C53D8A47FD18D53B8
:1042C000D8A47CD1090EF16F760EF06F090EF36F52
:1042D0008E0EF26F0001DCEC0CF0012C6DD10901A7
:1042E0008E51006E8F51036E035005E100520001A4
:1042F000D8B4B0D00901035006E1410E005C0001C2
:10430000D8B4B0D00901035006E15F0E005C000193
:10431000D8B4B0D00901035006E17C0E005C000166
:10432000D8B4B0D00901035006E1B10E005C000121
:10433000D8B4B0D00901035006E1C90E005C0001F9
:10434000D8B4B0D00901035006E1E10E005C0001D1
:10435000D8B4B0D00901010E035C06E10E0E005C7A
:104360000001D8B4AFD00901010E035C06E1220EB2
:10437000005C0001D8B4AED00901010E035C06E177
:10438000370E005C0001D8B4ADD00901010E035C0A
:1043900006E15D0E005C0001D8B4ACD00901010E4D
:1043A000035C06E17F0E005C0001D8B4ABD00901CC
:1043B000010E035C06E1A30E005C0001D8B4AAD094
:1043C0000901010E035C06E1EF0E005C0001D8B4A8
:1043D000A9D00901010E035C06E1FD0E005C00019D
:1043E000D8B4A8D00901020E035C06E13E0E005CC1
:1043F0000001D8B4A7D00901020E035C06E1AE0E9D
:10440000005C0001D8B4A6D00901030E035C06E1EC
:10441000020E005C0001D8B4A5D00901030E035CB4
:1044200006E14B0E005C0001D8B4A4D00901030ED4
:10443000035C06E18C0E005C0001D8B4A3D0090136
:10444000030E035C06E1C60E005C0001D8B4A2D0E6
:104450000901A7D009016AC9E9FF6BC9EAFF140E77
:10446000EF6EA6D009016AC9E9FF6BC9EAFF130E16
:10447000EF6E9ED009016AC9E9FF6BC9EAFF120E0F
:10448000EF6E96D009016AC9E9FF6BC9EAFF110E08
:10449000EF6E8ED009016AC9E9FF6BC9EAFF100E01
:1044A000EF6E86D009016AC9E9FF6BC9EAFF0F0EFA
:1044B000EF6E7ED009016AC9E9FF6BC9EAFF0E0EF3
:1044C000EF6E76D009016AC9E9FF6BC9EAFF0D0EEC
:1044D000EF6E6ED009016AC9E9FF6BC9EAFF0C0EE5
:1044E000EF6E66D009016AC9E9FF6BC9EAFF0B0EDE
:1044F000EF6E5ED009016AC9E9FF6BC9EAFF0A0ED7
:10450000EF6E56D009016AC9E9FF6BC9EAFF090ECF
:10451000EF6E4ED009016AC9E9FF6BC9EAFF080EC8
:10452000EF6E46D009016AC9E9FF6BC9EAFF070EC1
:10453000EF6E3ED009016AC9E9FF6BC9EAFF060EBA
:10454000EF6E36D009016AC9E9FF6BC9EAFF050EB3
:10455000EF6E2ED009016AC9E9FF6BC9EAFF040EAC
:10456000EF6E26D009016AC9E9FF6BC9EAFF030EA5
:10457000EF6E1ED009016AC9E9FF6BC9EAFF020E9E
:10458000EF6E16D009016AC9E9FF6BC9EAFF010E97
:10459000EF6E0ED009016AC9E9FF6BC9EAFFEF6A45
:1045A00007D06AC9E9FF6BC9EAFF140EEF6E00D0AD
:1045B000010E016E7FD000017AD009018C510808EC
:1045C000D8A474D08D53D8A471D0090EF16F820E87
:1045D000F06F090EF36F8E0EF26F0001DCEC0CF041
:1045E000012C65D009018E51006E8F51036E03506E
:1045F00004E10052000125E00901035005E1010E2C
:10460000005C000126E00901035005E1020E005C98
:10461000000127E00901035005E1030E005C0001E1
:1046200028E00901035005E1040E005C000129E0C7
:104630000901035005E1050E005C00012AE00901B3
:104640002FD009016AC9E9FF6BC9EAFF140EEF6EAA
:104650002AD009016AC9E9FF6BC9EAFF0F0EEF6EA4
:1046600022D009016AC9E9FF6BC9EAFF090EEF6EA2
:104670001AD009016AC9E9FF6BC9EAFF050EEF6E9E
:1046800012D009016AC9E9FF6BC9EAFF030EEF6E98
:104690000AD009016AC9E9FF6BC9EAFFEF6A03D0D2
:1046A000FF0E016E07D0010E016E04D00001FF0E57
:1046B000016E0901000112003A0E09016C6F520EE1
:1046C0006D6F460E6E6F430E6F6F706F380E716FA9
:1046D000300E726F736F746B3A0E766F720E776F67
:1046E000460E786F796F440E7A6F450E7B6F300EF1
:1046F0007C6F7D6F7E6F7F6F806B836B826B856B52
:10470000846B6AC9E9FF6BC9EAFFEF6A090EF16FB2
:104710006C0EF06F090EF36F820EF26F0001DCEC8D
:104720000CF0012CE2D1090182510A0802E1835305
:1047300006E08253D8A4D8D18353D8A4D5D1090E8A
:10474000F16F760EF06F090EF36F840EF26F0001B9
:10475000DCEC0CF0012CC9D10901855102080CE2F6
:10476000FF0A03E18451B90807E26AC9E9FF6BC98E
:10477000EAFF1E0EEF6EB5D1855102080CE2FF0A6A
:1047800003E18451B00807E26AC9E9FF6BC9EAFF97
:104790001D0EEF6EA6D1855102080CE2FF0A03E15F
:1047A0008451A60807E26AC9E9FF6BC9EAFF1C0E3B
:1047B000EF6E97D1855102080CE2FF0A03E18451A4
:1047C0009D0807E26AC9E9FF6BC9EAFF1B0EEF6E9D
:1047D00088D1855102080CE2FF0A03E18451930855
:1047E00007E26AC9E9FF6BC9EAFF1A0EEF6E79D1D9
:1047F000855102080CE2FF0A03E18451880807E2B0
:104800006AC9E9FF6BC9EAFF190EEF6E6AD18551DB
:1048100002080CE2FF0A03E184517D0807E26AC93D
:10482000E9FF6BC9EAFF180EEF6E5BD185510208F4
:104830000CE2FF0A03E18451720807E26AC9E9FF4A
:104840006BC9EAFF170EEF6E4CD1855102080CE2DE
:10485000FF0A03E18451660807E26AC9E9FF6BC9F0
:10486000EAFF160EEF6E3DD1855102080CE2FF0AF9
:1048700003E184515A0807E26AC9E9FF6BC9EAFFFC
:10488000150EEF6E2ED1855102080CE2FF0A03E1EE
:1048900084514D0807E26AC9E9FF6BC9EAFF140EAB
:1048A000EF6E1FD1855102080CE2FF0A03E184512B
:1048B0003F0807E26AC9E9FF6BC9EAFF130EEF6E12
:1048C00010D1855102080CE2FF0A03E1845131083E
:1048D00007E26AC9E9FF6BC9EAFF120EEF6E01D168
:1048E000855102080CE2FF0A03E18451220807E225
:1048F0006AC9E9FF6BC9EAFF110EEF6EF2D085516C
:1049000002080CE2FF0A03E18451120807E26AC9B7
:10491000E9FF6BC9EAFF100EEF6EE3D08551020884
:104920000CE2FF0A03E18451010807E26AC9E9FFCA
:104930006BC9EAFF0F0EEF6ED4D0855101080CE26F
:10494000FF0A03E18451EF0807E26AC9E9FF6BC976
:10495000EAFF0E0EEF6EC5D0855101080CE2FF0A8A
:1049600003E18451DC0807E26AC9E9FF6BC9EAFF89
:104970000D0EEF6EB6D0855101080CE2FF0A03E17F
:104980008451C70807E26AC9E9FF6BC9EAFF0C0E48
:10499000EF6EA7D0855101080CE2FF0A03E18451B4
:1049A000B10807E26AC9E9FF6BC9EAFF0B0EEF6EB7
:1049B00098D0855101080CE2FF0A03E1845199085F
:1049C00007E26AC9E9FF6BC9EAFF0A0EEF6E89D0F8
:1049D000855101080CE2FF0A03E184517F0807E2D8
:1049E0006AC9E9FF6BC9EAFF090EEF6E7AD08551FB
:1049F00001080CE2FF0A03E18451610807E26AC979
:104A0000E9FF6BC9EAFF080EEF6E6BD08551010814
:104A10000CE2FF0A03E18451400807E26AC9E9FF9A
:104A20006BC9EAFF070EEF6E5CD0855101080CE2FE
:104A3000FF0A03E184511B0807E26AC9E9FF6BC959
:104A4000EAFF060EEF6E4DD0855100080CE2FF0A1A
:104A500003E18451E80807E26AC9E9FF6BC9EAFF8C
:104A6000050EEF6E3ED0855100080CE2FF0A03E10F
:104A70008451BE0807E26AC9E9FF6BC9EAFF040E68
:104A8000EF6E2FD0855100080CE2FF0A03E184513C
:104A9000800807E26AC9E9FF6BC9EAFF030EEF6EFF
:104AA00020D0855100080CE2FF0A03E18451300850
:104AB00007E26AC9E9FF6BC9EAFF020EEF6E11D087
:104AC000855303E18451BF0807E26AC9E9FF6BC956
:104AD000EAFF010EEF6E05D06AC9E9FF6BC9EAFF74
:104AE000EF6A010E016E04D00001FF0E016E090194
:104AF000000112003A0E0901796F720E7A6F460EAC
:104B00007B6F420E7C6F7D6F430E7E6F300E7F6F2A
:104B1000806F816F826F836B866B856B77C9E9FFCE
:104B200078C9EAFFEC6AED52EF6A090EF16F790E6F
:104B3000F06F090EF36F850EF26F0001DCEC0CF0E4
:104B4000012CBFD0090177C9E9FF78C9EAFF86C9FE
:104B5000ECFFED5285C9EFFF865103081FE2FF0A03
:104B600003E185517F081AE28651040817E377C9EB
:104B7000E9FF78C9EAFFECCF8AF9ED52EFCF89F966
:104B8000800E895D006E020E8A5978C9EAFF77C9E6
:104B9000E9FFEC6EED5200C0EFFF8FD086510208A6
:104BA0001FE2FF0A03E185517F081AE286510308DC
:104BB00017E377C9E9FF78C9EAFFECCF8AF9ED522C
:104BC000EFCF89F9000E895D006E020E8A5978C90F
:104BD000EAFF77C9E9FFEC6EED5200C0EFFF6DD040
:104BE000865101081FE2FF0A03E185517F081AE29E
:104BF0008651020817E377C9E9FF78C9EAFFECCFCD
:104C00008AF9ED52EFCF89F9800E895D006E010EB1
:104C10008A5978C9EAFF77C9E9FFEC6EED5200C006
:104C2000EFFF4BD078C903F077C9E9FF78C9EAFFF5
:104C3000ECCF88F9ED52EFCF87F9885100081FE2D9
:104C4000FF0A03E187517F081AE28651010817E342
:104C500077C9E9FF78C9EAFFECCF8AF9ED52EFCFC7
:104C600089F9000E895D006E010E8A5978C9EAFF44
:104C700077C9E9FFEC6EED5200C0EFFF1ED08653FE
:104C800003E185517F0819E28651000816E377C9D0
:104C9000E9FF78C9EAFFECCF8AF9ED52EFCF89F945
:104CA000800E895D006E000E8A5978C9EAFF77C9C7
:104CB000E9FFEC6EED5200C0EFFF010E016E04D073
:104CC0000001FF0E016E09010001120009017A6B5B
:104CD000796B3A0E7B6F720E7C6F460E7D6F420EC3
:104CE0007E6F7F6F450E806F300E816F826F836F96
:104CF000846F856B77C9E9FF78C9EAFFEC6AED52EA
:104D0000EF6A090EF16F7B0EF06F090EF36F790EEB
:104D1000F26F0001DCEC0CF0012CB4D0090177C972
:104D2000E9FF78C9EAFF7AC9ECFFED5279C9EFFFD4
:104D30007A5103081FE2FF0A03E179517F081AE262
:104D40007A51040817E377C9E9FF78C9EAFFECCF85
:104D50008AF9ED52EFCF89F9800E895D006E020E5F
:104D60008A5978C9EAFF77C9E9FFEC6EED5200C0B5
:104D7000EFFF84D07A5102081FE2FF0A03E1795164
:104D80007F081AE27A51030817E377C9E9FF78C967
:104D9000EAFFECCF8AF9ED52EFCF89F9000E895D79
:104DA000006E020E8A5978C9EAFF77C9E9FFEC6EF6
:104DB000ED5200C0EFFF62D07A5101081FE2FF0AF6
:104DC00003E179517F081AE27A51020817E377C9A3
:104DD000E9FF78C9EAFFECCF8AF9ED52EFCF89F904
:104DE000800E895D006E010E8A5978C9EAFF77C985
:104DF000E9FFEC6EED5200C0EFFF40D07A510008A1
:104E00001FE2FF0A03E179517F081AE27A51010893
:104E100017E377C9E9FF78C9EAFFECCF8AF9ED52C9
:104E2000EFCF89F9000E895D006E010E8A5978C9AD
:104E3000EAFF77C9E9FFEC6EED5200C0EFFF1ED02C
:104E40007A5303E179517F0819E27A51000816E399
:104E500077C9E9FF78C9EAFFECCF8AF9ED52EFCFC5
:104E600089F9800E895D006E000E8A5978C9EAFFC3
:104E700077C9E9FFEC6EED5200C0EFFF010E016E45
:104E800004D00001FF0E016E0901000112003A0E6C
:104E900009016C6F520E6D6F460E6E6F420E6F6F92
:104EA000460E706F360E716F300E726F736F746BCB
:104EB000776B766B6AC9E9FF6BC9EAFFEF6A090E87
:104EC000F16F6C0EF06F090EF36F760EF26F00014A
:104ED000DCEC0CF0012C0BD009016AC9E9FF6BC9AD
:104EE000EAFF76C9EFFF010E016E04D00001FF0E4C
:104EF000016E0901000112003A0E09016C6F520E99
:104F00006D6F300E6E6F430E6F6F370E706F716F77
:104F1000300E726F736F746B796B786B6AC9E9FFCF
:104F20006BC9EAFFEF6A090EF16F6C0EF06F090EA4
:104F3000F36F780EF26F0001DCEC0CF0012C0BD05B
:104F400009016AC9E9FF6BC9EAFF78C9EFFF010EE1
:104F5000016E04D00001FF0E016E09010001120074
:104F60003A0E09016A6F520E6B6F460E6C6F420E5D
:104F70006D6F440E6E6F390E6F6F300E706F716F04
:104F8000726B756B746B090EF16F6A0EF06F090E20
:104F9000F36F740EF26F0001DCEC0CF0012C4DD0BD
:104FA00074C972F0410E09016F6F090EF16F6A0E3C
:104FB000F06F090EF36F740EF26F0001DCEC0CF071
:104FC000012C3BD074C973F0420E09016F6F090EBA
:104FD000F16F6A0EF06F090EF36F740EF26F00013D
:104FE000DCEC0CF0012C29D074C974F0430E0901DB
:104FF0006F6F090EF16F6A0EF06F090EF36F740E8A
:10500000F26F0001DCEC0CF0012C17D074C975F0C4
:10501000440E09016F6F090EF16F6A0EF06F090EF1
:10502000F36F740EF26F0001DCEC0CF0012C05D074
:1050300074C976F0010E016E02D0FF0E016E8DEF85
:1050400034F03A0E09016A6F520E6B6F460E6C6FA8
:10505000420E6D6F440E6E6F460E6F6F300E706FA6
:10506000716F726B756B746B090EF16F6A0EF06F76
:10507000090EF36F740EF26F0001DCEC0CF0012CE2
:105080004FD074C977F0450E09016E6F300E6F6F07
:10509000090EF16F6A0EF06F090EF36F740EF26F66
:1050A0000001DCEC0CF0012C3BD074C978F0310E1F
:1050B00009016F6F090EF16F6A0EF06F090EF36F41
:1050C000740EF26F0001DCEC0CF0012C29D074C9D5
:1050D00079F0320E09016F6F090EF16F6A0EF06FF1
:1050E000090EF36F740EF26F0001DCEC0CF0012C72
:1050F00017D074C97AF0330E09016F6F090EF16F82
:105100006A0EF06F090EF36F740EF26F0001DCECA3
:105110000CF0012C05D074C97BF0010E016E02D099
:10512000FF0E016E9DEF34F03A0E09016A6F520EC8
:105130006B6F460E6C6F420E6D6F430E6E6F390EC5
:105140006F6F300E706F716F726B756B746B090ED1
:10515000F16F6A0EF06F090EF36F740EF26F0001BB
:10516000DCEC0CF0012C4DD074C96DF0410E09013E
:105170006F6F090EF16F6A0EF06F090EF36F740E08
:10518000F26F0001DCEC0CF0012C3BD074C96EF026
:10519000420E09016F6F090EF16F6A0EF06F090E72
:1051A000F36F740EF26F0001DCEC0CF0012C29D0CF
:1051B00074C96FF0430E09016F6F090EF16F6A0E2B
:1051C000F06F090EF36F740EF26F0001DCEC0CF05F
:1051D000012C17D074C970F0440E09016F6F090ECD
:1051E000F16F6A0EF06F090EF36F740EF26F00012B
:1051F000DCEC0CF0012C05D074C971F0010E016ECD
:1052000002D0FF0E016EADEF34F070C97CF064C0C7
:105210007DF065C07EF066C07FF067C080F068C03A
:1052200081F06AC082F069C083F06CC084F06BC00A
:1052300085F06DC086F06EC087F06FC088F070C0DA
:1052400089F071C08AF072C08BF073C08CF074C0AA
:105250008DF075C08EF076C08FF077C090F078C07A
:1052600091F079C092F07AC093F07BC094F0010E77
:10527000016E61EF29F009016C6B6B6B6E6B6D6BEE
:105280006F6B6A51100803E2FF0E016E77D06C6BF2
:10529000400E6B6F716B6A35026E7135036E0236AC
:1052A0000336023603360236033602360336E00E84
:1052B000021602506B2703506C236AC970F9000173
:1052C000A4D709016F6B6E6B6D6B6E5339E16D5135
:1052D000180836E37C0E6D25E96E000E6E21EA6E2D
:1052E000EFCF70F96CC9AAFF6BC9A9FF70C9A8FFFD
:1052F000A69CA69EA684F250006EF29E0F01550E4B
:10530000A76EAA0EA76EA682A6B2FED7A6940050DC
:10531000F2127C0E09016D25E96E000E6E21EA6E17
:10532000EF506F276B2BD8B46C2B0A0E0C01B66FA5
:1053300000016BEC07F009016D2BD8B46E2BC5D7BB
:10534000FF0E6F1B010E6F276CC9AAFF6BC9A9FF67
:105350006FC9A8FFA69CA69EA684F250006EF29E7E
:105360000F01550EA76EAA0EA76EA682A6B2FED793
:10537000A6940050F212010E016E09010001BAEF6D
:1053800034F009016B5100017C5D03E0FF0E016EFA
:1053900032D07DC064F07EC065F07FC066F080C012
:1053A00067F081C068F082C06AF083C069F084C091
:1053B0006CF085C06BF086C06DF087C06EF088C061
:1053C0006FF089C070F08AC071F08BC072F08CC031
:1053D00073F08DC074F08EC075F08FC076F090C001
:1053E00077F091C078F092C079F093C07AF094C0D1
:1053F0007BF0010E016E06EF2AF06AC96BF9EEEC44
:105400001CF0012C06D06AC96BF9BBD7015004D03F
:1054100003D0FF0E016E00D0CDEF34F009016C6BAC
:105420006B6B3A0E6D6F520E6E6F460E6F6F420EC3
:10543000706F460E716F726F300E736F746F756B95
:10544000090EF16F6D0EF06F090EF36F6B0EF26FB8
:105450000001DCEC0CF0012C56D0570E09016E6FE8
:105460006A5105082FE16BA704D04D82010E016E31
:105470004DD0786B550E776F00017AEC25F009015D
:10548000786B570E776F000121DC09016B876BC9C0
:10549000CFF9090ED16F730ED06F00019BEC18F09D
:1054A000090E0901D06F6D0ECF6F0001DBEC14F017
:1054B000012C06D04D82010E016E090127D000019A
:1054C00022D009016BB705D04D92010E016E1ED09E
:1054D00019D06B976BC9CFF9090ED16F730ED06FCE
:1054E00000019BEC18F0090E0901D06F6D0ECF6F13
:1054F0000001DBEC14F0012C06D04D92010E016E80
:10550000090104D00001FF0E016E09010001120023
:1055100009016D6B6C6B3A0E6E6F770E6F6F460EF6
:10552000706F420E716F726F430E736F300E746F37
:10553000756F766F776F786B6B5101080EE26B5168
:1055400002080BE303E16A517F0807E3800E6A2536
:105550006C6F020E6B216D6F56D06B5100080EE21E
:10556000FF0A03E16A517F0809E26B51010806E373
:105570006AC96CF9020E6B256D6F45D06B5100083E
:1055800002E3000E01D0010E7A6F6B51010804E3B3
:1055900005E16A517F0802E2000E01D0010E7A1582
:1055A00007E0800E6A256C6F010E6B216D6F2BD0AA
:1055B0006B5305E16A517F0802E3000E01D0010E32
:1055C0007A6F6B51000802E2000E01D0010E7A15CD
:1055D00006E06AC96CF9010E6B256D6F14D06B5330
:1055E00003E16A517F0802E2000E01D0010E010BB7
:1055F00007E0800E6A256C6F000E6B216D6F03D083
:10560000FF0E016E1DD06DC9D2F96CC9D1F9090E1A
:10561000D46F740ED36F00014BEC1AF0090E090120
:10562000D06F6E0ECF6F0001DBEC14F0012C05D0B3
:10563000010E016E090104D00001FF0E016E090187
:105640000001120009016D6B6C6B3A0E6E6F770EE4
:105650006F6F460E706F420E716F726F450E736FF3
:10566000300E746F756F766F776F786B6B510108C2
:105670000EE26B5102080BE303E16A517F0807E376
:10568000800E6A256C6F020E6B216D6F56D06B51C8
:1056900000080EE2FF0A03E16A517F0809E26B513C
:1056A000010806E36AC96CF9020E6B256D6F45D0DF
:1056B0006B51000802E3000E01D0010E7A6F6B51AE
:1056C000010804E305E16A517F0802E2000E01D0FF
:1056D000010E7A1507E0800E6A256C6F010E6B21B2
:1056E0006D6F2BD06B5305E16A517F0802E3000E0A
:1056F00001D0010E7A6F6B51000802E2000E01D05A
:10570000010E7A1506E06AC96CF9010E6B256D6F02
:1057100014D06B5303E16A517F0802E2000E01D0FE
:10572000010E010B07E0800E6A256C6F000E6B21E5
:105730006D6F03D0FF0E016E1DD06DC9D2F96CC91B
:10574000D1F9090ED46F740ED36F00014BEC1AF02F
:10575000090E0901D06F6E0ECF6F0001DBEC14F063
:10576000012C05D0010E016E090104D00001FF0ECD
:10577000016E0901000112003A0E09017A6F520E02
:105780007B6F460E7C6F430E7D6F7E6F390E7F6F91
:10579000300E806F816F826B3A0E846F520E856F70
:1057A000460E866F430E876F886F380E896F300EF6
:1057B0008A6F8B6F8C6B8F6B8E6B916B906B3A0ECD
:1057C000926F720E936F460E946F956F440E966FA4
:1057D000410E976F300E986F996F9A6F9B6F9C6B0D
:1057E00078C9E9FF79C9EAFFEF6A090EF16F840E03
:1057F000F06F090EF36F8E0EF26F0001DCEC0CF00F
:10580000012C4ED109018E5107081CE18F531AE17A
:10581000090EF16F7A0EF06F090EF36F900EF26FB2
:105820000001DCEC0CF0012C0BD0090178C9E9FF78
:1058300079C9EAFF90C9EFFF010E016E34D1000172
:105840002FD109018E510A08D8A429D18F53D8A489
:1058500026D1090EF16F920EF06F090EF36F900EC4
:10586000F26F0001DCEC0CF0012C1AD1090178C9AF
:10587000E9FF79C9EAFF050EEF6E9051006E915174
:10588000036E030E035C06E1C00E005C0001D8B499
:10589000A7D00901040E035C06E14D0E005C000177
:1058A000D8B4A6D00901040E035C06E1650E005CC5
:1058B0000001D8B49DD00901040E035C06E1800EFE
:1058C000005C0001D8B49CD00901040E035C06E121
:1058D000B30E005C0001D8B493D00901040E035C40
:1058E00006E1F10E005C0001D8B492D00901050E6A
:1058F000035C06E14C0E005C0001D8B491D00901B4
:10590000050E035C06E17F0E005C0001D8B488D070
:105910000901060E035C06E10D0E005C0001D8B41F
:1059200087D00901060E035C06E1400E005C000111
:10593000D8B47ED00901060E035C06E1CD0E005CF2
:105940000001D8B47DD00901070E035C05E10052C7
:105950000001D8B475D00901070E035C06E18E0E74
:10596000005C0001D8B474D00901070E035C06E1A5
:10597000C10E005C0001D8B46BD00901080E035CB5
:1059800006E14F0E005C0001D8B46AD00901080E90
:10599000035C05E1810E005C000162E00901090E73
:1059A000035C05E14D0E005C000162E00901090E97
:1059B000035C05E1800E005C00015AE009010A0E5B
:1059C000035C05E1F70E005C00015AE009010A0ED4
:1059D000035C05E1B20E005C000152E0090158D001
:1059E000090178C9E9FF79C9EAFF050EEF6E54D0C5
:1059F000090178C9E9FF79C9EAFF060EEF6E4CD0BC
:105A0000090178C9E9FF79C9EAFF070EEF6E44D0B2
:105A1000090178C9E9FF79C9EAFF080EEF6E3CD0A9
:105A2000090178C9E9FF79C9EAFF090EEF6E34D0A0
:105A3000090178C9E9FF79C9EAFF0A0EEF6E2CD097
:105A4000090178C9E9FF79C9EAFF0B0EEF6E24D08E
:105A5000090178C9E9FF79C9EAFF0C0EEF6E1CD085
:105A6000090178C9E9FF79C9EAFF0D0EEF6E14D07C
:105A7000090178C9E9FF79C9EAFF0E0EEF6E0CD073
:105A8000090178C9E9FF79C9EAFF0F0EEF6E04D06A
:105A9000FF0E016E08D000D0010E016E04D000018F
:105AA000FF0E016E0901000112003A0E09017B6F21
:105AB000520E7C6F460E7D6F430E7E6F7F6F380EE9
:105AC000806F300E816F826F836B866B856B3A0EB1
:105AD000876F770E886F460E896F8A6F440E8B6FC3
:105AE000410E8C6F300E8D6F8E6F8F6F906F916B3C
:105AF0003A0E936F570E946F460E956F430E966F46
:105B0000976F390E986F300E996F9A6F9B6BC00E1E
:105B10009F6F030EA06FC00EA16F030EA26F4D0EFC
:105B2000A36F040EA46F650EA56F040EA66F800E02
:105B3000A76F040EA86FB30EA96F040EAA6FF10E23
:105B4000AB6F040EAC6FF10EAD6F040EAE6F4C0E6A
:105B5000AF6F050EB06F7F0EB16F050EB26F0D0EF9
:105B6000B36F060EB46F7F0EB56F050EB66FCD0E18
:105B7000B76F060EB86F400EB96F060EBA6F8E0E75
:105B8000BB6F070EBC6FBD6BBE6F4F0EBF6F080EB5
:105B9000C06FC10EC16F070EC26F4D0EC36F090EED
:105BA000C46F800EC56F090EC66FF70EC76F0A0E61
:105BB000C86FB20EC96F0A0ECA6FCB6BCC6BCD6BC0
:105BC000CE6B7A51040863E27A510F0860E3090E44
:105BD000F16F7B0EF06F090EF36F850EF26F00010F
:105BE000DCEC0CF0012C52D0090185510A0836E199
:105BF000865334E1050E7A5D040DF350D06BCF6F00
:105C0000000E82B4010E006ED89000360050036A78
:105C1000CF25016ED051032201509F0FE96E090E6E
:105C20000320EA6EECCFD0F9ED52EFCFCFF9D0C917
:105C3000D2F9CFC9D1F9090ED46F8D0ED36F0001FF
:105C40004BEC1AF0090E0901D06F870ECF6F0001DF
:105C5000DBEC14F001501ED019D009018551070862
:105C600016E1865314E17AC9CFF9090ED16F990E66
:105C7000D06F00019BEC18F0090E0901D06F930E54
:105C8000CF6F0001DBEC14F0015004D00901FF0ECE
:105C9000016E000112000901776B766B090E796FB6
:105CA000760E786F000168DD012C40D00901755334
:105CB00008E1050E7A6F0001F8DE01503BD036D0C6
:105CC00009017551020819E1775311E176510D0868
:105CD0000EE3010E7625786F000E7721796F78C973
:105CE0007AF90001E2DE015025D005D00901010E4C
:105CF000016E00011FD01AD009017551030817E188
:105D0000765302E177530EE0010E765D786F000E58
:105D10007759796F78C97AF90001C7DE01500AD046
:105D200005D00901010E016E000104D00901FF0E2A
:105D3000016E000112003A0E09016B6F570E6C6F75
:105D4000460E6D6F430E6E6F6F6F380E706F300EB4
:105D5000716F726F736B6A51030830E0300E716FB0
:105D6000726F6A51000A000105E00B0A09E0010A9E
:105D70000CE010D0300E0901716F726F00010AD073
:105D8000380E0901726F000105D0370E0901726FDC
:105D9000000100D0090E0901D06F6B0ECF6F00011A
:105DA000DBEC14F0012C05D04D94010E016E1DD0DA
:105DB00003D0FF0E016E19D005D00901300E716FAE
:105DC000410E726F090E0901D06F6B0ECF6F00018B
:105DD000DBEC14F0012C07D04D840901756B000138
:105DE0005ADF015002D0FF0E016E12003A0E090177
:105DF0006B6F520E6C6F460E6D6F430E6E6F6F6F52
:105E0000380E706F300E716F726F736B3A0E756F64
:105E1000770E766F460E776F786F440E796F450E6A
:105E20007A6F300E7B6F7C6F7D6F7E6F7F6B826BC6
:105E3000816B846B836B856B866BC00E876F886B01
:105E4000310E896F010E8A6F810E8B6F010E8C6F80
:105E5000BF0E8D6F010E8E6FF20E8F6F010E906F61
:105E60001C0E916F020E926F410E936F020E946F93
:105E7000620E956F020E966F800E976F020E986FEE
:105E80009A0E996F020E9A6FB20E9B6F020E9C6F64
:105E9000C80E9D6F020E9E6FDD0E9F6F020EA06FEB
:105EA000F00EA16F020EA26FA36F030EA46F130E6C
:105EB000A56F030EA66F230EA76F030EA86F320EF9
:105EC000A96F030EAA6F400EAB6F030EAC6F4E0EA0
:105ED000AD6F030EAE6F5B0EAF6F030EB06F670E4C
:105EE000B16F030EB26F730EB36F030EB46F7E0EFD
:105EF000B56F030EB66F890EB76F030EB86F940EB1
:105F0000B96F030EBA6F9E0EBB6F030EBC6FA70E68
:105F1000BD6F030EBE6FB10EBF6F030EC06FBA0E22
:105F2000C16F030EC26FC30EC36F030EC46FC56B88
:105F3000C66BC76BC86BC96BCA6BCB6BCC6BCD6BBD
:105F4000CE6B6A511F0803E2FF0E016E3FD0090EAF
:105F5000F16F6B0EF06F090EF36F810EF26F00019F
:105F6000DCEC0CF0012C2FD0090181510A082AE148
:105F7000825328E1D8906A35036A850FE96E090ECD
:105F80000320EA6EECCF03F0ED52EFCF83F903C0AC
:105F900084F984C9D2F983C9D1F9090ED46F7B0E73
:105FA000D36F00014BEC1AF0090E0901D06F750E8A
:105FB000CF6F0001DBEC14F0012C05D0010E016E57
:105FC000090104D00001FF0E016E09010001120059
:105FD0003A0E09016B6F520E6C6F460E6D6F430ED9
:105FE0006E6F6F6F380E706F300E716F726F736BF4
:105FF0003A0E756F570E766F460E776F430E786FB9
:10600000796F390E7A6F300E7B6F7C6F7D6B3A0E35
:106010007F6F770E806F460E816F826F440E836FA5
:10602000430E846F300E856F866F876F886F896B24
:106030008C6B8B6B8E6B8D6B140E8F6F130E906F42
:10604000120E916F110E926F100E936F0F0E946FD0
:106050000E0E956F0D0E966F0C0E976F0B0E986FC0
:106060000A0E996F090E9A6F080E9B6F070E9C6FB0
:10607000060E9D6F050E9E6F040E9F6F030EA06FA0
:10608000020EA16F010EA26FA36BC60EA46F030ECA
:10609000A56F8C0EA66F030EA76F4B0EA86F030E95
:1060A000A96F020EAA6F030EAB6FAE0EAC6F020E9D
:1060B000AD6F3E0EAE6F020EAF6FFD0EB06F010EF4
:1060C000B16FEF0EB26F010EB36FA30EB46F010E7E
:1060D000B56F7F0EB66F010EB76F5D0EB86F010E14
:1060E000B96F370EBA6F010EBB6F220EBC6F010E77
:1060F000BD6F0E0EBE6F010EBF6FE10EC06FC16BA4
:10610000C90EC26FC36BB10EC46FC56B7C0EC66F78
:10611000C76B5F0EC86FC96B410ECA6FCB6BCC6B80
:10612000CD6B6A5114085BE3090EF16F6B0EF06FD3
:10613000090EF36F8B0EF26F0001DCEC0CF0012CFA
:106140004DD009018B510A0828E18C5326E1D890E3
:106150006A35036AA40FE96E090E0320EA6EECCFDC
:1061600003F0ED52EFCF8DF903C08EF98EC9D2F94D
:106170008DC9D1F9090ED46F850ED36F00014BEC98
:106180001AF0090E0901D06F7F0ECF6F0001DBEC12
:1061900014F0015027D022D009018B5108081FE1CB
:1061A0008C531DE1036A6A518F0FE96E090E0320BB
:1061B000EA6EEFCFCEF9CEC9CFF9090ED16F7B0EC3
:1061C000D06F00019BEC18F0090E0901D06F750E1D
:1061D000CF6F0001DBEC14F0015004D00901FF0E79
:1061E000016E000112003A0E09016B6F570E6C6FC1
:1061F000460E6D6F450E6E6F430E6F6F450E706FDE
:10620000300E716F726F736B6A51020803E1320EC8
:10621000726F02D0300E726F090ED06F6B0ECF6F9F
:106220000001DBEC14F0012C0BD009016A510208CB
:1062300002E14D8601D04D96010E016E04D00001A1
:10624000FF0E016E0901000112003A0E0901776F7D
:10625000520E786F460E796F420E7A6F460E7B6F44
:106260007C6F300E7D6F7E6F7F6B826B816B090E52
:10627000F16F770EF06F090EF36F810EF26F000170
:10628000DCEC0CF0012C27D009017651030802E167
:10629000818301D08193570E786F81C9CFF9090EA0
:1062A000D16F7D0ED06F00019BEC18F0090E090133
:1062B000D06F770ECF6F0001DBEC14F0012C0BD008
:1062C00009017651030802E14D8801D04D98010E75
:1062D000016E04D00001FF0E016E090100011200E1
:1062E0000901796B786B3A0E7A6F520E7B6F460E0E
:1062F0007C6F420E7D6F460E7E6F7F6F300E806F1B
:10630000816F826B76C9E9FF77C9EAFFEF6A090EF0
:10631000F16F7A0EF06F090EF36F780EF26F0001D5
:10632000DCEC0CF0012C16D0090178A308D076C95A
:10633000E9FF77C9EAFF030EEF6E4D8807D076C9F3
:10634000E9FF77C9EAFF020EEF6E4D98010E016E6C
:1063500004D00001FF0E016E0901000112003A0E87
:1063600009016B6F570E6C6F460E6D6F420E6E6FAC
:10637000460E6F6F360E706F300E716F726F736BEB
:10638000756B6A51350803E2FF0E016E3CD0090EB1
:10639000776F750E766F0001A3DF012C31D04DB8F9
:1063A0000DD0030E0901766F00014FDF012C01D0E3
:1063B00005D0FF0E016E090126D000016AC9CFF990
:1063C000090E0901D16F710ED06F00019BEC18F01E
:1063D000090E0901D06F6B0ECF6F0001DBEC14F0DA
:1063E000012C0ED0390E0901706F090ED06F6B0EA3
:1063F000CF6F0001DBEC14F00150090104D0000163
:10640000FF0E016E0901000112003A0E09016A6FC8
:10641000570E6B6F460E6C6F420E6D6F440E6E6FB3
:10642000390E6F6F300E706F716F726B72C0CFF973
:10643000090ED16F700ED06F00019BEC18F0090EA1
:106440000901D06F6A0ECF6F0001DBEC14F0012C54
:106450005BD0410E09016F6F73C0CFF9090ED16F88
:10646000700ED06F00019BEC18F0090E0901D06F7F
:106470006A0ECF6F0001DBEC14F0012C45D0420E08
:1064800009016F6F74C0CFF9090ED16F700ED06F14
:1064900000019BEC18F0090E0901D06F6A0ECF6F56
:1064A0000001DBEC14F0012C2FD0430E09016F6FBB
:1064B00075C0CFF9090ED16F700ED06F00019BEC43
:1064C00018F0090E0901D06F6A0ECF6F0001DBECE6
:1064D00014F0012C19D0440E09016F6F76C0CFF96A
:1064E000090ED16F700ED06F00019BEC18F0090EF1
:1064F0000901D06F6A0ECF6F0001DBEC14F0012CA4
:1065000003D0010E016E02D0FF0E016E7BEF35F05D
:106510003A0E09016A6F570E6B6F460E6C6F420E92
:106520006D6F440E6E6F460E6F6F300E706F716F31
:10653000726B77C0CFF9090ED16F700ED06F00016A
:106540009BEC18F0090E0901D06F6A0ECF6F0001A5
:10655000DBEC14F0012C5DD0450E09016E6F300E9E
:106560006F6F78C0CFF9090ED16F700ED06F000138
:106570009BEC18F0090E0901D06F6A0ECF6F000175
:10658000DBEC14F0012C45D0310E09016F6F79C09E
:10659000CFF9090ED16F700ED06F00019BEC18F08F
:1065A000090E0901D06F6A0ECF6F0001DBEC14F009
:1065B000012C2FD0320E09016F6F7AC0CFF9090E6E
:1065C000D16F700ED06F00019BEC18F0090E09011D
:1065D000D06F6A0ECF6F0001DBEC14F0012C19D0E4
:1065E000330E09016F6F7BC0CFF9090ED16F700EAA
:1065F000D06F00019BEC18F0090E0901D06F6A0EF4
:10660000CF6F0001DBEC14F0012C03D0010E016E02
:1066100002D0FF0E016E82EF35F03A0E09016A6F6B
:10662000570E6B6F460E6C6F420E6D6F430E6E6FA2
:10663000390E6F6F300E706F716F726B6DC0CFF966
:10664000090ED16F700ED06F00019BEC18F0090E8F
:106650000901D06F6A0ECF6F0001DBEC14F0012C42
:106660005BD0410E09016F6F6EC0CFF9090ED16F7B
:10667000700ED06F00019BEC18F0090E0901D06F6D
:106680006A0ECF6F0001DBEC14F0012C45D0420EF6
:1066900009016F6F6FC0CFF9090ED16F700ED06F07
:1066A00000019BEC18F0090E0901D06F6A0ECF6F44
:1066B0000001DBEC14F0012C2FD0430E09016F6FA9
:1066C00070C0CFF9090ED16F700ED06F00019BEC36
:1066D00018F0090E0901D06F6A0ECF6F0001DBECD4
:1066E00014F0012C19D0440E09016F6F71C0CFF95D
:1066F000090ED16F700ED06F00019BEC18F0090EDF
:106700000901D06F6A0ECF6F0001DBEC14F0012C91
:1067100003D0010E016E02D0FF0E016E89EF35F03D
:106720003A0E09016B6F570E6C6F300E6D6F430E92
:106730006E6F370E6F6F706F300E716F726F736B9D
:106740006AC9CFF9090ED16F710ED06F00019BECB1
:1067500018F0090E0901D06F6B0ECF6F0001DBEC52
:1067600014F0012C33D0380E0901706F090ED06F70
:106770006B0ECF6F0001DBEC14F0012C27D0390E2B
:106780000901706F090ED06F6B0ECF6F0001DBEC4B
:1067900014F0012C1BD0410E0901706F090ED06F4F
:1067A0006B0ECF6F0001DBEC14F0012C0FD0420E0A
:1067B0000901706F090ED06F6B0ECF6F0001DBEC1B
:1067C00014F0012C03D0010E016E02D0FF0E016EF9
:1067D00012000901676B666B686B010E696F642DAF
:1067E000D3D0090E6B6F680E6A6F0001E1EC1FF0E9
:1067F000090E09016B6F680E6A6F000150EC20F002
:10680000090E09016B6F680E6A6F00018EEC20F0B3
:10681000090E09016B6F680E6A6F0001CDEC20F064
:106820004DC064F0648F656B666B64A51FD0090E64
:1068300009016B6F680E6A6F000110EC21F0012CEA
:1068400003D068C965F002D009016969090E090120
:106850006B6F680E6A6F00015CEC23F0012C03D0B3
:1068600068C966F003D00901696900016A6B696B48
:106870006C6B6B6B64A323D0090E0901786F660EF5
:10688000776F00017AEC25F0012C05D067C96AF01A
:1068900066C969F002D009016969090E0901786FBA
:1068A000660E776F000166EC26F0012C05D067C9F3
:1068B0006CF066C96BF003D0090169690001676B70
:1068C00064A910D0090E09016B6F680E6A6F000190
:1068D00047EC27F0012C03D068C967F003D0090109
:1068E00069690001686B090E09016B6F680E6A6FB8
:1068F00000017CEC27F0012C03D068C968F003D0BC
:10690000090169690001736B73C072F0766B76C020
:1069100075F075C074F0B0EF27F0012C01D003D0F2
:10692000090169690001786B78C077F07B6B7BC0E7
:106930007AF07AC079F021EF28F0012C01D003D051
:106940000901696900016E6B6EC06DF0716B71C0F9
:1069500070F070C06FF094EF28F0012C01D002D0DD
:10696000090169690901692D09D065C96AF9000140
:106970003BEF29F00150E9D005D00901FF0E016E6F
:106980000001E3D0DFD0090164510208D8A4DBD0B4
:1069900065C96AF90001FDEF29F0012CD0D04EC085
:1069A0006AF94EC04EF064C04DF04DA225D0050EE0
:1069B00009016A6F00010EEC2AF0012C19D06AC09F
:1069C0006BF969C06AF988EC2AF0012C0DD06CC013
:1069D0006BF96BC06AF922EC2BF0012C01D003D0CB
:1069E00009016969000103D009016969000103D047
:1069F0000901696900010BD009016A6B00010EEC05
:106A00002AF0012C01D003D00901696900014DB0C1
:106A10000CD0020E09016A6F000189EC1DF0012CF7
:106A200001D003D00901696900014DA41DD0030EF6
:106A300009016A6F00019BEC2EF0012C14D066C096
:106A40006AF9F6EC2EF0012C0BD065C06AF9E8EC7F
:106A50002FF0012C01D003D009016969000103D096
:106A600009016969000122D009016A6B00019BECF0
:106A70002EF0012C1BD04DA60DD0020E09016A6F1D
:106A80000001F3EC30F0012C01D003D00901696959
:106A900000010CD0030E09016A6F0001F3EC30F025
:106AA000012C01D003D00901696900014DA816D05D
:106AB000030E0901766F000125EC31F0012C0AD09C
:106AC00067C06AF94CDC012C01D003D00901696967
:106AD000000103D00901696900010CD0020E09010F
:106AE000766F000125EC31F0012C01D003D00901B3
:106AF000696900018AD4012C01D003D009016969B8
:106B0000000106D5012C01D003D0090169690001FB
:106B100084D5012C01D003D009016969000168C046
:106B20006AF9FEDD012C01D004D00901696905D0A4
:106B30000001010E016E09D0090105D00001FF0E10
:106B4000016E03D0090169C901F0000141EF37F07E
:106B50000901316B5A6B5B6B010E5C6F5D6F5E6F91
:106B60005F6F616B606B040E2F25E96E000E3021A4
:106B7000EA6EEF500208D8A498D0050E2F25E96ED2
:106B8000000E3021EA6EEFCF62F962C96BF90001A5
:106B9000EEEC1CF0012C83D00B0E0901326F050EB8
:106BA0002F25E96E000E3021EA6EEF500F0B336F88
:106BB000346B090EE36F320EE26F020EE46F0001D8
:106BC000F4EC0FF0050E09012F25E96E000E3021BF
:106BD000EA6E010EEF245B6F48C831F960C062F9BC
:106BE0000001DAEC18F07DA109D0030E09016A6FEB
:106BF000000189EC1DF001C05DF908D0020E090109
:106C00006A6F000189EC1DF001C05DF95BC962F992
:106C1000B8EC1DF001C05CF931C962F9DAEC18F08A
:106C20000901616B606B270E636F100E626F0001CC
:106C300046EC14F0012C01D003D0FF0E016E2BD1D5
:106C4000090EEA6E460EE96E006A026A140E016EC3
:106C50003BEC07F0120E09015A6F090EE36F460E66
:106C6000E26F090EE56F5A0EE46F000129EC10F097
:106C700001C05EF909015C2D13D05D2D11D05F2D8F
:106C80000FD05E2D0DD0050E2F25E96E000E3021A0
:106C9000EA6EEFCF59F0010E016E0001FCD0090140
:106CA000FF0E016E0001F7D00901040E2F25E96ED9
:106CB000000E3021EA6EEF50FB0FD8B070D0050FF8
:106CC00000014CEF37F0050E09012F25E96E000E8B
:106CD0003021EA6E010EEF245B6F090E326F5BC943
:106CE00062F9000164EF1EF0012C01D003D0FF0E09
:106CF000016ED1D0050E09012F25E96E000E30215D
:106D0000EA6EEFCF62F962C963F90001F6EF1EF097
:106D1000090145D0050E09012F25E96E000E30212D
:106D2000EA6E010EEF245B6F0A0E326F5BC962F9E7
:106D3000000134EC1FF0012C01D003D0FF0E016ED6
:106D4000AAD009012CD0FF0E016EA5D0090127D0D1
:106D5000050E09012F25E96E000E3021EA6E200E86
:106D6000EF245B6F5BC962F9000134EC1FF0015046
:106D700092D0090114D0050E09012F25E96E000EED
:106D80003021EA6E200EEF245B6F5BC962F90001CF
:106D9000B8EC1DF001507FD0090101D00901050EAA
:106DA0002F25E96E000E3021EA6EEFCF59F0050E67
:106DB0002F25E96E000E3021EA6EEF500F0B336F76
:106DC000346B090EE36F320EE26F020EE46F0001C6
:106DD000F4EC0FF00901616B606B270E636F100E0E
:106DE000626F000146EC14F0012C01D003D0FF0EBD
:106DF000016E51D0090EEA6E460EE96E006A026A13
:106E0000140E016E3BEC07F0120E09015A6F090EC9
:106E1000E36F460EE26F090EE56F5A0EE46F000154
:106E200029EC10F0012C01D003D0FF0E016E33D0FD
:106E3000040E09012F25E96E000E3021EA6EEF2CB9
:106E400001D009D0040E2F25E96E000E3021EA6E24
:106E5000EF5002081DE1040E2F25E96E000E3021CF
:106E6000EA6EEFCF62F9050E2F25E96E000E302194
:106E7000EA6EEFCF63F962C964F963C965F900018D
:106E8000A8D4012C01D003D0FF0E016E04D009015B
:106E9000010E016E00011200E824F76AF736B90FFF
:106EA000F66E6E0EF722000EF86EFB6E0A00F550BD
:106EB000FA6E0800F550F96EC66C146D466D506D93
:106EC000766D0901316B4CAC28D02FC9E9FF30C970
:106ED000EAFF08013951EF5CD8B402D009011DD096
:106EE0003A39006EF00E0016005080090901316F2A
:106EF0003151000170EC06F009012FC9E9FF30C9DA
:106F0000EAFF700EEF6E30C9E3F92FC9E2F9E46BC6
:106F1000E569000128EC0FF0090100011200AA6ADE
:106F2000A96A5AC0A8FFA69CA69EA684F250006E2D
:106F3000F29E0F01550EA76EAA0EA76EA682A6B2EC
:106F4000FED7A6940050F212AA6A010EA96E5BC089
:106F5000A8FFA69CA69EA684F2CF00F0F29E550E36
:106F6000A76EAA0EA76EA682A6B2FED7A694005060
:106F7000F212AA6A020EA96E5CC0A8FFA69CA69E89
:106F8000A684F2CF00F0F29E550EA76EAA0EA76E51
:106F9000A682A6B2FED7A6940050F212AA6A030EE9
:106FA000A96E5DC0A8FFA69CA69EA684F2CF00F0A5
:106FB000F29E550EA76EAA0EA76EA682A6B2FED7A7
:106FC000A6940050F21262C02FF9AA6A040EA96EAC
:106FD00062C0A8FFA69CA69EA684F2CF00F0F29EF7
:106FE000550EA76EAA0EA76EA682A6B2FED7A694CD
:106FF0000050F21261C02FF9AA6A050EA96E61C095
:10700000A8FFA69CA69EA684F2CF00F0F29E550E85
:10701000A76EAA0EA76EA682A6B2FED7A6940050AF
:10702000F212AA6A060EA96E60C0A8FFA69CA69ED0
:10703000A684F2CF00F0F29E550EA76EAA0EA76EA0
:10704000A682A6B2FED7A6940050F212010E016EDF
:1070500000016AEF49F0010E09013B6F3C6F050E1C
:107060003D6F090E3E6F0D0E3F6F110E406F150EF6
:10707000416F190E426F436B3A0E446F570E456FC6
:10708000460E466F380E476F410E486F300E496FFF
:107090004A6F4B6F4C6B4E6B4F6B5091090EEA6E03
:1070A000310EE96E006A026A0A0E016E00013BECC5
:1070B00007F00901305324E1090EEA6E310EE96E42
:1070C000000E0001F7EC02F00A000900F550EE6E28
:1070D0000009FBE1090E0901D06F310ECF6F0001ED
:1070E000DBEC14F001C04FF909014F2D05D0080168
:1070F00047914793479509014FC901F092D08DD030
:1071000030AB07D03051070B4E6F303B0F0E3017AE
:1071100002D0010E4E6F0801495109014E5D20E079
:10712000036A4E513B0FE96E090E0320EA6EEFCF62
:1071300051F951C9CFF9090ED16F4A0ED06F000134
:107140009BEC18F0090E0901D06F440ECF6F0001BF
:10715000DBEC14F0012C05D04EC949F8090150812F
:1071600000010901305102082CE150B104D008019E
:1071700047B525D00901090EEA6E310EE96E000E01
:10718000000124EC03F00A000900F550EE6E00093E
:10719000FBE1090E0901D06F310ECF6F0001DBEC6E
:1071A00014F001C04FF909014F2D05D008014781A6
:1071B0004793478509014FC901F033D008012ED00C
:1071C00009013051030829E150B104D0080147B347
:1071D00025D00901090EEA6E310EE96E000E00019C
:1071E00033EC03F00A000900F550EE6E0009FBE1F4
:1071F000090E0901D06F310ECF6F0001DBEC14F0E6
:1072000001C04FF909014F2D05D00801478147837F
:10721000479509014FC901F004D00801FF0E016E26
:107220000901000112000901316B326B3051020873
:1072300008E03051030805E0305303E1FF0E016E12
:107240005AD0090E776F320E766F000170EC31F074
:10725000012C01D004D0FF0E016E09014CD00901B0
:10726000305317E13251020803E1010E016E43D0A1
:10727000020E766F000125EC31F0012C06D0010ED4
:10728000016E090138D005D00001FF0E016E090121
:1072900032D0325102080CE1030E766F000125EC6A
:1072A00031F0012C01D005D0FF0E016E090123D071
:1072B0000001090E09016B6F310E6A6F000147EC86
:1072C00027F0012C01D004D0FF0E016E090113D06C
:1072D00009013051020805E131513E0801E3312B2B
:1072E00003D0315301E0310731C96AF90001AFEC35
:1072F00031F001500901000153EF4BF00901326BED
:10730000316B305306E03051020803E0305103087E
:107310002EE1090E786F310E776F00017AEC25F0BF
:10732000012C24D009013051000A000105E0020AB5
:1073300008E0010A0CE012D056C032F955C031F90C
:107340000DD00901312BD8B4322B000107D009012F
:107350003151D8B432073107000100D032C96BF97E
:1073600031C96AF988EC2AF0015003D00901FF0EF7
:10737000016E00011EEF4CF00901326B316B30538E
:1073800006E03051020803E0305103082EE1090EF7
:10739000786F310E776F000166EC26F0012C24D057
:1073A00009013051000A000105E0020A08E0010A63
:1073B0000CE012D058C032F957C031F90DD0090194
:1073C000312BD8B4322B000107D009013151D8B488
:1073D00032073107000100D032C96BF931C96AF9AF
:1073E00022EC2BF0015003D00901FF0E016E0001C9
:1073F00025EF4DF00901316B326B090E6B6F310EC9
:107400006A6F000110EC21F0012C29D031C932F94A
:1074100009013051000A000105E0020A08E0010AF2
:107420000DE012D0090E0901316F00010DD00901E4
:1074300031510A0801E3322B000106D00901315312
:1074400001E03207000100D009013151325D08E04E
:1074500032C96AF90001E8EC2FF0015004D00901AB
:10746000FF0E016E000112000901316B326B090E33
:107470006B6F310E6A6F00015CEC23F0012C30D091
:1074800009013051000A000105E0020A07E0010A83
:107490000EE015D00901326B000111D00901315104
:1074A000230803E3010E3125326F000108D00901E2
:1074B000315303E0010E315D326F000100D009014C
:1074C0003251315D09E032C96AF90001F6EC2EF063
:1074D000015008D005D00901010E016E000102D053
:1074E000FF0E016E4AEF4FF03A0E0901316F570E51
:1074F000326F460E336F346F330E356F366F300E8A
:10750000376F386F396B3051020803E1310E386F35
:1075100002D0300E386F090ED06F310ECF6F0001E0
:10752000DBEC14F0012C0BD009013051020802E110
:107530004F8601D04F96010E016E04D00001FF0E60
:10754000016E0901000169EF50F03A0E0901326F36
:10755000520E336F460E346F380E356F360E366F5F
:10756000300E376F386F396F3A6B3A0E3C6F570EEB
:107570003D6F460E3E6F380E3F6F350E406F430E27
:10758000416F300E426F310E436F446B3A0E466FBF
:10759000770E476F460E486F380E496F350E4A6FAB
:1075A000410E4B6F300E4C6F4D6F4E6F4F6F506BE7
:1075B000536B526B54914DA0BBD0090EF16F320E3C
:1075C000F06F090EF36F520EF26F0001DCEC0CF05D
:1075D000012C50D00901522D4CD053534AE1090ED1
:1075E000D06F3C0ECF6F0001DBEC14F0012C42D0C9
:1075F0000801476B0901536B526B54B13AD00A0E24
:107600000C01B66F00016BEC07F0090E0901F16F78
:10761000320EF06F090EF36F520EF26F0001DCECC8
:107620000CF0012C24D009015251006E5351036E0D
:10763000035005E1010E005C00010FE00901035059
:1076400005E1020E005C00010AE00901035004E1BB
:107650000052000109E009010AD0090108D0FF0E1B
:10766000016E68D0090103D00901548100D00901DD
:10767000C4D7000130C9D2F92FC9D1F9090E0901C7
:10768000D46F4C0ED36F00014BEC1AF0090E0901B8
:10769000D06F460ECF6F0001DBEC14F0012C46D00A
:1076A0000901536B526B549154B13FD00A0E0C0137
:1076B000B66F00016BEC07F0090E0901F16F320E95
:1076C000F06F090EF36F520EF26F0001DCEC0CF05C
:1076D000012C29D009015251006E5351036E035001
:1076E00005E1010E005C00010FE00901035005E116
:1076F000020E005C00010AE00901035004E100529F
:1077000000010CE009010FD009010DD009015481DD
:10771000FF0E016E00010ED0090105D0010E016EB1
:1077200009D0090100D00901BFD7000100D009012B
:10773000FF0E016E000148EF51F00901316B306B13
:107740003A0E326F520E336F460E346F420E356F63
:10775000430E366F390E376F300E386F396F3A6B14
:107760003A0E3C6F570E3D6F460E3E6F420E3F6F16
:10777000430E406F390E416F300E426F436F446BC2
:10778000476B466B496B486B2F515F0803E2FF0E56
:10779000016ECFD0090EF16F320EF06F090EF36F4C
:1077A000300EF26F0001DCEC0CF0012CBFD00901AF
:1077B0002F51305D05E1315303E1010E016EB9D067
:1077C000036A2FC946F903C047F9280E465D4A6F80
:1077D000000E47594B6F036E4A514BAF08D0000E55
:1077E000D8804A55006E000E4B55036E0050466F10
:1077F00003C047F92F51270805E3461F471F462BB3
:10780000D8B4472B280E4625486F000E4721496FF4
:1078100048C94AF948C9CFF9090ED16F420ED06F55
:1078200000019BEC18F0090E0901D06F3C0ECF6FE0
:107830000001DBEC14F0012C79D0410E0901416FFD
:10784000380E4625486F000E4721496F48C94AF94E
:1078500048C9CFF9090ED16F420ED06F00019BECE1
:1078600018F0090E0901D06F3C0ECF6F0001DBEC60
:1078700014F0012C5BD0420E0901416F400E4625E9
:10788000486F000E4721496F48C94AF948C9CFF9E6
:10789000090ED16F420ED06F00019BEC18F0090E5B
:1078A0000901D06F3C0ECF6F0001DBEC14F0012C0E
:1078B0003DD0430E0901416F4625486F000E472118
:1078C000496F48C94AF948C9CFF9090ED16F420E2C
:1078D000D06F00019BEC18F0090E0901D06F3C0E2F
:1078E000CF6F0001DBEC14F0012C20D0440E090115
:1078F000416F480E4625486F000E4721496F48C921
:107900004AF948C9CFF9090ED16F420ED06F000174
:107910009BEC18F0090E0901D06F3C0ECF6F0001EF
:10792000DBEC14F00150090104D00001FF0E016EE0
:107930000901000112000901316B306B3A0E326F00
:10794000520E336F460E346F420E356F440E366F53
:10795000376F300E386F396F3A6B3A0E3C6F570EF7
:107960003D6F460E3E6F420E3F6F440E406F390E24
:10797000416F300E426F436F446B476B466B496BF0
:10798000486B2F51CF0803E2FF0E016EACD0090EF9
:10799000F16F320EF06F090EF36F300EF26F0001CF
:1079A000DCEC0CF0012C9CD009012F51305D05E17D
:1079B000315303E1010E016E96D0036A2FC946F9D7
:1079C00003C047F9700E465D4A6F000E47594B6F72
:1079D000036E4A514BAF08D0000ED8804A55006E56
:1079E000000E4B55036E0050466F03C047F92F51F0
:1079F0006F0805E3461F471F462BD8B4472BA00E40
:107A00004625486F000E4721496F48C94AF948C9C1
:107A1000CFF9090ED16F420ED06F00019BEC18F028
:107A2000090E0901D06F3C0ECF6F0001DBEC14F0A2
:107A3000012C56D0410E0901416F090ED06F3C0E4A
:107A4000CF6F0001DBEC14F0012C4AD0420E09018B
:107A5000416F900E4625486F000E4721496F48C977
:107A60004AF948C9CFF9090ED16F420ED06F000113
:107A70009BEC18F0090E0901D06F3C0ECF6F00018E
:107A8000DBEC14F0012C2CD0430E0901416F700E79
:107A90004625486F000E4721496F48C94AF948C931
:107AA000CFF9090ED16F420ED06F00019BEC18F098
:107AB000090E0901D06F3C0ECF6F0001DBEC14F012
:107AC000012C0ED0440E0901416F090ED06F3C0EFF
:107AD000CF6F0001DBEC14F00150090104D000016C
:107AE000FF0E016E0901000112000901316B306BBC
:107AF0003A0E326F520E336F460E346F420E356FB0
:107B0000450E366F330E376F300E386F396F3A6B64
:107B10003A0E3C6F570E3D6F460E3E6F420E3F6F62
:107B2000440E406F460E416F300E426F436F446B00
:107B3000476B466B496B486B2F51AF0803E2FF0E52
:107B4000016EAED0090EF16F320EF06F090EF36FB9
:107B5000300EF26F0001DCEC0CF0012C9ED009011C
:107B60002F51305D05E1315303E1010E016E98D0D4
:107B7000036A2FC946F903C047F9500E465D4A6FA4
:107B8000000E47594B6F036E4A514BAF08D0000EA1
:107B9000D8804A55006E000E4B55036E0050466F5C
:107BA00003C047F92F514F0805E3461F471F462BD7
:107BB000D8B4472BA00E4625486F000E4721496FC9
:107BC00048C94AF948C9CFF9090ED16F420ED06FA2
:107BD00000019BEC18F0090E0901D06F3C0ECF6F2D
:107BE0000001DBEC14F0012C58D0450E0901406F68
:107BF000300E416F090ED06F3C0ECF6F0001DBECF1
:107C000014F0012C4AD0310E0901416F800E462537
:107C1000486F000E4721496F48C94AF948C9CFF952
:107C2000090ED16F420ED06F00019BEC18F0090EC7
:107C30000901D06F3C0ECF6F0001DBEC14F0012C7A
:107C40002CD0320E0901416F500E4625486F000EB0
:107C50004721496F48C94AF948C9CFF9090ED16F80
:107C6000420ED06F00019BEC18F0090E0901D06F95
:107C70003C0ECF6F0001DBEC14F0012C0ED0330E64
:107C80000901416F090ED06F3C0ECF6F0001DBEC94
:107C900014F00150090104D00001FF0E016E09012A
:107CA000000112000901026B016B2B6B2C6B2D6B19
:107CB000020E0801FF25E96E000E09010021EA6E9F
:107CC000EFCF2EF9030E0801FF25E96E000E090122
:107CD0000021EA6EEFCF2FF92FC92BF94DBE10D03E
:107CE0002B5100080DE0040E0801FF25E96E000E7F
:107CF00009010021EA6EEF50020802E0E3EF5DF0B7
:107D0000020E0801FF25E96E000E09010021EA6E4E
:107D1000EF500608D8A467EF44F085A611D0FFC83D
:107D2000E9FF090100C9EAFFEFCF2EF9010E476F05
:107D30002EC948F90001DCEC13F00901E3EF5DF016
:107D4000030E0801FF25E96E000E09010021EA6E0D
:107D5000EF50010A000119E0030AD8B4B7D0010AB4
:107D6000D8B4A4D1070AD8B48DD2010AD8B4D0D2DD
:107D7000020AD8B413D30F0AD8B448EF43F0060A66
:107D8000D8B4AFEF43F056EF44F0080E0801FF25DA
:107D9000E96E000E09010021EA6EEF3C8AD0FFC8AF
:107DA000E9FF090100C9EAFFEFCF2EF9010E306F9C
:107DB0002EC931F90001FBEC13F0010E0901036F2C
:107DC000040E0801FF25E96E000E09010021EA6E8C
:107DD000EFCF04F9050E0801FF25E96E000E090139
:107DE0000021EA6EEFCF05F9060E0801FF25E96EC6
:107DF000000E09010021EA6EEFCF06F9070E080117
:107E0000FF25E96E000E09010021EA6EEFCF07F9A8
:107E10004AA236D0060E0801FF25E96E000E0901C0
:107E20000021EA6EEF50030810E0060E0801FF255E
:107E3000E96E000E09010021EA6EEF50020803E12D
:107E4000010E066F02D0020E066F070E0801FF2515
:107E5000E96E000E09010021EA6EEF50030810E000
:107E6000070E0801FF25E96E000E09010021EA6EE8
:107E7000EF50020803E1010E076F02D0020E076FF8
:107E8000086B090EE36F030EE26F050EE46F00014D
:107E9000F4EC0FF0FFC8E9FF090100C9EAFFEFCFDA
:107EA0002EF9010E306F2EC931F9000118EC14F0D3
:107EB0000BD0FFC8E9FF00C9EAFFEFCF2EF92EC9AA
:107EC00047F90001C3EC13F065EF44F00E0E080112
:107ED000FF25E96E000E09010021EA6EEF3CD9D0C2
:107EE000FFC8E9FF090100C9EAFFEFCF2EF9010E33
:107EF000306F2EC931F90001FBEC13F0020E0901BD
:107F0000036F040E0801FF25E96E000E0901002130
:107F1000EA6EEFCF04F9050E0801FF25E96E000EA9
:107F200009010021EA6EEFCF05F9060E0801FF25D1
:107F3000E96E000E09010021EA6EEFCF06F9070E87
:107F40000801FF25E96E000E09010021EA6EEFCF5E
:107F500007F9080E0801FF25E96E000E090100214E
:107F6000EA6EEFCF08F9090E0801FF25E96E000E51
:107F700009010021EA6EEFCF09F90A0E0801FF2579
:107F8000E96E000E09010021EA6EEFCF0AF90B0E2F
:107F90000801FF25E96E000E09010021EA6EEFCF0E
:107FA0000BF90C0E0801FF25E96E000E09010021F6
:107FB000EA6EEFCF0CF90D0E0801FF25E96E000EF9
:107FC00009010021EA6EEFCF0DF90E6B090EE36F88
:107FD000030EE26F0B0EE46F0001F4EC0FF0270EBE
:107FE0000901636F100E626F000146EC14F0012C62
:107FF0003FD0090EEA6E170EE96E006A026A140E8F
:10800000016E3BEC07F0120E09012C6F090EE36FB5
:10801000170EE26F090EE56F2C0EE46F000129ECDC
:1080200010F0012C12D0FFC8E9FF090100C9EAFFD6
:10803000EFCF2EF9010E306F2EC931F9000118EC87
:1080400014F00901E3EF5DF00FD0FFC8E9FF09016B
:1080500000C9EAFFEFCF2EF9010E476F2EC948F98C
:108060000001DCEC13F00901E3EF5DF012D0000138
:10807000FFC8E9FF090100C9EAFFEFCF2EF9010EA1
:10808000476F2EC948F90001DCEC13F00901E3EF5A
:108090005DF0FFC8E9FF00C9EAFFEFCF2EF92EC956
:1080A00047F90001C3EC13F065EF44F00E0E080130
:1080B000FF25E96E000E09010021EA6EEF3CD6D0E3
:1080C000FFC8E9FF090100C9EAFFEFCF2EF9010E51
:1080D000306F2EC931F90001FBEC13F0030E0901DA
:1080E000036F040E0801FF25E96E000E090100214F
:1080F000EA6EEFCF04F9050E0801FF25E96E000EC8
:1081000009010021EA6EEFCF05F9060E0801FF25EF
:10811000E96E000E09010021EA6EEFCF06F9070EA5
:108120000801FF25E96E000E09010021EA6EEFCF7C
:1081300007F9080E0801FF25E96E000E090100216C
:10814000EA6EEFCF08F9090E0801FF25E96E000E6F
:1081500009010021EA6EEFCF09F90A0E0801FF2597
:10816000E96E000E09010021EA6EEFCF0AF90B0E4D
:108170000801FF25E96E000E09010021EA6EEFCF2C
:108180000BF90C0E0801FF25E96E000E0901002114
:10819000EA6EEFCF0CF90D0E0801FF25E96E000E17
:1081A00009010021EA6EEFCF0DF90E6B090EE36FA6
:1081B000030EE26F0B0EE46F0001F4EC0FF0270EDC
:1081C0000901636F100E626F000146EC14F0012C80
:1081D0003CD0090EEA6E170EE96E006A026A140EB0
:1081E000016E3BEC07F0120E09012C6F090EE36FD4
:1081F000170EE26F090EE56F2C0EE46F000129ECFB
:1082000010F0012C0FD0FFC8E9FF090100C9EAFFF7
:10821000EFCF2EF9010E306F2EC931F9000118ECA5
:1082200014F00ED0FFC8E9FF090100C9EAFFEFCF43
:108230002EF9010E476F2EC948F90001DCEC13F04E
:108240000901E3EF5DF012D00001FFC8E9FF090169
:1082500000C9EAFFEFCF2EF9010E476F2EC948F98A
:108260000001DCEC13F00901E3EF5DF0FFC8E9FF6A
:1082700000C9EAFFEFCF2EF92EC947F90001C3EC80
:1082800013F023D3040E0801FF25E96E000E090147
:108290000021EA6EEF3C30D0FFC8E9FF090100C9B8
:1082A000EAFFEFCF2EF9010E306F2EC931F9000130
:1082B000FBEC13F075EC14F0012C0FD0FFC8E9FFB4
:1082C000090100C9EAFFEFCF2EF9010E306F2EC968
:1082D00031F9000118EC14F00ED0FFC8E9FF0901D4
:1082E00000C9EAFFEFCF2EF9010E476F2EC948F9FA
:1082F0000001DCEC13F00BD0FFC8E9FF00C9EAFF76
:10830000EFCF2EF92EC947F90001C3EC13F0DDD2EF
:10831000040E0801FF25E96E000E09010021EA6E36
:10832000EF3C30D0FFC8E9FF090100C9EAFFEFCFF9
:108330002EF9010E306F2EC931F90001FBEC13F05C
:108340009DEC14F0012C0FD0FFC8E9FF090100C912
:10835000EAFFEFCF2EF9010E306F2EC931F900017F
:1083600018EC14F00ED0FFC8E9FF090100C9EAFFBC
:10837000EFCF2EF9010E476F2EC948F90001DCEC52
:1083800013F00BD0FFC8E9FF00C9EAFFEFCF2EF9C9
:108390002EC947F90001C3EC13F097D20E0E080165
:1083A000FF25E96E000E09010021EA6EEF3C64D161
:1083B000040E0801FF25E96E000E09010021EA6E96
:1083C000EF52D8A4D0D0FFC8E9FF090100C9EAFFE5
:1083D000EFCF2EF9010E306F2EC931F90001FBEC01
:1083E00013F0060E0901036F050E0801FF25E96E63
:1083F000000E09010021EA6EEFCF04F9060E080114
:10840000FF25E96E000E09010021EA6EEFCF05F9A4
:10841000070E0801FF25E96E000E09010021EA6E32
:10842000EFCF06F9080E0801FF25E96E000E0901DD
:108430000021EA6EEFCF07F9090E0801FF25E96E6A
:10844000000E09010021EA6EEFCF08F90A0E0801BB
:10845000FF25E96E000E09010021EA6EEFCF09F950
:108460000B0E0801FF25E96E000E09010021EA6EDE
:10847000EFCF0AF90C0E0801FF25E96E000E090185
:108480000021EA6EEFCF0BF90D0E0801FF25E96E12
:10849000000E09010021EA6EEFCF0CF90D6B090EF9
:1084A000E36F030EE26F0A0EE46F0001F4EC0FF0CD
:1084B000270E0901636F100E626F000146EC14F085
:1084C000012C3FD0090EEA6E170EE96E006A026AAF
:1084D000140E016E3BEC07F0120E09012C6F090E11
:1084E000E36F170EE26F090EE56F2C0EE46F0001CB
:1084F00029EC10F0012C12D0FFC8E9FF090100C9D6
:10850000EAFFEFCF2EF9010E306F2EC931F90001CD
:1085100018EC14F00901E3EF5DF00FD0FFC8E9FF9C
:10852000090100C9EAFFEFCF2EF9010E476F2EC9EE
:1085300048F90001DCEC13F00901E3EF5DF012D023
:108540000001FFC8E9FF090100C9EAFFEFCF2EF9DA
:10855000010E476F2EC948F90001DCEC13F0090148
:10856000E3EF5DF089D0040E0801FF25E96E000EEF
:1085700009010021EA6EEF2C7FD0FFC8E9FF090155
:1085800000C9EAFFEFCF2EF9010E306F2EC931F985
:108590000001FBEC13F0070E0901036F050E080143
:1085A000FF25E96E000E09010021EA6EEFCF04F904
:1085B000056B090EE36F030EE26F020EE46F00011C
:1085C000F4EC0FF0270E0901636F100E626F0001CB
:1085D00046EC14F0012C3FD0090EEA6E170EE96E3E
:1085E000006A026A140E016E3BEC07F0120E0901DC
:1085F0002C6F090EE36F170EE26F090EE56F2C0E5C
:10860000E46F000129EC10F0012C12D0FFC8E9FF43
:10861000090100C9EAFFEFCF2EF9010E306F2EC914
:1086200031F9000118EC14F00901E3EF5DF00FD00F
:10863000FFC8E9FF090100C9EAFFEFCF2EF9010EDB
:10864000476F2EC948F90001DCEC13F00901E3EF94
:108650005DF012D00001FFC8E9FF090100C9EAFF7F
:10866000EFCF2EF9010E476F2EC948F90001DCEC5F
:1086700013F00901E3EF5DF0FFC8E9FF00C9EAFF6D
:10868000EFCF2EF92EC947F90001C3EC13F01DD12D
:10869000050E0801FF25E96E000E09010021EA6EB2
:1086A000EF3C50D084A62DD0040E0801FF25E96EC2
:1086B000000E09010021EA6EEF50020A000105E0F8
:1086C000010A06E0130A07E00ED04E9CF0861AD08D
:1086D0004E8CF09617D04EAC03D04E9CF08602D054
:1086E0004E8CF0960FD0FFC8E9FF00C9EAFFEFCF2C
:1086F0002EF92EC947F90001C3EC13F00901E3EF8D
:108700005DF00001FFC8E9FF090100C9EAFFEFCFF2
:108710002EF9010E306F2EC931F90001FBEC13F078
:10872000FFC8E9FF090100C9EAFFEFCF2EF9010EEA
:10873000306F2EC931F9000118EC14F00901E3EF94
:108740005DF00BD0FFC8E9FF00C9EAFFEFCF2EF9BB
:108750002EC947F90001C3EC13F00001B6D0040E96
:108760000801FF25E96E000E09010021EA6EEF50B5
:10877000020816E0040E0801FF25E96E000E09014B
:108780000021EA6EEF500308D8A480D0050E08013E
:10879000FF25E96E000E09010021EA6EEF3C76D05C
:1087A000FFC8E9FF090100C9EAFFEFCF2EF9010E6A
:1087B000306F2EC931F90001FBEC13F0150E0901E1
:1087C000036F040E0801FF25E96E000E0901002168
:1087D000EA6EEFCF04F9056B090EE36F030EE26F4B
:1087E000020EE46F0001F4EC0FF0270E0901636F35
:1087F000100E626F000146EC14F0012C38D0090E07
:10880000EA6E170EE96E006A026A140E016E3BEC06
:1088100007F0120E09012C6F090EE36F170EE26FBD
:10882000090EE56F2C0EE46F000129EC10F0012C0D
:108830000FD0FFC8E9FF090100C9EAFFEFCF2EF909
:10884000010E306F2EC931F9000118EC14F00ED072
:10885000FFC8E9FF090100C9EAFFEFCF2EF9010EB9
:10886000476F2EC948F90001DCEC13F00ED0FFC8A9
:10887000E9FF090100C9EAFFEFCF2EF9010E476FAA
:108880002EC948F90001DCEC13F00BD0FFC8E9FF5A
:1088900000C9EAFFEFCF2EF92EC947F90001C3EC5A
:1088A00013F00901E3EF5DF000010FD0FFC8E9FF0D
:1088B00000C9EAFFEFCF2EF92EC947F90001C3EC3A
:1088C00013F00901E3EF5DF00001E2EF5DF0020E4D
:1088D0000801FF25E96E000E09010021EA6EEF5044
:1088E0000408D8A479EF56F0030E0801FF25E96EBD
:1088F000000E09010021EA6EEF50070A0001D8B40A
:10890000D5D0400AD8B426D1470AD8B4CCD1010A70
:10891000D8B467D2600AD8B403D35E0AD8B49FD360
:108920001D0AD8B4E3EF48F02A0AD8B479EF49F029
:10893000300AD8B4CDEF49F00D0AD8B4D2EF4AF0DE
:10894000370AD8B42CEF4BF0400AD8B48CEF4BF078
:10895000410AD8B4F7EF4BF0400AD8B451EF4CF0CD
:10896000470AD8B4FEEF4CF0400AD8B458EF4DF0A7
:108970007D0AD8B405EF4EF0320AD8B45FEF4EF05E
:10898000400AD8B4B9EF4EF0470AD8B423EF4FF0FD
:10899000400AD8B47DEF4FF07F0AD8B4E8EF4FF02B
:1089A000510AD8B442EF50F0010AD8B496EF50F013
:1089B0002B0AD8B4CCEF50F0080AD8B47BEF51F0B2
:1089C000010AD8B499EF51F0470AD8B4B7EF51F083
:1089D000300AD8B4D5EF51F0700AD8B4F3EF51F0A3
:1089E0005E0AD8B411EF52F0300AD8B42FEF52F02B
:1089F000700AD8B44DEF52F00F0AD8B46BEF52F0B2
:108A0000700AD8B489EF52F03E0AD8B4A6EF52F0FB
:108A1000430AD8B4C3EF52F0500AD8B4E0EF52F092
:108A2000400AD8B433EF53F0470AD8B497EF53F065
:108A3000400AD8B4B4EF53F0730AD8B4D1EF53F06E
:108A4000300AD8B454EF54F0400AD8B4B8EF54F018
:108A5000170AD8B42CEF55F0700AD8B449EF55F086
:108A6000780AD8B466EF55F0440AD8B483EF55F0CD
:108A7000660AD8B4A0EF55F0070AD8B4BDEF55F098
:108A8000010AD8B4DAEF55F0620AD8B4F7EF55F01E
:108A90007C0AD8B414EF56F0070AD8B431EF56F078
:108AA000010AD8B44EEF56F06BEF56F0050E0801F0
:108AB000FF25E96E000E09010021EA6EEF3C3DD072
:108AC000FFC8E9FF090100C9EAFFEFCF2EF9010E47
:108AD000306F2EC931F90001FBEC13F0040E0801D0
:108AE000FF25E96E000E09010021EA6EEFCF2EF995
:108AF0002EC930F9000198EC19F0012C0FD0FFC8F5
:108B0000E9FF090100C9EAFFEFCF2EF9010E306F2E
:108B10002EC931F9000118EC14F00ED0FFC8E9FF9E
:108B2000090100C9EAFFEFCF2EF9010E476F2EC9E8
:108B300048F90001DCEC13F00BD0FFC8E9FF00C9D5
:108B4000EAFFEFCF2EF92EC947F90001C3EC13F06D
:108B500077EF56F0080E0801FF25E96E000E0901B7
:108B60000021EA6EEF3C92D0FFC8E9FF090100C97D
:108B7000EAFFEFCF2EF9010E306F2EC931F9000157
:108B8000FBEC13F0040E0801FF25E96E000E09014D
:108B90000021EA6EEF50036A016F03C002F901354C
:108BA0002E6F02352F6F2E372F372E372F372E3758
:108BB0002F37F00E2E17050E0801FF25E96E000E67
:108BC00009010021EA6EEF500F0B2E11016F2FC922
:108BD00002F901352E6F02352F6F2E372F372E37C2
:108BE0002F372E372F37F00E2E17060E0801FF25D0
:108BF000E96E000E09010021EA6EEF500F0B2E11F5
:108C0000016F2FC902F901352E6F02352F6F2E37F4
:108C10002F372E372F372E372F37F00E2E17070E00
:108C20000801FF25E96E000E09010021EA6EEF50F0
:108C30000F0B2E11016F2FC902F902C931F901C9B9
:108C400030F9070E326F000109EC1BF0012C0FD038
:108C5000FFC8E9FF090100C9EAFFEFCF2EF9010EB5
:108C6000306F2EC931F9000118EC14F00ED0FFC896
:108C7000E9FF090100C9EAFFEFCF2EF9010E476FA6
:108C80002EC948F90001DCEC13F00BD0FFC8E9FF56
:108C900000C9EAFFEFCF2EF92EC947F90001C3EC56
:108CA00013F077EF56F0050E0801FF25E96E000E70
:108CB00009010021EA6EEF3C87D0040E0801FF2570
:108CC000E96E000E09010021EA6EEF50020832E160
:108CD0002F6B00014DEC1CF0012C1DD0FFC8E9FFEB
:108CE000090100C9EAFFEFCF2EF9010E306F2EC93E
:108CF00031F90001FBEC13F0FFC8E9FF090100C9DD
:108D0000EAFFEFCF2EF9010E306F2EC931F90001C5
:108D100018EC14F00ED0FFC8E9FF090100C9EAFF02
:108D2000EFCF2EF9010E476F2EC948F90001DCEC98
:108D300013F049D0040E0801FF25E96E000E090169
:108D40000021EA6EEF50030833E1010E2F6F00019E
:108D50004DEC1CF0012C1DD0FFC8E9FF090100C932
:108D6000EAFFEFCF2EF9010E306F2EC931F9000165
:108D7000FBEC13F0FFC8E9FF090100C9EAFFEFCFE0
:108D80002EF9010E306F2EC931F9000118EC14F0E4
:108D90000ED0FFC8E9FF090100C9EAFFEFCF2EF9A5
:108DA000010E476F2EC948F90001DCEC13F00BD01F
:108DB000FFC8E9FF00C9EAFFEFCF2EF92EC947F936
:108DC0000001C3EC13F00BD0FFC8E9FF00C9EAFFB4
:108DD000EFCF2EF92EC947F90001C3EC13F077EF5E
:108DE00056F0050E0801FF25E96E000E090100216D
:108DF000EA6EEF3C88D0040E0801FF25E96E000EF4
:108E000009010021EA6EEF50020833E1020E2F6FD4
:108E1000000191EC1CF0012C1DD0FFC8E9FF0901F5
:108E200000C9EAFFEFCF2EF9010E306F2EC931F9DC
:108E30000001FBEC13F0FFC8E9FF090100C9EAFFDC
:108E4000EFCF2EF9010E306F2EC931F9000118EC69
:108E500014F00ED0FFC8E9FF090100C9EAFFEFCF07
:108E60002EF9010E476F2EC948F90001DCEC13F012
:108E700049D0040E0801FF25E96E000E090100210A
:108E8000EA6EEF50030833E1030E2F6F000191ECFF
:108E90001CF0012C1DD0FFC8E9FF090100C9EAFF41
:108EA000EFCF2EF9010E306F2EC931F90001FBEC26
:108EB00013F0FFC8E9FF090100C9EAFFEFCF2EF95F
:108EC000010E306F2EC931F9000118EC14F00ED0EC
:108ED000FFC8E9FF090100C9EAFFEFCF2EF9010E33
:108EE000476F2EC948F90001DCEC13F00BD0FFC826
:108EF000E9FF00C9EAFFEFCF2EF92EC947F90001BB
:108F0000C3EC13F00BD0FFC8E9FF00C9EAFFEFCFB5
:108F10002EF92EC947F90001C3EC13F077EF56F094
:108F2000050E0801FF25E96E000E09010021EA6E19
:108F3000EF3C88D0040E0801FF25E96E000E090100
:108F40000021EA6EEF50020833E1020E2F6F00019C
:108F5000BBEC1CF0012C1DD0FFC8E9FF090100C9C2
:108F6000EAFFEFCF2EF9010E306F2EC931F9000163
:108F7000FBEC13F0FFC8E9FF090100C9EAFFEFCFDE
:108F80002EF9010E306F2EC931F9000118EC14F0E2
:108F90000ED0FFC8E9FF090100C9EAFFEFCF2EF9A3
:108FA000010E476F2EC948F90001DCEC13F049D0DF
:108FB000040E0801FF25E96E000E09010021EA6E8A
:108FC000EF50030833E1030E2F6F0001BBEC1CF0E0
:108FD000012C1DD0FFC8E9FF090100C9EAFFEFCF4E
:108FE0002EF9010E306F2EC931F90001FBEC13F0A0
:108FF000FFC8E9FF090100C9EAFFEFCF2EF9010E12
:10900000306F2EC931F9000118EC14F00ED0FFC8F2
:10901000E9FF090100C9EAFFEFCF2EF9010E476F02
:109020002EC948F90001DCEC13F00BD0FFC8E9FFB2
:1090300000C9EAFFEFCF2EF92EC947F90001C3ECB2
:1090400013F00BD0FFC8E9FF00C9EAFFEFCF2EF9FC
:109050002EC947F90001C3EC13F077EF56F085A64F
:1090600012D0FFC8E9FF090100C9EAFFEFCF2EF9CE
:10907000010E476F2EC948F90001DCEC13F009011D
:10908000E3EF5DF00001060E0801FF25E96E000E1A
:1090900009010021EA6EEF3C88D00AD0040E0801D5
:1090A000FF25E96E000E09010021EA6E00A07DD0C7
:1090B000040E0801FF25E96E000E09010021EA6E89
:1090C000EF50040872E3050E0801FF25E96E000E5B
:1090D00009010021EA6EEF50F00B3BE1FFC8E9FF08
:1090E000090100C9EAFFEFCF2EF9010E306F2EC93A
:1090F00031F90001FBEC13F000C930F9FFC82FF97A
:10910000A8EC35F0012C13D0FFC8E9FF090100C914
:10911000EAFFEFCF2EF9010E306F2EC931F90001B1
:1091200018EC14F00901E3EF5DF012D00001FFC864
:10913000E9FF090100C9EAFFEFCF2EF9010E476FE1
:109140002EC948F90001DCEC13F00901E3EF5DF0F2
:109150002BD0050E0801FF25E96E000E0901002144
:10916000EA6EEF50700814E2050E0801FF25E96E63
:10917000000E09010021EA6EEF50730809E300C9EF
:1091800030F9FFC82FF9000161EC37F00CD009016C
:10919000FFC8E9FF00C9EAFFEFCF2EF92EC947F952
:1091A0000001C3EC13F009010BD0FFC8E9FF00C9AF
:1091B000EAFFEFCF2EF92EC947F90001C3EC13F0F7
:1091C000000177EF56F0080E0801FF25E96E000E4A
:1091D00009010021EA6EEF3C7FD0FFC8E9FF0901D9
:1091E00000C9EAFFEFCF2EF9010E306F2EC931F919
:1091F0000001FBEC13F0040E0801FF25E96E000EE0
:1092000009010021EA6EEF50036A016F03C002F901
:1092100001352E6F02352F6F2E372F372E372F3710
:109220002E372F37F00E2E17050E0801FF25E96E99
:10923000000E09010021EA6EEF500F0B2E11016F95
:109240002FC902F901352E6F02352F6F2E372F37B8
:109250002E372F372E372F37F00E2E17060E080118
:10926000FF25E96E000E09010021EA6EEF500F0B99
:109270002E11016F2FC902F901352E6F02352F6FA4
:109280002E372F372E372F372E372F37F00E2E173A
:10929000070E0801FF25E96E000E09010021EA6EA4
:1092A000EF500F0B2E11016F2FC902F902C962F0A6
:1092B00001C961F0FFC8E9FF090100C9EAFFEFCF6A
:1092C0002EF9010E306F2EC931F9000118EC14F09F
:1092D0008FEF37F00CD00901FFC8E9FF00C9EAFFA2
:1092E000EFCF2EF92EC947F90001C3EC13F077EF49
:1092F00056F0050E0801FF25E96E000E0901002158
:10930000EA6EEF3C3DD0FFC8E9FF090100C9EAFF62
:10931000EFCF2EF9010E306F2EC931F90001FBECB1
:1093200013F0040E0801FF25E96E000E090100216B
:10933000EA6EEFCF2EF92EC930F900012BEC38F090
:10934000012C0FD0FFC8E9FF090100C9EAFFEFCFE8
:109350002EF9010E306F2EC931F9000118EC14F00E
:109360000ED0FFC8E9FF090100C9EAFFEFCF2EF9CF
:10937000010E476F2EC948F90001DCEC13F00BD049
:10938000FFC8E9FF00C9EAFFEFCF2EF92EC947F960
:109390000001C3EC13F077EF56F0050E0801FF252E
:1093A000E96E000E09010021EA6EEF3CEDD0040EDB
:1093B0000801FF25E96E000E09010021EA6EEF5059
:1093C000020817E0040E0801FF25E96E000E0901EE
:1093D0000021EA6EEF5003080CE0040E0801FF259F
:1093E000E96E000E09010021EA6EEF501008D8A4C2
:1093F000CAD0FFC8E9FF090100C9EAFFEFCF2EF983
:10940000010E306F2EC931F90001FBEC13F0040E90
:109410000801FF25E96E000E09010021EA6EEF50F8
:10942000020826E1020E6A6F000189EC1DF0012C92
:1094300010D04D90FFC8E9FF090100C9EAFFEFCF46
:109440002EF9010E306F2EC931F9000118EC14F01D
:109450000ED0FFC8E9FF090100C9EAFFEFCF2EF9DE
:10946000010E476F2EC948F90001DCEC13F08AD0D9
:10947000040E0801FF25E96E000E09010021EA6EC5
:10948000EF50030826E1030E6A6F000189EC1DF01E
:10949000012C10D04D80FFC8E9FF090100C9EAFF87
:1094A000EFCF2EF9010E306F2EC931F9000118EC03
:1094B00014F00ED0FFC8E9FF090100C9EAFFEFCFA1
:1094C0002EF9010E476F2EC948F90001DCEC13F0AC
:1094D00059D0040E0801FF25E96E000E0901002194
:1094E000EA6EEF5010084FE14DA027D0020E6A6FD0
:1094F000000189EC1DF0012C10D04D90FFC8E9FF50
:10950000090100C9EAFFEFCF2EF9010E306F2EC915
:1095100031F9000118EC14F00ED0FFC8E9FF090181
:1095200000C9EAFFEFCF2EF9010E476F2EC948F9A7
:109530000001DCEC13F026D00901030E6A6F000174
:1095400089EC1DF0012C10D04D80FFC8E9FF090106
:1095500000C9EAFFEFCF2EF9010E306F2EC931F9A5
:10956000000118EC14F00ED0FFC8E9FF090100C992
:10957000EAFFEFCF2EF9010E476F2EC948F900011F
:10958000DCEC13F009010BD0FFC8E9FF00C9EAFFCA
:10959000EFCF2EF92EC947F90001C3EC13F00001FB
:1095A00077EF56F0050E0801FF25E96E000E090160
:1095B0000021EA6EEF3C43D0FFC8E9FF090100C972
:1095C000EAFFEFCF2EF9010E306F2EC931F90001FD
:1095D000FBEC13F0040E0801FF25E96E000E0901F3
:1095E0000021EA6EEFCF2EF92EC96AF900010EECC8
:1095F0002AF0012C15D0FFC8E9FF090100C9EAFFD4
:10960000EFCF2EF9010E306F2EC931F9000118ECA1
:1096100014F000C930F9FFC82FF961EC37F00ED013
:10962000FFC8E9FF090100C9EAFFEFCF2EF9010EDB
:10963000476F2EC948F90001DCEC13F00BD0FFC8CE
:10964000E9FF00C9EAFFEFCF2EF92EC947F9000163
:10965000C3EC13F077EF56F0050E0801FF25E96E15
:10966000000E09010021EA6EEF3C49D0FFC8E9FF76
:10967000090100C9EAFFEFCF2EF9010E306F2EC9A4
:1096800031F90001FBEC13F0040E0801FF25E96E2F
:10969000000E09010021EA6EEFCF2EF92EC930F934
:1096A000000113EF39F0012C1BD000C930F9FFC8BD
:1096B0002FF961EC37F0FFC8E9FF090100C9EAFFA3
:1096C000EFCF2EF9010E306F2EC931F9000118ECE1
:1096D00014F000C930F9FFC82FF961EC37F00ED053
:1096E000FFC8E9FF090100C9EAFFEFCF2EF9010E1B
:1096F000476F2EC948F90001DCEC13F00BD0FFC80E
:10970000E9FF00C9EAFFEFCF2EF92EC947F90001A2
:10971000C3EC13F077EF56F0080E0801FF25E96E51
:10972000000E09010021EA6EEF3C54D0FFC8E9FFAA
:10973000090100C9EAFFEFCF2EF9010E306F2EC9E3
:1097400031F90001FBEC13F0060E0801FF25E96E6C
:10975000000E09010021EA6EEF500F0B2D6F2D391D
:109760002E6FF00E2E17070E0801FF25E96E000E72
:1097700009010021EA6EEF500F0B2E112D6F2DC93C
:109780006AF90001AFEC31F0012C15D0FFC8E9FFF8
:10979000090100C9EAFFEFCF2EF9010E306F2EC983
:1097A00031F9000118EC14F000C930F9FFC82FF9A5
:1097B00061EC37F00ED0FFC8E9FF090100C9EAFFEC
:1097C000EFCF2EF9010E476F2EC948F90001DCECEE
:1097D00013F00BD0FFC8E9FF00C9EAFFEFCF2EF965
:1097E0002EC947F90001C3EC13F077EF56F0050ED0
:1097F0000801FF25E96E000E09010021EA6EEF3C29
:1098000043D0FFC8E9FF090100C9EAFFEFCF2EF9F5
:10981000010E306F2EC931F90001FBEC13F0040E7C
:109820000801FF25E96E000E09010021EA6EEFCF65
:109830002EF92EC930F900017EEF39F0012C15D038
:10984000FFC8E9FF090100C9EAFFEFCF2EF9010EB9
:10985000306F2EC931F9000118EC14F000C930F94D
:10986000FFC82FF961EC37F00ED0FFC8E9FF0901FE
:1098700000C9EAFFEFCF2EF9010E476F2EC948F954
:109880000001DCEC13F00BD0FFC8E9FF00C9EAFFD0
:10989000EFCF2EF92EC947F90001C3EC13F077EF93
:1098A00056F0080E0801FF25E96E000E090100219F
:1098B000EA6EEF3C96D0FFC8E9FF090100C9EAFF54
:1098C000EFCF2EF9010E306F2EC931F90001FBECFC
:1098D00013F0040E0801FF25E96E000E09010021B6
:1098E000EA6EEF50036A016F03C002F901352E6F73
:1098F00002352F6F2E372F372E372F372E372F3732
:10990000F00E2E17050E0801FF25E96E000E090165
:109910000021EA6EEF500F0B2E11016F2FC902F9D3
:1099200001352E6F02352F6F2E372F372E372F37F9
:109930002E372F37F00E2E17060E0801FF25E96E81
:10994000000E09010021EA6EEF500F0B2E11016F7E
:109950002FC902F901352E6F02352F6F2E372F37A1
:109960002E372F372E372F37F00E2E17070E080100
:10997000FF25E96E000E09010021EA6EEF500F0B82
:109980002E11016F2FC902F902C96BF901C96AF9D9
:10999000000188EC2AF0012C15D0FFC8E9FF09016D
:1099A00000C9EAFFEFCF2EF9010E306F2EC931F951
:1099B000000118EC14F000C930F9FFC82FF961EC70
:1099C00037F00ED0FFC8E9FF090100C9EAFFEFCF69
:1099D0002EF9010E476F2EC948F90001DCEC13F097
:1099E0000BD0FFC8E9FF00C9EAFFEFCF2EF92EC95F
:1099F00047F90001C3EC13F077EF56F0050E0801AC
:109A0000FF25E96E000E09010021EA6EEF3C43D00C
:109A1000FFC8E9FF090100C9EAFFEFCF2EF9010EE7
:109A2000306F2EC931F90001FBEC13F0040E080170
:109A3000FF25E96E000E09010021EA6EEFCF2EF935
:109A40002EC930F90001BCEF39F0012C15D0FFC848
:109A5000E9FF090100C9EAFFEFCF2EF9010E306FCF
:109A60002EC931F9000118EC14F000C930F9FFC813
:109A70002FF961EC37F00ED0FFC8E9FF090100C9EA
:109A8000EAFFEFCF2EF9010E476F2EC948F900010A
:109A9000DCEC13F00BD0FFC8E9FF00C9EAFFEFCF01
:109AA0002EF92EC947F90001C3EC13F077EF56F0F9
:109AB000080E0801FF25E96E000E09010021EA6E7B
:109AC000EF3C96D0FFC8E9FF090100C9EAFFEFCFDC
:109AD0002EF9010E306F2EC931F90001FBEC13F0A5
:109AE000040E0801FF25E96E000E09010021EA6E4F
:109AF000EF50036A016F03C002F901352E6F023582
:109B00002F6F2E372F372E372F372E372F37F00E58
:109B10002E17050E0801FF25E96E000E0901002130
:109B2000EA6EEF500F0B2E11016F2FC902F90135AC
:109B30002E6F02352F6F2E372F372E372F372E37B8
:109B40002F37F00E2E17060E0801FF25E96E000EC6
:109B500009010021EA6EEF500F0B2E11016F2FC982
:109B600002F901352E6F02352F6F2E372F372E3722
:109B70002F372E372F37F00E2E17070E0801FF252F
:109B8000E96E000E09010021EA6EEF500F0B2E1155
:109B9000016F2FC902F902C96BF901C96AF9000105
:109BA00022EC2BF0012C15D0FFC8E9FF090100C9F8
:109BB000EAFFEFCF2EF9010E306F2EC931F9000107
:109BC00018EC14F000C930F9FFC82FF961EC37F038
:109BD0000ED0FFC8E9FF090100C9EAFFEFCF2EF957
:109BE000010E476F2EC948F90001DCEC13F00BD0D1
:109BF000FFC8E9FF00C9EAFFEFCF2EF92EC947F9E8
:109C00000001C3EC13F077EF56F0050E0801FF25B5
:109C1000E96E000E09010021EA6EEF3C43D0FFC857
:109C2000E9FF090100C9EAFFEFCF2EF9010E306FFD
:109C30002EC931F90001FBEC13F0040E0801FF25D9
:109C4000E96E000E09010021EA6EEFCF2EF92EC950
:109C50006AF900019BEC2EF0012C15D0FFC8E9FF3A
:109C6000090100C9EAFFEFCF2EF9010E306F2EC9AE
:109C700031F9000118EC14F000C930F9FFC82FF9D0
:109C800061EC37F00ED0FFC8E9FF090100C9EAFF17
:109C9000EFCF2EF9010E476F2EC948F90001DCEC19
:109CA00013F00BD0FFC8E9FF00C9EAFFEFCF2EF990
:109CB0002EC947F90001C3EC13F077EF56F0050EFB
:109CC0000801FF25E96E000E09010021EA6EEF3C54
:109CD00043D0FFC8E9FF090100C9EAFFEFCF2EF921
:109CE000010E306F2EC931F90001FBEC13F0040EA8
:109CF0000801FF25E96E000E09010021EA6EEFCF91
:109D00002EF92EC930F90001FAEC39F0012C15D0EA
:109D1000FFC8E9FF090100C9EAFFEFCF2EF9010EE4
:109D2000306F2EC931F9000118EC14F000C930F978
:109D3000FFC82FF961EC37F00ED0FFC8E9FF090129
:109D400000C9EAFFEFCF2EF9010E476F2EC948F97F
:109D50000001DCEC13F00BD0FFC8E9FF00C9EAFFFB
:109D6000EFCF2EF92EC947F90001C3EC13F077EFBE
:109D700056F0080E0801FF25E96E000E09010021CA
:109D8000EA6EEF3C53D0FFC8E9FF090100C9EAFFC2
:109D9000EFCF2EF9010E306F2EC931F90001FBEC27
:109DA00013F0060E0801FF25E96E000E09010021DF
:109DB000EA6EEFCF2DF92D392E6FF00E2E17070E0C
:109DC0000801FF25E96E000E09010021EA6EEF503F
:109DD0000F0B2E112D6F2DC96AF90001E8EC2FF041
:109DE000012C15D0FFC8E9FF090100C9EAFFEFCF38
:109DF0002EF9010E306F2EC931F9000118EC14F064
:109E000000C930F9FFC82FF961EC37F00ED0FFC858
:109E1000E9FF090100C9EAFFEFCF2EF9010E476FF4
:109E20002EC948F90001DCEC13F00BD0FFC8E9FFA4
:109E300000C9EAFFEFCF2EF92EC947F90001C3ECA4
:109E400013F077EF56F0050E0801FF25E96E000EBE
:109E500009010021EA6EEF3C43D0FFC8E9FF090188
:109E600000C9EAFFEFCF2EF9010E306F2EC931F98C
:109E70000001FBEC13F0040E0801FF25E96E000E53
:109E800009010021EA6EEFCF2EF92EC930F9000149
:109E900034EF3AF0012C15D0FFC8E9FF090100C9E1
:109EA000EAFFEFCF2EF9010E306F2EC931F9000114
:109EB00018EC14F000C930F9FFC82FF961EC37F045
:109EC0000ED0FFC8E9FF090100C9EAFFEFCF2EF964
:109ED000010E476F2EC948F90001DCEC13F00BD0DE
:109EE000FFC8E9FF00C9EAFFEFCF2EF92EC947F9F5
:109EF0000001C3EC13F077EF56F0080E0801FF25C0
:109F0000E96E000E09010021EA6EEF3C54D0FFC853
:109F1000E9FF090100C9EAFFEFCF2EF9010E306F0A
:109F20002EC931F90001FBEC13F0060E0801FF25E4
:109F3000E96E000E09010021EA6EEF500F0B2D6F44
:109F40002D392E6FF00E2E17070E0801FF25E96E32
:109F5000000E09010021EA6EEF500F0B2E112D6F3C
:109F60002DC96AF90001F6EC2EF0012C15D0FFC8BE
:109F7000E9FF090100C9EAFFEFCF2EF9010E306FAA
:109F80002EC931F9000118EC14F000C930F9FFC8EE
:109F90002FF961EC37F00ED0FFC8E9FF090100C9C5
:109FA000EAFFEFCF2EF9010E476F2EC948F90001E5
:109FB000DCEC13F00BD0FFC8E9FF00C9EAFFEFCFDC
:109FC0002EF92EC947F90001C3EC13F077EF56F0D4
:109FD000050E0801FF25E96E000E09010021EA6E59
:109FE000EF3C43D0FFC8E9FF090100C9EAFFEFCF0A
:109FF0002EF9010E306F2EC931F90001FBEC13F080
:10A00000040E0801FF25E96E000E09010021EA6E29
:10A01000EFCF2EF92EC96AF90001F3EC30F0012CD4
:10A0200015D0FFC8E9FF090100C9EAFFEFCF2EF9FB
:10A03000010E306F2EC931F9000118EC14F000C97F
:10A0400030F9FFC82FF961EC37F00ED0FFC8E9FFF7
:10A05000090100C9EAFFEFCF2EF9010E476F2EC9A3
:10A0600048F90001DCEC13F00BD0FFC8E9FF00C990
:10A07000EAFFEFCF2EF92EC947F90001C3EC13F028
:10A0800077EF56F0050E0801FF25E96E000E090175
:10A090000021EA6EEF3C3DD0FFC8E9FF090100C98D
:10A0A000EAFFEFCF2EF9010E306F2EC931F9000112
:10A0B000FBEC13F0040E0801FF25E96E000E090108
:10A0C0000021EA6EEFCF2EF92EC930F9000174EFAE
:10A0D0003AF0012C0FD0FFC8E9FF090100C9EAFFDF
:10A0E000EFCF2EF9010E306F2EC931F9000118ECB7
:10A0F00014F00ED0FFC8E9FF090100C9EAFFEFCF55
:10A100002EF9010E476F2EC948F90001DCEC13F05F
:10A110000BD0FFC8E9FF00C9EAFFEFCF2EF92EC927
:10A1200047F90001C3EC13F077EF56F0050E080174
:10A13000FF25E96E000E09010021EA6EEF3C1FD0F9
:10A14000FFC8E9FF090100C9EAFFEFCF2EF9010EB0
:10A15000306F2EC931F90001FBEC13F0FFC8E9FFA5
:10A16000090100C9EAFFEFCF2EF9010E306F2EC9A9
:10A1700031F9000118EC14F00901E3EF5DF0FFC8BC
:10A18000E9FF00C9EAFFEFCF2EF92EC947F9000118
:10A19000C3EC13F077EF56F0080E0801FF25E96EC7
:10A1A000000E09010021EA6EEF3C98D0FFC8E9FFDC
:10A1B000090100C9EAFFEFCF2EF9010E306F2EC959
:10A1C00031F90001FBEC13F0040E0801FF25E96EE4
:10A1D000000E09010021EA6EEF50036A016F03C00F
:10A1E00002F901352E6F02352F6F2E372F372E379C
:10A1F0002F372E372F37F00E2E17050E0801FF25AB
:10A20000E96E000E09010021EA6EEF500F0B2E11CE
:10A21000016F2FC902F901352E6F02352F6F2E37CE
:10A220002F372E372F372E372F37F00E2E17060EDB
:10A230000801FF25E96E000E09010021EA6EEF50CA
:10A240000F0B2E11016F2FC902F901352E6F023548
:10A250002F6F2E372F372E372F372E372F37F00E01
:10A260002E17070E0801FF25E96E000E09010021D7
:10A27000EA6EEF500F0B2E11016F2FC902F902C9C0
:10A2800030F901C92FF90A0E316F0001A5EF3AF03C
:10A29000012C15D0FFC8E9FF090100C9EAFFEFCF83
:10A2A0002EF9010E306F2EC931F9000118EC14F0AF
:10A2B00000C930F9FFC82FF961EC37F00ED0FFC8A4
:10A2C000E9FF090100C9EAFFEFCF2EF9010E476F40
:10A2D0002EC948F90001DCEC13F00BD0FFC8E9FFF0
:10A2E00000C9EAFFEFCF2EF92EC947F90001C3ECF0
:10A2F00013F077EF56F0FFC8E9FF090100C9EAFF44
:10A30000EFCF2EF9010E306F2EC931F90001FBECB1
:10A3100013F0FFC8E9FF090100C9EAFFEFCF2EF9EA
:10A32000010E306F2EC931F9000118EC14F077EFEF
:10A3300056F0FFC8E9FF090100C9EAFFEFCF2EF987
:10A34000010E306F2EC931F90001FBEC13F0FFC88C
:10A35000E9FF090100C9EAFFEFCF2EF9010E306FC6
:10A360002EC931F9000118EC14F077EF56F0FFC850
:10A37000E9FF090100C9EAFFEFCF2EF9010E306FA6
:10A380002EC931F90001FBEC13F0FFC8E9FF090108
:10A3900000C9EAFFEFCF2EF9010E306F2EC931F957
:10A3A000000118EC14F077EF56F0FFC8E9FF09013F
:10A3B00000C9EAFFEFCF2EF9010E306F2EC931F937
:10A3C0000001FBEC13F0FFC8E9FF090100C9EAFF37
:10A3D000EFCF2EF9010E306F2EC931F9000118ECC4
:10A3E00014F077EF56F0FFC8E9FF090100C9EAFF52
:10A3F000EFCF2EF9010E306F2EC931F90001FBECC1
:10A4000013F0FFC8E9FF090100C9EAFFEFCF2EF9F9
:10A41000010E306F2EC931F9000118EC14F077EFFE
:10A4200056F0FFC8E9FF090100C9EAFFEFCF2EF996
:10A43000010E306F2EC931F90001FBEC13F0FFC89B
:10A44000E9FF090100C9EAFFEFCF2EF9010E306FD5
:10A450002EC931F9000118EC14F077EF56F0FFC85F
:10A46000E9FF090100C9EAFFEFCF2EF9010E306FB5
:10A470002EC931F90001FBEC13F0FFC8E9FF090117
:10A4800000C9EAFFEFCF2EF9010E306F2EC931F966
:10A49000000118EC14F077EF56F0FFC8E9FF09014E
:10A4A00000C9EAFFEFCF2EF9010E306F2EC931F946
:10A4B0000001FBEC13F0FFC8E9FF090100C9EAFF46
:10A4C000EFCF2EF9010E306F2EC931F9000118ECD3
:10A4D00014F077EF56F0FFC8E9FF090100C9EAFF61
:10A4E000EFCF2EF9010E306F2EC931F90001FBECD0
:10A4F00013F0FFC8E9FF090100C9EAFFEFCF2EF909
:10A50000010E306F2EC931F9000118EC14F077EF0D
:10A5100056F0FFC8E9FF090100C9EAFFEFCF2EF9A5
:10A52000010E306F2EC931F90001FBEC13F0FFC8AA
:10A53000E9FF090100C9EAFFEFCF2EF9010E306FE4
:10A540002EC931F9000118EC14F0D1D3FFC8E9FF8E
:10A55000090100C9EAFFEFCF2EF9010E306F2EC9B5
:10A5600031F90001FBEC13F0FFC8E9FF090100C954
:10A57000EAFFEFCF2EF9010E306F2EC931F900013D
:10A5800018EC14F0B4D3FFC8E9FF090100C9EAFFD1
:10A59000EFCF2EF9010E306F2EC931F90001FBEC1F
:10A5A00013F0FFC8E9FF090100C9EAFFEFCF2EF958
:10A5B000010E306F2EC931F9000118EC14F097D359
:10A5C000050E0801FF25E96E000E09010021EA6E63
:10A5D000EF3C3DD0FFC8E9FF090100C9EAFFEFCF1A
:10A5E0002EF9010E306F2EC931F90001FBEC13F08A
:10A5F000040E0801FF25E96E000E09010021EA6E34
:10A60000EFCF2EF92EC975F900014BEC2EF0012C7D
:10A610000FD0FFC8E9FF090100C9EAFFEFCF2EF90B
:10A62000010E306F2EC931F9000118EC14F00ED074
:10A63000FFC8E9FF090100C9EAFFEFCF2EF9010EBB
:10A64000476F2EC948F90001DCEC13F00BD0FFC8AE
:10A65000E9FF00C9EAFFEFCF2EF92EC947F9000143
:10A66000C3EC13F044D3080E0801FF25E96E000E79
:10A6700009010021EA6EEF3C4ED0FFC8E9FF090155
:10A6800000C9EAFFEFCF2EF9010E306F2EC931F964
:10A690000001FBEC13F0060E0801FF25E96E000E29
:10A6A00009010021EA6EEF500F0B2D6F2D392E6F2F
:10A6B000F00E2E17070E0801FF25E96E000E0901A6
:10A6C0000021EA6EEF500F0B2E112D6F2DC97AF974
:10A6D000000155EC2DF0012C0FD0FFC8E9FF090156
:10A6E00000C9EAFFEFCF2EF9010E306F2EC931F904
:10A6F000000118EC14F00ED0FFC8E9FF090100C9F1
:10A70000EAFFEFCF2EF9010E476F2EC948F900017D
:10A71000DCEC13F00BD0FFC8E9FF00C9EAFFEFCF74
:10A720002EF92EC947F90001C3EC13F0E0D2FFC89F
:10A73000E9FF090100C9EAFFEFCF2EF9010E306FE2
:10A740002EC931F90001FBEC13F0FFC8E9FF090144
:10A7500000C9EAFFEFCF2EF9010E306F2EC931F993
:10A76000000118EC14F0C3D2FFC8E9FF090100C9C9
:10A77000EAFFEFCF2EF9010E306F2EC931F900013B
:10A78000FBEC13F0FFC8E9FF090100C9EAFFEFCFB6
:10A790002EF9010E306F2EC931F9000118EC14F0BA
:10A7A000A6D2050E0801FF25E96E000E0901002161
:10A7B000EA6EEF3C6DD0FFC8E9FF090100C9EAFF6E
:10A7C000EFCF2EF9010E306F2EC931F90001FBECED
:10A7D00013F0040E0801FF25E96E000E09010021A7
:10A7E000EA6EEF5003080AE1040E0801FF25E96E46
:10A7F000000E09010021EA6EEF6A0AD0040E08017A
:10A80000FF25E96E000E09010021EA6E030EEF6ECE
:10A81000040E0801FF25E96E000E09010021EA6E11
:10A82000EFCF2EF92EC96AF900019BEC2EF0012C16
:10A8300020D0FFC8E9FF090100C9EAFFEFCF2EF9D8
:10A84000010E306F2EC931F9000118EC14F0030E1F
:10A850000801FF25E96E000E09010021EA6E390E9C
:10A86000EF6E00C930F9FFC82FF9000161EC37F035
:10A870000ED0FFC8E9FF090100C9EAFFEFCF2EF9AA
:10A88000010E476F2EC948F90001DCEC13F00BD024
:10A89000FFC8E9FF00C9EAFFEFCF2EF92EC947F93B
:10A8A0000001C3EC13F023D2050E0801FF25E96E69
:10A8B000000E09010021EA6EEF3C4ED0FFC8E9FF0F
:10A8C000090100C9EAFFEFCF2EF9010E306F2EC942
:10A8D00031F90001FBEC13F0040E0801FF25E96ECD
:10A8E000000E09010021EA6EEFCF2EF92EC930F9D2
:10A8F0000001FAEC39F0012C20D0FFC8E9FF090172
:10A9000000C9EAFFEFCF2EF9010E306F2EC931F9E1
:10A91000000118EC14F0030E0801FF25E96E000E8B
:10A9200009010021EA6E0B0EEF6E00C930F9FFC875
:10A930002FF9000161EC37F00ED0FFC8E9FF0901E3
:10A9400000C9EAFFEFCF2EF9010E476F2EC948F973
:10A950000001DCEC13F00BD0FFC8E9FF00C9EAFFEF
:10A96000EFCF2EF92EC947F90001C3EC13F0BFD188
:10A97000080E0801FF25E96E000E09010021EA6EAC
:10A98000EF3C5ED0FFC8E9FF090100C9EAFFEFCF45
:10A990002EF9010E306F2EC931F90001FBEC13F0D6
:10A9A000060E0801FF25E96E000E09010021EA6E7E
:10A9B000EFCF2DF92D392E6FF00E2E17070E08014F
:10A9C000FF25E96E000E09010021EA6EEF500F0B22
:10A9D0002E112D6F2DC96AF90001E8EC2FF0012C22
:10A9E00020D0FFC8E9FF090100C9EAFFEFCF2EF927
:10A9F000010E306F2EC931F9000118EC14F0030E6E
:10AA00000801FF25E96E000E09010021EA6E4B0ED8
:10AA1000EF6E00C930F9FFC82FF9000161EC37F083
:10AA20000ED0FFC8E9FF090100C9EAFFEFCF2EF9F8
:10AA3000010E476F2EC948F90001DCEC13F00BD072
:10AA4000FFC8E9FF00C9EAFFEFCF2EF92EC947F989
:10AA50000001C3EC13F04BD1FFC8E9FF090100C9A5
:10AA6000EAFFEFCF2EF9010E306F2EC931F9000148
:10AA7000FBEC13F0FFC8E9FF090100C9EAFFEFCFC3
:10AA80002EF9010E306F2EC931F9000118EC14F0C7
:10AA90002ED1FFC8E9FF090100C9EAFFEFCF2EF967
:10AAA000010E306F2EC931F90001FBEC13F0FFC825
:10AAB000E9FF090100C9EAFFEFCF2EF9010E306F5F
:10AAC0002EC931F9000118EC14F011D1FFC8E9FFCB
:10AAD000090100C9EAFFEFCF2EF9010E306F2EC930
:10AAE00031F90001FBEC13F0FFC8E9FF090100C9CF
:10AAF000EAFFEFCF2EF9010E306F2EC931F90001B8
:10AB000018EC14F0F4D0FFC8E9FF090100C9EAFF0E
:10AB1000EFCF2EF9010E306F2EC931F90001FBEC99
:10AB200013F0FFC8E9FF090100C9EAFFEFCF2EF9D2
:10AB3000010E306F2EC931F9000118EC14F0D7D096
:10AB4000FFC8E9FF090100C9EAFFEFCF2EF9010EA6
:10AB5000306F2EC931F90001FBEC13F0FFC8E9FF9B
:10AB6000090100C9EAFFEFCF2EF9010E306F2EC99F
:10AB700031F9000118EC14F0BAD0FFC8E9FF09015F
:10AB800000C9EAFFEFCF2EF9010E306F2EC931F95F
:10AB90000001FBEC13F0FFC8E9FF090100C9EAFF5F
:10ABA000EFCF2EF9010E306F2EC931F9000118ECEC
:10ABB00014F09DD0FFC8E9FF090100C9EAFFEFCFFB
:10ABC0002EF9010E306F2EC931F90001FBEC13F0A4
:10ABD000FFC8E9FF090100C9EAFFEFCF2EF9010E16
:10ABE000306F2EC931F9000118EC14F080D0FFC885
:10ABF000E9FF090100C9EAFFEFCF2EF9010E306F1E
:10AC00002EC931F90001FBEC13F0FFC8E9FF09017F
:10AC100000C9EAFFEFCF2EF9010E306F2EC931F9CE
:10AC2000000118EC14F063D0FFC8E9FF090100C966
:10AC3000EAFFEFCF2EF9010E306F2EC931F9000176
:10AC4000FBEC13F0FFC8E9FF090100C9EAFFEFCFF1
:10AC50002EF9010E306F2EC931F9000118EC14F0F5
:10AC600046D0FFC8E9FF090100C9EAFFEFCF2EF97E
:10AC7000010E306F2EC931F90001FBEC13F0FFC853
:10AC8000E9FF090100C9EAFFEFCF2EF9010E306F8D
:10AC90002EC931F9000118EC14F029D0FFC8E9FFE2
:10ACA000090100C9EAFFEFCF2EF9010E306F2EC95E
:10ACB00031F90001FBEC13F0FFC8E9FF090100C9FD
:10ACC000EAFFEFCF2EF9010E306F2EC931F90001E6
:10ACD00018EC14F00CD0FFC8E9FF00C9EAFFEFCF71
:10ACE0002EF92EC947F90001C3EC13F000D0E2EFB2
:10ACF0005DF0020E0801FF25E96E000E090100213A
:10AD0000EA6EEF500808D8A4E5D0030E0801FF252D
:10AD1000E96E000E09010021EA6EEF50020A0001FF
:10AD200005E0060A0FE0140A19E0D2D0FFC8E9FFD7
:10AD300000C9EAFFEFCF2EF92EC947F90001C3EC95
:10AD400013F0C6D0FFC8E9FF00C9EAFFEFCF2EF924
:10AD50002EC947F90001C3EC13F0BAD0070E080161
:10AD6000FF25E96E000E09010021EA6EEF3CA4D038
:10AD7000040E0801FF25E96E000E09010021EA6EAC
:10AD8000EFCF2EF9000E2EBF010E000AD8A494D0EA
:10AD9000050E0801FF25E96E000E09010021EA6E8B
:10ADA000EF50F00BD8A488D0060E0801FF25E96EFD
:10ADB000000E09010021EA6EEF50F00BD8A47CD000
:10ADC000FFC8E9FF090100C9EAFFEFCF2EF9010E24
:10ADD000306F2EC931F90001FBEC13F0040E0801AD
:10ADE000FF25E96E000E09010021EA6EEFCF3FF862
:10ADF0000801050EFF25E96E000E09010021EA6E2B
:10AE0000EFCF40F80801060EFF25E96E000E09019C
:10AE10000021EA6EEFCF41F80801AA6A070EA96E79
:10AE20003FC8A8FFA69CA69EA684F250006EF29E84
:10AE30000F01550EA76EAA0EA76EA682A6B2FED768
:10AE4000A6940050F212AA6A080EA96E40C8A8FF84
:10AE5000A69CA69EA684F2CF00F0F29E550EA76E89
:10AE6000AA0EA76EA682A6B2FED7A6940050F21232
:10AE7000AA6A090EA96E41C8A8FFA69CA69EA68430
:10AE8000F2CF00F0F29E550EA76EAA0EA76EA68214
:10AE9000A6B2FED7A6940050F212FFC8E9FF09013E
:10AEA00000C9EAFFEFCF2EF9010E306F2EC931F93C
:10AEB000000118EC14F00BD0FFC8E9FF00C9EAFF4D
:10AEC000EFCF2EF92EC947F90001C3EC13F000D0E3
:10AED000E2EF5DF0020E0801FF25E96E000E0901A8
:10AEE0000021EA6EEF507E08D8A4FCEF5CF0030E60
:10AEF0000801FF25E96E000E09010021EA6EEF2C22
:10AF0000C2D0040E0801FF25E96E000E09010021E0
:10AF1000EA6EEF504A08D8A4B6D00A0E0801FF2501
:10AF2000E96E000E09010021EA6EEF3C9DD0FFC8DA
:10AF3000E9FF090100C9EAFFEFCF2EF9010E306FDA
:10AF40002EC931F90001FBEC13F0060E0801FF25B4
:10AF5000E96E000E09010021EA6EEF50036A016FED
:10AF600003C002F901352E6F02352F6F2E372F37B0
:10AF70002E372F372E372F37F00E2E17070E0801DA
:10AF8000FF25E96E000E09010021EA6EEF500F0B5C
:10AF90002E11016F2FC902F901352E6F02352F6F67
:10AFA0002E372F372E372F372E372F37F00E2E17FD
:10AFB000080E0801FF25E96E000E09010021EA6E66
:10AFC000EF500F0B2E11016F2FC902F901352E6FB3
:10AFD00002352F6F2E372F372E372F372E372F373B
:10AFE000F00E2E17090E0801FF25E96E000E09016B
:10AFF0000021EA6EEF500F0B2E11016F2FC902F9DD
:10B00000050E0801FF25E96E000E09010021EA6E18
:10B01000EFCF2EF902C931F901C930F92EC932F941
:10B02000000109EC1BF0012C0FD0FFC8E9FF09015A
:10B0300000C9EAFFEFCF2EF9010E306F2EC931F9AA
:10B04000000118EC14F00ED0FFC8E9FF090100C997
:10B05000EAFFEFCF2EF9010E476F2EC948F9000124
:10B06000DCEC13F00CD00901FFC8E9FF00C9EAFFCE
:10B07000EFCF2EF92EC947F90001C3EC13F00901F7
:10B08000E3EF5DF0EAD0030E0801FF25E96E000E44
:10B0900009010021EA6EEF2CE0D0040E0801FF2523
:10B0A000E96E000E09010021EA6EEF500B08D8A4EA
:10B0B000D4D085A611D0FFC8E9FF090100C9EAFF75
:10B0C000EFCF2EF9010E476F2EC948F90001DCECD5
:10B0D00013F00901E3EF5DF0080E0801FF25E96EAA
:10B0E000000E09010021EA6EEF3CA9D0FFC8E9FF7C
:10B0F000090100C9EAFFEFCF2EF9010E306F2EC90A
:10B1000031F90001FBEC13F0070E0801FF25E96E91
:10B11000000E09010021EA6EEF50070822E3070E36
:10B120000801FF25E96E000E09010021EA6EEFCF4C
:10B1300060F00001AA6A060EA96E60C0A8FFA69C76
:10B14000A69EA684F250006EF29E0F01550EA76EC9
:10B15000AA0EA76EA682A6B2FED7A6940050F2123F
:10B1600009010C0E036F050E0801FF25E96E000EA4
:10B1700009010021EA6EEFCF04F9060E0801FF2550
:10B18000E96E000E09010021EA6EEFCF05F9066BAA
:10B19000090EE36F030EE26FE46F0001F4EC0FF0B1
:10B1A000270E0901636F100E626F000146EC14F068
:10B1B000012C35D0090EEA6E170EE96E006A026A9C
:10B1C000140E016E3BEC07F0120E09012C6F090EF4
:10B1D000E36F170EE26F090EE56F2C0EE46F0001AE
:10B1E00029EC10F0012C0FD0FFC8E9FF090100C9BC
:10B1F000EAFFEFCF2EF9010E306F2EC931F90001B1
:10B2000018EC14F00BD0FFC8E9FF00C9EAFFEFCF3C
:10B210002EF92EC947F90001C3EC13F00ED0FFC878
:10B22000E9FF090100C9EAFFEFCF2EF9010E476FD0
:10B230002EC948F90001DCEC13F00CD00901FFC85D
:10B24000E9FF00C9EAFFEFCF2EF92EC947F9000147
:10B25000C3EC13F00901E3EF5DF0030E0801FF25D5
:10B26000E96E000E09010021EA6EEF50010A0001AB
:10B270000DE0520AD8B40CD2070AD8B473D2010A2E
:10B28000D8B4DAD2030AD8B441D3AAD3070E08013E
:10B29000FF25E96E000E09010021EA6EEF3CECD1BA
:10B2A000040E0801FF25E96E000E09010021EA6E77
:10B2B000EF50060A000109E00F0A5EE0030AD8B465
:10B2C000B2D07A0AD8B409D1C9D1050E0801FF2538
:10B2D000E96E000E09010021EA6EEF520CE1060E44
:10B2E0000801FF25E96E000E09010021EA6EEF2C2E
:10B2F00002D04E8024D0050E0801FF25E96E000E15
:10B3000009010021EA6EEF520CE1060E0801FF254B
:10B31000E96E000E09010021EA6EEF5202E14E9043
:10B320000ED0FFC8E9FF00C9EAFFEFCF2EF92EC902
:10B3300047F90001C3EC13F00901E3EF5DF0FFC82A
:10B34000E9FF090100C9EAFFEFCF2EF9010E306FC6
:10B350002EC931F90001FBEC13F0FFC8E9FF090128
:10B3600000C9EAFFEFCF2EF9010E306F2EC931F977
:10B37000000118EC14F07ED1050E0801FF25E96EDE
:10B38000000E09010021EA6EEF520CE1060E0801E1
:10B39000FF25E96E000E09010021EA6EEF2C02D0B4
:10B3A0004E8224D0050E0801FF25E96E000E09012A
:10B3B0000021EA6EEF520CE1060E0801FF25E96E4E
:10B3C000000E09010021EA6EEF5202E14E920ED00A
:10B3D000FFC8E9FF00C9EAFFEFCF2EF92EC947F9F0
:10B3E0000001C3EC13F00901E3EF5DF0FFC8E9FFD2
:10B3F000090100C9EAFFEFCF2EF9010E306F2EC907
:10B4000031F90001FBEC13F0FFC8E9FF090100C9A5
:10B41000EAFFEFCF2EF9010E306F2EC931F900018E
:10B4200018EC14F027D1050E0801FF25E96E000E77
:10B4300009010021EA6EEF520EE1060E0801FF2518
:10B44000E96E000E09010021EA6EEF50020803E1E7
:10B450008C9A959A25D0050E0801FF25E96E000EFD
:10B4600009010021EA6EEF520EE1060E0801FF25E8
:10B47000E96E000E09010021EA6EEF50030803E1B6
:10B480008C8A959A0DD0FFC8E9FF00C9EAFFEFCF7B
:10B490002EF92EC947F90001C3EC13F0090193D32B
:10B4A000FFC8E9FF090100C9EAFFEFCF2EF9010E3D
:10B4B000306F2EC931F90001FBEC13F0FFC8E9FF32
:10B4C000090100C9EAFFEFCF2EF9010E306F2EC936
:10B4D00031F9000118EC14F0CDD085A610D0FFC8CA
:10B4E000E9FF090100C9EAFFEFCF2EF9010E476F0E
:10B4F0002EC948F90001DCEC13F0090164D3050EF4
:10B500000801FF25E96E000E09010021EA6EEF52E5
:10B510000CE1060E0801FF25E96E000E090100216D
:10B52000EA6EEF5202E1056B24D0050E0801FF25FB
:10B53000E96E000E09010021EA6EEF520DE1060EE0
:10B540000801FF25E96E000E09010021EA6EEF2CCB
:10B5500003D0010E056F0DD0FFC8E9FF00C9EAFF57
:10B56000EFCF2EF92EC947F90001C3EC13F0090102
:10B570002AD3FFC8E9FF090100C9EAFFEFCF2EF97E
:10B58000010E306F2EC931F90001FBEC13F0130EE0
:10B590000901036F050E0801FF25E96E000E090180
:10B5A0000021EA6EEFCF04F9066B090EE36F030E7C
:10B5B000E26FE46F0001F4EC0FF0270E0901636FF6
:10B5C000100E626F000146EC14F0012C38D0090E09
:10B5D000EA6E170EE96E006A026A140E016E3BEC09
:10B5E00007F0120E09012C6F090EE36F170EE26FC0
:10B5F000090EE56F2C0EE46F000129EC10F0012C10
:10B600000FD0FFC8E9FF090100C9EAFFEFCF2EF90B
:10B61000010E306F2EC931F9000118EC14F00ED074
:10B62000FFC8E9FF090100C9EAFFEFCF2EF9010EBB
:10B63000476F2EC948F90001DCEC13F00ED0FFC8AB
:10B64000E9FF090100C9EAFFEFCF2EF9010E476FAC
:10B650002EC948F90001DCEC13F00CD0FFC8E9FF5B
:10B6600000C9EAFFEFCF2EF92EC947F90001C3EC5C
:10B6700013F000D00CD00901FFC8E9FF00C9EAFFB0
:10B68000EFCF2EF92EC947F90001C3EC13F0B3D167
:10B69000080E0801FF25E96E000E09010021EA6E7F
:10B6A000EF3C54D0FFC8E9FF090100C9EAFFEFCF22
:10B6B0002EF9010E306F2EC931F90001FBEC13F0A9
:10B6C000060E0801FF25E96E000E09010021EA6E51
:10B6D000EFCF2DF92D392E6FF00E2E17070E080122
:10B6E000FF25E96E000E09010021EA6EEF500F0BF5
:10B6F0002E112D6F2DC92FF900019DEC3BF0012C6F
:10B7000015D0FFC8E9FF090100C9EAFFEFCF2EF904
:10B71000010E306F2EC931F9000118EC14F000C988
:10B7200030F9FFC82FF961EC37F00ED0FFC8E9FF00
:10B73000090100C9EAFFEFCF2EF9010E476F2EC9AC
:10B7400048F90001DCEC13F009013DD2FFC8E9FF24
:10B7500000C9EAFFEFCF2EF92EC947F90001C3EC6B
:10B7600013F049D1080E0801FF25E96E000E09010A
:10B770000021EA6EEF3C54D0FFC8E9FF090100C97F
:10B78000EAFFEFCF2EF9010E306F2EC931F900011B
:10B79000FBEC13F0060E0801FF25E96E000E09010F
:10B7A0000021EA6EEFCF2DF92D392E6FF00E2E17F6
:10B7B000070E0801FF25E96E000E09010021EA6E5F
:10B7C000EF500F0B2E112D6F2DC92FF900019BEC9F
:10B7D0003CF0012C15D0FFC8E9FF090100C9EAFFC0
:10B7E000EFCF2EF9010E306F2EC931F9000118ECA0
:10B7F00014F000C930F9FFC82FF961EC37F00ED012
:10B80000FFC8E9FF090100C9EAFFEFCF2EF9010ED9
:10B81000476F2EC948F90001DCEC13F00901D3D1C0
:10B82000FFC8E9FF00C9EAFFEFCF2EF92EC947F99B
:10B830000001C3EC13F0DFD0080E0801FF25E96E0C
:10B84000000E09010021EA6EEF3C54D0FFC8E9FF69
:10B85000090100C9EAFFEFCF2EF9010E306F2EC9A2
:10B8600031F90001FBEC13F0060E0801FF25E96E2B
:10B87000000E09010021EA6EEFCF2DF92D392E6F50
:10B88000F00E2E17070E0801FF25E96E000E0901C4
:10B890000021EA6EEF500F0B2E112D6F2DC92FF9DD
:10B8A000000175EC3DF0012C15D0FFC8E9FF09013E
:10B8B00000C9EAFFEFCF2EF9010E306F2EC931F922
:10B8C000000118EC14F000C930F9FFC82FF961EC41
:10B8D00037F00ED0FFC8E9FF090100C9EAFFEFCF3A
:10B8E0002EF9010E476F2EC948F90001DCEC13F068
:10B8F000090169D1FFC8E9FF00C9EAFFEFCF2EF9BE
:10B900002EC947F90001C3EC13F075D0080E0801E9
:10B91000FF25E96E000E09010021EA6EEF3C54D0CC
:10B92000FFC8E9FF090100C9EAFFEFCF2EF9010EB8
:10B93000306F2EC931F90001FBEC13F0060E08013F
:10B94000FF25E96E000E09010021EA6EEFCF2DF907
:10B950002D392E6FF00E2E17070E0801FF25E96E08
:10B96000000E09010021EA6EEF500F0B2E112D6F12
:10B970002DC96AF9000190EC33F0012C15D0FFC8F5
:10B98000E9FF090100C9EAFFEFCF2EF9010E306F80
:10B990002EC931F9000118EC14F000C930F9FFC8C4
:10B9A0002FF961EC37F00ED0FFC8E9FF090100C99B
:10B9B000EAFFEFCF2EF9010E476F2EC948F90001BB
:10B9C000DCEC13F00901FFD0FFC8E9FF00C9EAFF72
:10B9D000EFCF2EF92EC947F90001C3EC13F00BD0BD
:10B9E000FFC8E9FF00C9EAFFEFCF2EF92EC947F9DA
:10B9F0000001C3EC13F0E6D0020E0801FF25E96E4A
:10BA0000000E09010021EA6EEF525DE1030E08010C
:10BA1000FF25E96E000E09010021EA6EEF2C47D0E8
:10BA2000040E0801FF25E96E000E09010021EA6EEF
:10BA3000EF3C3DD0FFC8E9FF00C9EAFF08013951DA
:10BA4000EF5CD8B402D0090132D0FFC8E9FF00C9C9
:10BA5000EAFF08013939006EF00E00160050800927
:10BA6000EF6E010EFF25E96E000E09010021EA6E5E
:10BA7000500EEF6E020E0801FF25E96E000E09015F
:10BA80000021EA6EEF68030E0801FF25E96E000E43
:10BA900009010021EA6EEF6A00C9E3F9FFC8E2F983
:10BAA000E46BE569000128EC0FF00CD00901FFC838
:10BAB000E9FF00C9EAFFEFCF2EF92EC947F90001CF
:10BAC000C3EC13F07FD0020E0801FF25E96E000ED3
:10BAD00009010021EA6EEF50F00B200868E1030E27
:10BAE0000801FF25E96E000E09010021EA6EEF3C16
:10BAF0005ED0020E0801FF25E96E000E090100214B
:10BB0000EA6EEF5021080BE0020E0801FF25E96EF6
:10BB1000000E09010021EA6EEF50220824E108011D
:10BB20003939006EF00E0016005080090901176FB8
:10BB3000020E0801FF25E96E000E09010021EA6EE0
:10BB4000EF500F0B6009186F040E196F1A691B6B09
:10BB5000090EE36F170EE26FE46BE569000128EC54
:10BB60000FF023D0090108013939006EF00E0016DC
:10BB7000005080090901176F020E0801FF25E96EC8
:10BB8000000E09010021EA6EEF500F0B6009186FDB
:10BB9000050E196F1A691B6B090EE36F170EE26F22
:10BBA000E46BE569000128EC0FF00CD00901FFC837
:10BBB000E9FF00C9EAFFEFCF2EF92EC947F90001CE
:10BBC000C3EC13F00901000151EF6AF00901496B60
:10BBD000486B3A0E4A6F520E4B6F460E4C6F4D6FCC
:10BBE000450E4E6F370E4F6F300E506F516F526BC8
:10BBF000090EF16F4A0EF06F090EF36F480EF26FE7
:10BC00000001DCEC0CF0012C2AD009014851006E37
:10BC10004951036E035004E10052000109E009019B
:10BC2000035005E1010E005C00010DE0090116D092
:10BC3000090146C9E9FF47C9EAFF020EEF6E010E8E
:10BC4000016E10D00BD0090146C9E9FF47C9EAFFD0
:10BC5000030EEF6E010E016E05D000D00001FF0E45
:10BC6000016E0901000199EF60F00901496B486B11
:10BC70003A0E4A6F720E4B6F460E4C6F380E4D6F78
:10BC8000350E4E6F320E4F6F300E506F516F526F38
:10BC9000536F546B46C9E9FF47C9EAFFEC6AED529E
:10BCA000EF6A090EF16F4A0EF06F090EF36F480E3E
:10BCB000F26F0001DCEC0CF0012C01D003D0FF0E80
:10BCC000016E0CD0090146C9E9FF47C9EAFF49C91D
:10BCD000ECFFED5248C9EFFF010E016E000146EF87
:10BCE00061F00901496B486B3A0E4A6F520E4B6F77
:10BCF000460E4C6F4D6F330E4E6F4F6F300E506FC0
:10BD0000516F526B090EF16F4A0EF06F090EF36F0F
:10BD1000480EF26F0001DCEC0CF0012C16D009018A
:10BD200048A108D04F8646C9E9FF47C9EAFF020E7D
:10BD3000EF6E07D04F9646C9E9FF47C9EAFF030EE9
:10BD4000EF6E010E016E04D00001FF0E016E0901BD
:10BD50000001D0EF63F0900E0901486F500E496F5B
:10BD6000020E4A6F4B6B4C6B4D6B4E6B4F69506BB9
:10BD7000516B526B4739006EF00E0016005080096F
:10BD8000486F090EE36F480EE26FE46BE56900014E
:10BD900028EC0FF0D9EF66F03A0E0901486F520E09
:10BDA000496F460E4A6F420E4B6F430E4C6F390E71
:10BDB0004D6F300E4E6F4F6F506B536B526B46C9C9
:10BDC000E9FF47C9EAFFEF6A090EF16F480EF06F0D
:10BDD000090EF36F520EF26F0001DCEC0CF0012C37
:10BDE0000BD0090146C9E9FF47C9EAFF52C9EFFF75
:10BDF000010E016E04D00001FF0E016E0901000169
:10BE00004CEF68F03A0E0901486F520E496F460E2A
:10BE10004A6F420E4B6F440E4C6F4D6F300E4E6F9B
:10BE20004F6F506B536B526B46C9E9FF47C9EAFF2E
:10BE3000EF6A090EF16F480EF06F090EF36F520EA4
:10BE4000F26F0001DCEC0CF0012C0BD0090146C9AB
:10BE5000E9FF47C9EAFF52C9EFFF010E016E04D0A6
:10BE60000001FF0E016E0901000195EF68F03A0E26
:10BE70000901486F520E496F460E4A6F420E4B6FD2
:10BE8000450E4C6F330E4D6F300E4E6F4F6F506B33
:10BE9000536B526B46C9E9FF47C9EAFFEF6A090EC7
:10BEA000F16F480EF06F090EF36F520EF26F000142
:10BEB000DCEC0CF0012C0BD0090146C9E9FF47C9A5
:10BEC000EAFF52C9EFFF010E016E04D00001FF0E20
:10BED000016E09010001DEEF68F00901026B016BE0
:10BEE000036B900E2C6F500E2D6F2E6B2F6B306BE3
:10BEF000316B3269336B900E346F500E356F366B89
:10BF00003769900E386F500E396F3A6B3B6B3C6B54
:10BF10003D6B3E6B3F6B406B416B4269436B446BC7
:10BF2000FFC8E9FF090100C9EAFFEF38006EF00E13
:10BF30000016005080092C6F2CC938F92CC934F92F
:10BF40002CC938F9020E0801FF25E96E000E09011F
:10BF50000021EA6EEF5229E1030E0801FF25E96E88
:10BF6000000E09010021EA6EEF50020A000101E013
:10BF70000CD0FFC8E9FF00C9EAFFEFCF45F945C97A
:10BF800047F9000153EC12F00CD0FFC8E9FF00C9DB
:10BF9000EAFFEFCF45F945C947F90001C3EC13F0BB
:10BFA00000D076EF69F076EF69F0020E0801FF2508
:10BFB000E96E000E09010021EA6EEF500408D8A4D2
:10BFC00047EF64F0040E0801FF25E96E000E090139
:10BFD0000021EA6EEF3C3AEF64F0030E0801FF2502
:10BFE000E96E000E09010021EA6EEF50000A00011F
:10BFF000D8B483D0010AD8B494D03E0AD8B4B8D00B
:10C00000780AD8B4C3D00D0AD8B404D1020AD8B47F
:10C0100034D1080AD8B474D1010AD8B471D1070A4E
:10C02000D8B46ED16E0AD8B46BD10F0AD8B468D127
:10C030006A0AD8B465D1640AD8B462D1440AD8B4C3
:10C040006FD16B0AD8B480D15F0AD8B47DD13F0AD2
:10C05000D8B47AD10D0AD8B477D17C0AD8B474D1C7
:10C06000620AD8B471D1010AD8B46ED1600AD8B4CA
:10C070006BD1450AD8B468D1670AD8B472D1610AC5
:10C08000D8B46FD1390AD8B46CD1020AD8B469D106
:10C09000540AD8B472D1600AD8B497D1020AD8B47D
:10C0A00094D16F0AD8B49ED1760AD8B4C3D1070A06
:10C0B000D8B404D27D0AD8B445D2070AD8B442D243
:10C0C0000D0AD8B48DD2710AD8B4B2D2090AD8B444
:10C0D000E3D2050AD8B4E0D2020AD8B411D32D0AAB
:10C0E000D8B442D3030AD8B452D3010AD8B478D30F
:10C0F000410AD8B482D32DEF64F04DBE04D0030EB4
:10C100000901366F03D0020E0901366F3769090E37
:10C11000E36F340EE26FE46BE569000128EC0FF089
:10C12000A8D30901036B090E476F030E466F000188
:10C130004DD5012C0ED003C936F9090E0901E36F64
:10C14000340EE26FE46BE569000128EC0FF091D347
:10C150000ED0FFC8E9FF090100C9EAFFEFCF45F99A
:10C16000010E476F45C948F90001DCEC13F081D39B
:10C1700059C02EF909012F69090EE36F2C0EE26FE9
:10C18000E46BE569000128EC0FF073D30901026B41
:10C19000016B090E476F010E466F00018EEC15F022
:10C1A000012C29D009010239456F0F0E4517455161
:10C1B0000F0B2E6F02510F0B2F6F0231466F0131A3
:10C1C000456F4633453346334533463345330F0ECB
:10C1D000461745510F0B306F01510F0B316F32690C
:10C1E000090EE36F2C0EE26FE46BE569000128ECA9
:10C1F0000FF03FD30ED0FFC8E9FF090100C9EAFFE5
:10C20000EFCF45F9010E476F45C948F90001DCEC55
:10C2100013F02FD30901036B090E796F030E786FAA
:10C220000001BCEC2BF0012C19D009012E6B2F6BF7
:10C230000339006EF00E001600500F0B306F0351E3
:10C240000F0B316F3269090EE36F2C0EE26FE46B56
:10C25000E569000128EC0FF00CD30ED0FFC8E9FF10
:10C26000090100C9EAFFEFCF45F9010E476F45C943
:10C2700048F90001DCEC13F0FCD20901026B016B00
:10C28000090E476F010E466F0001EFD4012C29D033
:10C2900009010239456F0F0E451745510F0B2E6FDF
:10C2A00002510F0B2F6F0231466F0131456F46333C
:10C2B000453346334533463345330F0E4617455114
:10C2C0000F0B306F01510F0B316F3269090EE36FA5
:10C2D0002C0EE26FE46BE569000128EC0FF0C9D287
:10C2E0000ED0FFC8E9FF090100C9EAFFEFCF45F909
:10C2F000010E476F45C948F90001DCEC13F0B9D2D3
:10C3000009012E6B2F6B306B316B3269090EE36FB5
:10C310002C0EE26FE46BE569000128EC0FF0A9D266
:10C3200009013A6B3B6B3C6B3D6B3E6B3F6B406B6B
:10C33000416B4269090EE36F380EE26FE46BE56909
:10C34000000128EC0FF095D2030E0901366F090E9B
:10C35000E36F340EE26FE46BE569000128EC0FF047
:10C3600088D20901366B090EE36F340EE26FE46B7D
:10C37000E569000128EC0FF07CD20901036B090E7E
:10C380006B6F030E6A6F00018EEC20F0012C0ED053
:10C3900003C936F9090E0901E36F340EE26FE46B4D
:10C3A000E569000128EC0FF064D20ED0FFC8E9FF68
:10C3B000090100C9EAFFEFCF45F9010E476F45C9F2
:10C3C00048F90001DCEC13F054D2020E0901366F7B
:10C3D000090EE36F340EE26FE46BE569000128ECAF
:10C3E0000FF047D20901036B090E6B6F030E6A6FE2
:10C3F000000150EC20F0012C0ED003C936F9090ED3
:10C400000901E36F340EE26FE46BE569000128EC8B
:10C410000FF02FD20ED0FFC8E9FF090100C9EAFFD3
:10C42000EFCF45F9010E476F45C948F90001DCEC33
:10C4300013F01FD20901026B016B090E786F010E18
:10C44000776F00017AEC25F0012C29D0090102391F
:10C45000456F0F0E451745510F0B2E6F02510F0BF5
:10C460002F6F0231466F0131456F463345334633F6
:10C470004533463345330F0E461745510F0B306F8A
:10C4800001510F0B316F3269090EE36F2C0EE26F11
:10C49000E46BE569000128EC0FF0EBD10ED0FFC88A
:10C4A000E9FF090100C9EAFFEFCF45F9010E476F27
:10C4B00045C948F90001DCEC13F0DBD10901026B3E
:10C4C000016B090E786F010E776F000166EC26F0A4
:10C4D000012C29D009010239456F0F0E451745512E
:10C4E0000F0B2E6F02510F0B2F6F0231466F013170
:10C4F000456F4633453346334533463345330F0E98
:10C50000461745510F0B306F01510F0B316F3269D8
:10C51000090EE36F2C0EE26FE46BE569000128EC75
:10C520000FF0A7D10ED0FFC8E9FF090100C9EAFF4B
:10C53000EFCF45F9010E476F45C948F90001DCEC22
:10C5400013F097D10901036B090E6B6F030E6A6F2D
:10C550000001E1EC1FF0012C34D0030E0801FF258F
:10C56000E96E000E09010021EA6EEF50390803E17F
:10C5700003C936F91BD0035303E1030E366F16D0FF
:10C580000351030803E1020E366F10D0FFC8E9FF24
:10C59000090100C9EAFFEFCF45F9010E476F45C910
:10C5A00048F90001DCEC13F064D10901090EE36FD6
:10C5B000340EE26FE46BE569000128EC0FF059D10D
:10C5C0000ED0FFC8E9FF090100C9EAFFEFCF45F926
:10C5D000010E476F45C948F90001DCEC13F049D161
:10C5E0000901036B090E6B6F030E6A6F0001CDEC3E
:10C5F00020F0012C0ED003C936F909013769090E64
:10C60000E36F340EE26FE46BE569000128EC0FF094
:10C610000ED0FFC8E9FF090100C9EAFFEFCF45F9D5
:10C62000010E476F45C948F90001DCEC13F021D138
:10C630000901036B090E6B6F030E6A6F000147EC73
:10C6400027F0012C1AD009012E6B2F6B0339006ED5
:10C650000F0E001600500F0B306F03510F0B316F90
:10C660003269090EE36F2C0EE26F070EE46FE56B83
:10C67000000128EC0FF0FDD00ED0FFC8E9FF090142
:10C6800000C9EAFFEFCF45F9010E476F45C948F9E8
:10C690000001DCEC13F0EDD00901036B090E6B6FA8
:10C6A000030E6A6F000110EC21F0012C1AD0090171
:10C6B0002E6B2F6B0339006E0F0E001600500F0B00
:10C6C000306F03510F0B316F3269090EE36F2C0E7F
:10C6D000E26F070EE46FE56B000128EC0FF0C9D0A4
:10C6E0000ED0FFC8E9FF090100C9EAFFEFCF45F905
:10C6F000010E476F45C948F90001DCEC13F0B9D0D1
:10C700000901036B090E6B6F030E6A6F00015CEC8D
:10C7100023F0012C1AD009012E6B2F6B0339006E08
:10C720000F0E001600500F0B306F03510F0B316FBF
:10C730003269090EE36F2C0EE26F070EE46FE56BB2
:10C74000000128EC0FF095D00ED0FFC8E9FF0901D9
:10C7500000C9EAFFEFCF45F9010E476F45C948F917
:10C760000001DCEC13F085D04FA004D0020E0901CB
:10C770002E6F03D0030E09012E6F090EE36F2C0EEE
:10C78000E26FE46BE569000128EC0FF072D009015B
:10C79000036B090E476F030E466F000171EF5EF0E9
:10C7A000012C0FD003C936F909013769090EE36F6F
:10C7B000340EE26FE46BE569000128EC0FF059D00C
:10C7C0000ED0FFC8E9FF090100C9EAFFEFCF45F924
:10C7D000010E476F45C948F90001DCEC13F049D060
:10C7E0000901366B3769090EE36F340EE26FE46BB3
:10C7F000E569000128EC0FF03CD062390901456F72
:10C800000F0E451745510F0B2E6F62C045F945516C
:10C810000F0B2F6F000162310901466F000161317A
:10C820000901456F46334533463345334633453377
:10C830000F0E461745510F0B306F000161510F0B62
:10C840000901316F3269090EE36F2C0EE26FE46B60
:10C85000E569000128EC0FF00CD0FFC8E9FF00C922
:10C86000EAFFEFCF45F945C947F90001C3EC13F0E2
:10C8700000D00BD0FFC8E9FF00C9EAFFEFCF45F9B0
:10C8800045C947F90001C3EC13F076EF69F0020ED9
:10C890000801FF25E96E000E09010021EA6EEF5044
:10C8A0000608D8A441D2040E0801FF25E96E000E47
:10C8B00009010021EA6EEF3C2BD2030E0801FF258F
:10C8C000E96E000E09010021EA6EEF50080A00012E
:10C8D0000FE0180A21E0010AD8B491D0030AD8B4B5
:10C8E00001D1310AD8B480D12D0AD8B492D102D264
:10C8F0004EBC04D0020E0901366F03D0030E0901AD
:10C90000366F3769090EE36F340EE26FE46BE56949
:10C91000000128EC0FF0FAD185A610D0FFC8E9FF7E
:10C92000090100C9EAFFEFCF45F9010E476F45C97C
:10C9300048F90001DCEC13F076EF69F00F0E090105
:10C94000046F056B090EE36F040EE26F010EE46FD6
:10C950000001F4EC0FF0270E0901636F100E626FF7
:10C96000000146EC14F0012C3BD0090EEA6E180EC3
:10C97000E96E006A026A140E016E3BEC07F0120EBB
:10C980000901446F090EE36F180EE26F090EE56F9F
:10C99000440EE46F000129EC10F0012C12D01BC9E9
:10C9A0002EF91CC92FF909013069090EE36F2C0E0D
:10C9B000E26FE46BE569000128EC0FF076EF69F0B7
:10C9C0000ED0FFC8E9FF090100C9EAFFEFCF45F922
:10C9D000010E476F45C948F90001DCEC13F00ED099
:10C9E000FFC8E9FF090100C9EAFFEFCF45F9010ED1
:10C9F000476F45C948F90001DCEC13F087D185A6E3
:10CA000010D0FFC8E9FF090100C9EAFFEFCF45F9DF
:10CA1000010E476F45C948F90001DCEC13F076EFD1
:10CA200069F00D0E0901046F056B090EE36F040E2A
:10CA3000E26F010EE46F0001F4EC0FF0270E090124
:10CA4000636F100E626F000146EC14F0012C3BD0B6
:10CA5000090EEA6E180EE96E006A026A140E016E83
:10CA60003BEC07F0120E0901446F090EE36F180E3C
:10CA7000E26F090EE56F440EE46F000129EC10F03F
:10CA8000012C12D01BC92EF91CC92FF909013069DC
:10CA9000090EE36F2C0EE26FE46BE569000128ECF0
:10CAA0000FF076EF69F00ED0FFC8E9FF090100C969
:10CAB000EAFFEFCF45F9010E476F45C948F900017C
:10CAC000DCEC13F00ED0FFC8E9FF090100C9EAFF52
:10CAD000EFCF45F9010E476F45C948F90001DCEC7D
:10CAE00013F014D185A610D0FFC8E9FF090100C9D1
:10CAF000EAFFEFCF45F9010E476F45C948F900013C
:10CB0000DCEC13F076EF69F00E0E0901046F056B93
:10CB1000090EE36F040EE26F010EE46F0001F4EC06
:10CB20000FF0270E0901636F100E626F000146ECD3
:10CB300014F0012C4AD0090EEA6E180EE96E006A54
:10CB4000026A140E016E3BEC07F0090EEA6E380E15
:10CB5000E96E006A026A0C0E016E3BEC07F0120EE1
:10CB60000901446F090EE36F180EE26F090EE56FBD
:10CB7000440EE46F000129EC10F0012C26D00801CE
:10CB80003939006EF00E0016005080090901386F27
:10CB9000500E396F1BC93AF91CC93BF91DC93CF944
:10CBA0001EC93DF91FC93EF920C93FF921C940F905
:10CBB00022C941F94269090EE36F380EE26FE46B56
:10CBC000E569000128EC0FF091D3FFC8E9FF0901E6
:10CBD00000C9EAFFEFCF45F9010E476F45C948F993
:10CBE0000001DCEC13F092D05150020804E309017B
:10CBF000366B04D00001010E0901366F3769090E4A
:10CC0000E36F340EE26FE46BE569000128EC0FF08E
:10CC10007DD0160E0901046F056B090EE36F040E3B
:10CC2000E26F010EE46F0001F4EC0FF0270E090132
:10CC3000636F100E626F000146EC14F0012C4AD0B5
:10CC4000090EEA6E180EE96E006A026A140E016E91
:10CC50003BEC07F0090EEA6E380EE96E006A026AD4
:10CC60000C0E016E3BEC07F0120E0901446F090E29
:10CC7000E36F180EE26F090EE56F440EE46F0001DA
:10CC800029EC10F0012C26D008013939006EF00E85
:10CC90000016005080090901386F500E396F1BC90A
:10CCA0003AF91CC93BF91DC93CF91EC93DF91FC918
:10CCB0003EF920C93FF921C940F922C941F9426929
:10CCC000090EE36F380EE26FE46BE569000128ECB2
:10CCD0000FF00CD3FFC8E9FF090100C9EAFFEFCF4D
:10CCE00045F9010E476F45C948F90001DCEC13F026
:10CCF000FDD20CD0FFC8E9FF00C9EAFFEFCF45F92C
:10CD000045C947F90001C3EC13F000D00CD009016C
:10CD1000FFC8E9FF00C9EAFFEFCF45F945C947F968
:10CD20000001C3EC13F0E2D2020E0801FF25E96E08
:10CD3000000E09010021EA6EEF5008083BE1030EE6
:10CD40000801FF25E96E000E09010021EA6EEF508F
:10CD50000E0A000103E01E0A0DE01FD0FFC8E9FF24
:10CD600000C9EAFFEFCF45F945C947F90001ABEF2C
:10CD70005EF01FD009012E6B3FC82FF940C830F973
:10CD800041C831F93269090EE36F2C0EE26FE46B92
:10CD9000E569000128EC0FF00CD0FFC8E9FF00C9DD
:10CDA000EAFFEFCF45F945C947F90001C3EC13F09D
:10CDB00000D09CD2020E0801FF25E96E000E090189
:10CDC0000021EA6EEF507E08D8A485D2030E080138
:10CDD000FF25E96E000E09010021EA6EEF50010AFD
:10CDE00000010DE0520AD8B445D1070AD8B48BD15E
:10CDF000010AD8B4D1D1030AD8B417D25FD2050E34
:10CE00000801FF25E96E000E09010021EA6EEF3CE2
:10CE100025D1040E0801FF25E96E000E090100214D
:10CE2000EA6EEF50060A00010AE00F0A1CE0030A4E
:10CE30002EE0010A40E07B0AD8B4A1D001D14EB067
:10CE400004D0030E0901366F03D0020E0901366FBC
:10CE50003769090EE36F340EE26FE46BE569000198
:10CE600028EC0FF0F9D04EB204D0030E0901366F52
:10CE700003D0020E0901366F3769090EE36F340ED5
:10CE8000E26FE46BE569000128EC0FF0E5D083AABE
:10CE900004D0030E0901366F03D0020E0901366F6C
:10CEA0003769090EE36F340EE26FE46BE569000148
:10CEB00028EC0FF0D1D085A60FD0FFC8E9FF0901FB
:10CEC00000C9EAFFEFCF45F9010E476F45C948F9A0
:10CED0000001DCEC13F00AD2110E0901046F056B9E
:10CEE000090EE36F040EE26F010EE46F0001F4EC33
:10CEF0000FF0270E0901636F100E626F000146EC00
:10CF000014F0012C2CD0090EEA6E180EE96E006A9E
:10CF1000026A140E016E3BEC07F0120E0901446F19
:10CF2000090EE36F180EE26F090EE56F440EE46F11
:10CF3000000129EC10F0012C12D01BC92EF91CC9DC
:10CF40002FF960C030F909013169090EE36F2C0E29
:10CF5000E26FE46BE569000128EC0FF0C7D1FFC870
:10CF6000E9FF090100C9EAFFEFCF45F9010E476F5C
:10CF700045C948F90001DCEC13F0B8D16DD085A6A5
:10CF80000FD0FFC8E9FF090100C9EAFFEFCF45F95B
:10CF9000010E476F45C948F90001DCEC13F0A6D13A
:10CFA000140E0901046F056B090EE36F040EE26FA6
:10CFB000010EE46F0001F4EC0FF0270E0901636F1E
:10CFC000100E626F000146EC14F0012C2AD0090EFD
:10CFD000EA6E180EE96E006A026A140E016E3BECEE
:10CFE00007F0120E0901446F090EE36F180EE26F8D
:10CFF000090EE56F440EE46F000129EC10F0012CDE
:10D0000010D01BC92EF91CC92FF909013069090E6E
:10D01000E36F2C0EE26FE46BE569000128EC0FF082
:10D0200065D1FFC8E9FF090100C9EAFFEFCF45F963
:10D03000010E476F45C948F90001DCEC13F00CD034
:10D04000FFC8E9FF00C9EAFFEFCF45F945C947F935
:10D050000001C3EC13F000D00CD00901FFC8E9FFB8
:10D0600000C9EAFFEFCF45F945C947F90001C3EC14
:10D0700013F02FD1040E0801FF25E96E000E0901FF
:10D080000021EA6EEF3C33D0036B090E476F030EAD
:10D09000466F0001CCEF5EF0012C19D009012E6B18
:10D0A0002F6B0339006E0F0E001600500F0B306F00
:10D0B00003510F0B316F3269090EE36F2C0EE26FD3
:10D0C000E46BE569000128EC0FF003D10ED0FFC836
:10D0D000E9FF090100C9EAFFEFCF45F9010E476FEB
:10D0E00045C948F90001DCEC13F00CD00901FFC878
:10D0F000E9FF00C9EAFFEFCF45F945C947F900014B
:10D10000C3EC13F0E6D0040E0801FF25E96E000E13
:10D1100009010021EA6EEF3C33D0036B090E476F23
:10D12000030E466F000102EF5FF0012C19D00901D8
:10D130002E6B2F6B0339006E0F0E001600500F0B75
:10D14000306F03510F0B316F3269090EE36F2C0EF4
:10D15000E26FE46BE569000128EC0FF0BAD00ED065
:10D16000FFC8E9FF090100C9EAFFEFCF45F9010E49
:10D17000476F45C948F90001DCEC13F00CD00901F8
:10D18000FFC8E9FF00C9EAFFEFCF45F945C947F9F4
:10D190000001C3EC13F09DD0040E0801FF25E96ED9
:10D1A000000E09010021EA6EEF3C33D0036B090E3B
:10D1B000476F030E466F000137EF5FF0012C19D067
:10D1C00009012E6B2F6B0339006E0F0E00160050F5
:10D1D0000F0B306F03510F0B316F3269090EE36F84
:10D1E0002C0EE26FE46BE569000128EC0FF071D0C2
:10D1F0000ED0FFC8E9FF090100C9EAFFEFCF45F9EA
:10D20000010E476F45C948F90001DCEC13F00CD062
:10D210000901FFC8E9FF00C9EAFFEFCF45F945C999
:10D2200047F90001C3EC13F054D0040E0801FF25A8
:10D23000E96E000E09010021EA6EEF3C33D0036B6A
:10D24000090E6B6F030E6A6F00017CEC27F0012C56
:10D2500019D009012E6B2F6B0339006E0F0E0016CB
:10D2600000500F0B306F03510F0B316F3269090EF5
:10D27000E36F2C0EE26FE46BE569000128EC0FF020
:10D2800028D00ED0FFC8E9FF090100C9EAFFEFCF9F
:10D2900045F9010E476F45C948F90001DCEC13F070
:10D2A0000CD00901FFC8E9FF00C9EAFFEFCF45F93B
:10D2B00045C947F90001C3EC13F00BD0FFC8E9FFE3
:10D2C00000C9EAFFEFCF45F945C947F90001C3ECB2
:10D2D00013F00CD00901FFC8E9FF00C9EAFFEFCF46
:10D2E00045F945C947F90001C3EC13F064EF6AF052
:10D2F0000801F7C8E9FFF8C8EAFF3951EF5C21E0FF
:10D30000F7C8E9FFF8C8EAFF3A51EF5C1AE0F7C83E
:10D31000E9FFF8C8EAFFEF50880813E0F7C8E9FF13
:10D32000F8C8EAFFEF5089080CE0F8C8E3F9F7C83D
:10D33000E2F90901E46BE569000128EC0FF026D160
:10D340000801F7C8E9FFF8C8EAFF3A51EF5C02E1CB
:10D350004C8C5B82F7C8E9FFF8C8EAFFEF508808F9
:10D360004FE1010EF725E96E000EF821EA6EEF504D
:10D37000300812E1030EF725E96E000EF821EA6E7F
:10D38000EF3C0AD0F8C800F9F7C8FFF80001BDEF7C
:10D390000FF04C9CFBD00801010EF725E96E000E42
:10D3A000F821EA6EEF2C20D0020EF725E96E000E70
:10D3B000F821EA6EEF5218E1030EF725E96E000E30
:10D3C000F821EA6EEF2C10D0040EF725E96E000E5E
:10D3D000F821EA6EEF3C08D0F8C800F9F7C8FFF86A
:10D3E0000001DBEF0FF0D2D0F8C8E3F9F7C8E2F99B
:10D3F0000901E46BE569000128EC0FF0C7D00801D2
:10D40000F7C8E9FFF8C8EAFFEF5089083BE1010ED1
:10D41000F725E96E000EF821EA6EEF50090825E1C4
:10D42000020EF725E96E000EF821EA6EEF521DE1BB
:10D43000030EF725E96E000EF821EA6EEF500208A0
:10D4400014E1040EF725E96E000EF821EA6EEF3CB8
:10D450000CD0F7C8E9FFF8C8EAFFEFCFFFF8FFC824
:10D4600047F9000153EC12F091D0F7C8E9FFF8C872
:10D47000EAFFEFCFFFF8FFC847F90001C3EC13F054
:10D4800085D00801010EF725E96E000EF821EA6E3D
:10D49000EF2C0AD0F8C800F9F7C8FFF8000152EFE6
:10D4A0003EF074D012D00801010EF725E96E000E8F
:10D4B000F821EA6EEF50090809E1F8C800F9F7C849
:10D4C000FFF800016DEF5FF061D00801020EF72553
:10D4D000E96E000EF821EA6EEF3C4DD0010EF72503
:10D4E000E96E000EF821EA6EEF50210809E0010E06
:10D4F000F725E96E000EF821EA6EEF50220818E1D8
:10D50000F7C8E9FFF8C8EAFFEF38006EF00E001622
:10D5100000508009F96F010EF725E96E000EF82121
:10D52000EA6EEF504009FA6F040EFB6FFC6917D0EA
:10D53000F7C8E9FFF8C8EAFFEF38006EF00E0016F2
:10D5400000508009F96F010EF725E96E000EF821F1
:10D55000EA6EEF504009FA6F050EFB6FFC69080E8A
:10D560000901E36FF90EE26FE46BE569000128EC55
:10D570000FF00CD00BD0F7C8E9FFF8C8EAFFEFCFE7
:10D58000FFF8FFC847F90001C3EC13F012000801CF
:10D59000A06B9F6B3A0EBA6F520EBB6F460EBC6FFC
:10D5A000430EBD6F450EBE6F300EBF6FC06FC16FB3
:10D5B000C26B3A0EC46F570EC56F460EC66F380E5B
:10D5C000C76F360EC86F310EC96F300ECA6F320E7C
:10D5D000CB6FCC6B3A0ED06F570ED16F460ED26F19
:10D5E000380ED36F450ED46F300ED56FD66F330E15
:10D5F000D76FD86B3A0EDC6F570EDD6F460EDE6FBD
:10D60000DF6F330EE06F320EE16F300EE26FE36FCB
:10D61000E46B3A0EE86F770EE96F460EEA6F440E40
:10D62000EB6F340EEC6F360EED6F300EEE6F320E88
:10D63000EF6F340EF06F300EF16FF26BF56BF46B31
:10D64000F66B080E0901F16FBA0EF06F080EF36F5A
:10D650009F0EF26F0001DCEC0CF0012C08D00801E9
:10D660009F3D03D0A05301E1F62B14D00001080127
:10D67000F42BD8B4F52BF55303E1F451640803E21D
:10D68000FF0E016EC2D0050E0C01B66F00016BECEF
:10D6900007F00801080EF86FA10EF76F180EF96F6A
:10D6A00000016CEC0FF0012C09D0080E0801F86F96
:10D6B000A10EF76F00011CDE0801ECD70801F6533C
:10D6C0000CE0F651030802E209D007D0050E0C0168
:10D6D000B66F00016BEC07F00801B3D7030E090128
:10D6E000306F0001F8EC1BF0012C01D00CD0050EBE
:10D6F0000C01B66F00016BEC07F0030E0901306FEF
:10D700000001F8EC1BF009016A6B00019BEC2EF0A4
:10D71000080E0901D06FC40ECF6F0001DBEC14F0CE
:10D72000080E0901D06FD00ECF6F0001DBEC14F0B2
:10D73000080E0801F86FA10EF76F180EF96F0001BF
:10D740006CEC0FF0012C08D0080E0801F86FA10E48
:10D75000F76F0001CDDDECD7080E0901D06FDC0EAC
:10D76000CF6F0001DBEC14F0020E09016A6F0001BB
:10D77000AFEC31F0280E09012F6F00019DEC3BF05A
:10D78000080E0801F86FA10EF76F180EF96F00016F
:10D790006CEC0FF0012C08D0080E0801F86FA10EF8
:10D7A000F76F0001A5DDECD7500E09012F6F0001C6
:10D7B00075EC3DF0700E09012F6F00019BEC3CF001
:10D7C000300E09016A6F000190EC33F0080E080179
:10D7D000F86FA10EF76F180EF96F00016CEC0FF0E7
:10D7E000012C08D0080E0801F86FA10EF76F000198
:10D7F0007FDDECD7080E0901D06FE80ECF6F000176
:10D80000DBEC14F0010E016E080100011200900E15
:10D8100008016C6F380E6D6F6E696F6B6B39006E3F
:10D82000F00E0016005080096C6F080E0901E36FBE
:10D830006C0EE26FE46BE569000128EC0FF0DDEFA0
:10D840008FF00900F6CF89F8F7CF8AF8F8CF8BF878
:10D85000F550A4A8FED76D6E89C8F6FF8AC8F7FFF9
:10D860008BC8F8FF0801882F01D002D00001E9D74A
:10D87000000194EF7CF0080189BF10D00F0E006EFC
:10D88000883900160A0E005C03E2300E002602D032
:10D89000895100260050A4A8FED76D6E0F0E881780
:10D8A0000A0E885D02E2300E02D0899F89518827D6
:10D8B0008851A4A8FED76D6E00019CEF7CF00A0E83
:10D8C000006E002EFED70000959C8C9C0A0E006E08
:10D8D000002EFED700001200020E006E002EFED7B2
:10D8E0000000958E020E006E002EFED70000120082
:10D8F0000A0E006E002EFED70000958C0A0E006EF8
:10D90000002EFED700001200020E006E002EFED781
:10D910000000959E8C9E020E006E002EFED7000029
:10D9200012000601C1970001CADFD6DFE1DFECDF9C
:10D930000A0E006E002EFED70000C1DF1200EF526B
:10D9400010E0EACFEAF8E9CFE9F8EFCF1EFA33ECBE
:10D950000BF0EAC8EAFFE9C8E9FFE92AD8B4EA2AE5
:10D96000EED7E3EF6CF00801E86BE86BE8510708CD
:10D970001CE30001A4DF070ED8800801E855E96F19
:10D98000E7C800F0E951016E04E0D8900032012EA2
:10D99000FCD700A004D000019FDF03D008010001E4
:10D9A000B3DFA6DF0801E82BE1D7000188DF94DFB1
:10D9B0009FDF83BE04D0000E016E08D007D0EA6A54
:10D9C000020EE96EBCD7010E016E00D0120077DFA7
:10D9D0009BDF8EDF81DF0A0E006E002EFED7000077
:10D9E00012009FDF0801E351FE0BE66FE76F0001B5
:10D9F000BADFE4C8E7F8B7DFE5C8E7F8B4DFE7DF88
:10DA000012000900F55211E0F6CFB6FCF7CFB7FCD3
:10DA1000F8CFB8FCF550A4A8FED76D6EB6CCF6FFD3
:10DA2000B7CCF7FFB8CCF8FFECD712003A0E0801DC
:10DA3000886F570E896F310E8A6F370E8B6F300EDD
:10DA40008C6F310E8D6F8E6F8F6F906B3A0E926F61
:10DA5000570E936F460E946F430E956F410E966F5F
:10DA6000430E976F300E986F996F9A6B9C6B9D6BFE
:10DA70009E9151C09CF8540EE36F170EE46F020E96
:10DA8000E56F0001AEDF540E0801E36FE46B1C0E7E
:10DA9000E56F0001A6DF540E0801E36F010EE46F8D
:10DAA000100EE56F00019DDF08019C51010A000185
:10DAB00013E0030A2DE0010A47E0070A61E0010ACA
:10DAC000D8B47AD0030AD8B493D0010AD8B4ACD071
:10DAD000070AD8B4C5D0C4D0540E0801E36F300E85
:10DAE000E46F6C0EE56F00017CDF540E0801E36FFC
:10DAF000310EE46F010EE56F000173DF4AAE07D00F
:10DB0000A80EF66E060EF76E000EF86E7ADFC4D021
:10DB1000540E0801E36F300EE46F7C0EE56F0001D8
:10DB200060DF540E0801E36F310EE46F010EE56F04
:10DB3000000157DF4AAE07D0BE0EF66E060EF76E36
:10DB4000000EF86E5EDFA8D0540E0801E36F300EB1
:10DB5000E46F340EE56F000144DF540E0801E36FFB
:10DB6000310EE46F010EE56F00013BDF4AAE07D0D6
:10DB7000D00EF66E060EF76E000EF86E42DF8CD0F9
:10DB8000540E0801E36F300EE46F740EE56F000170
:10DB900028DF540E0801E36F310EE46F010EE56FCC
:10DBA00000011FDF4AAE07D0E20EF66E060EF76EDA
:10DBB000000EF86E26DF70D0540E0801E36F300EB1
:10DBC000E46F840EE56F00010CDF540E0801E36F73
:10DBD000310EE46F010EE56F000103DF4AAE07D09E
:10DBE000F40EF66E060EF76E000EF86E0ADF54D0D5
:10DBF000540E0801E36F300EE46F2C0EE56F000148
:10DC0000F0DE540E0801E36F310EE46F010EE56F94
:10DC10000001E7DE4AAE07D0060EF66E070EF76E7D
:10DC2000000EF86EEEDE38D0540E0801E36F300EB1
:10DC3000E46F6C0EE56F0001D4DE540E0801E36F53
:10DC4000310EE46F010EE56F0001CBDE4AAE07D066
:10DC5000180EF66E070EF76E000EF86ED2DE1CD0B0
:10DC6000540E0801E36F300EE46F2C0EE56F0001D7
:10DC7000B8DE540E0801E36F310EE46F010EE56F5C
:10DC80000001AFDE4AAE07D02A0EF66E070EF76E21
:10DC9000000EF86EB6DE00D09484000E82B4010E41
:10DCA000006E003808019D6FF00E9D179482000EE3
:10DCB00082B2010E006ED890003600509D13948001
:10DCC000000E82B0010E9D139C51010A00010FE06D
:10DCD000030A17E0010A1FE0070A27E0010A2DE006
:10DCE000030A35E0010A3CE0070A44E043D008019A
:10DCF0009D51100805E0330E8E6F300E8F6F9E81A0
:10DD000044D008019D51120805E0310E8E6F320E8D
:10DD10008F6F9E813AD008019D2D01D005D0300E25
:10DD20008E6F310E8F6F9E8130D008019D5304E0BD
:10DD3000300E8E6F8F6F9E8128D008019D51020892
:10DD400005E0300E8E6F320E8F6F9E811ED008015F
:10DD50009D51110804E0310E8E6F8F6F9E8115D09A
:10DD600008019D51100805E0310E8E6F300E8F6F47
:10DD70009E810BD008019D51110805E0330E8E6F76
:10DD8000310E8F6F9E8101D000D09EA11ED04AAE71
:10DD900008D03C0EF66E070EF76E000EF86E00010E
:10DDA00030DE080E0901D06F880ECF6F0001DBEC6A
:10DDB00014F0030E0901306F0001F8EC1BF0320E75
:10DDC0000C01B66F00016BEC07F0080E0901D06F73
:10DDD000920ECF6F0001DBEC14F0FA0E0C01B66F5F
:10DDE00000016BEC07F0C7EC6AF0B1EF7CF03A0E83
:10DDF00008018A6F770E8B6F460E8C6F8D6F330E16
:10DE00008E6F300E8F6F906F916F926F936F946BD8
:10DE10008951020805E1310E916F300E936F02D0E7
:10DE2000300E916F080E0901D06F8A0ECF6F00017E
:10DE3000DBEC14F0012C0BD008018951020802E13F
:10DE40004F8401D04F94010E016E04D00001FF0EEB
:10DE5000016E08010001120008018C6B8B6B8D6B49
:10DE60008E6B150E8F6F240E906F160E916FB00E85
:10DE7000926FD00E936F300E946FD60E956F800E0A
:10DE8000966F730E976F010E986F760E996F9A6B5F
:10DE9000550E9B6F200E9C6F180E9D6F460E9E6F49
:10DEA000170E9F6F020EA06F560EA16F280EA26F65
:10DEB000300EA36F1B0EA46F310EA56F820EA66FDE
:10DEC000320EA76F800EA86F330EA96F180EAA6FBF
:10DED000300EAB6F160EAC6F310EAD6F020EAE6F23
:10DEE000320EAF6FC00EB06F330EB16F0C0EB26F4B
:10DEF000300EB36F160EB46F310EB56F020EB66FE3
:10DF0000320EB76FC00EB86F330EB96F140EBA6F02
:10DF1000300EBB6F6E0EBC6F310EBD6F020EBE6F4A
:10DF2000320EBF6F800EC06F330EC16F180EC26FFE
:10DF3000300EC36F840EC46F310EC56F020EC66FF4
:10DF4000320EC76FC00EC86F330EC96F0C0ECA6F8A
:10DF5000300ECB6F840ECC6F310ECD6F020ECE6FB4
:10DF6000320ECF6FC00ED06F330ED16F140ED26F42
:10DF7000300ED36F1B0ED46F310ED56F820ED66F5D
:10DF8000320ED76F800ED86F330ED96F180EDA6F3E
:10DF9000300EDB6F160EDC6F310EDD6F020EDE6FA2
:10DFA000320EDF6FC00EE06F330EE16F0C0EE26FCA
:10DFB000720EE36F960EE46FC00EE56F000111DD87
:10DFC000720E0801E36F970EE46FE56B000109DD47
:10DFD000720E0801E36FA10EE46F200EE56F0001E1
:10DFE00000DD010E0C01B66F00016BEC07F0720E44
:10DFF0000801E36FA10EE46F300EE56F0001F1DC64
:10E00000010E0C01B66F00016BEC07F0720E0801F7
:10E01000E36FA10EE46F380EE56F0001E2DC010E44
:10E020000C01B66F00016BEC07F0720E0801E36F94
:10E03000A10EE46F3C0EE56F0001D3DC010E0C0174
:10E04000B66F00016BEC07F0720E0801E36FA10ED2
:10E05000E46F7C0EE56F0001C4DC010E0C01B66FAD
:10E0600000016BEC07F0720E0801E36FA10EE46F84
:10E070003C0EE56F0001B5DC010E0C01B66F00012E
:10E080006BEC07F0720E0801E36F960EE46FC00EA2
:10E09000E56F0001A6DC720E0801E36F410EE46F2C
:10E0A000100EE56F00019DDC720E0801E36F960E05
:10E0B000E46F040EE56F000194DC720E0801E36F5B
:10E0C000970EE46FE56B00018CDC720E0801E36FC4
:10E0D000410EE46F100EE56F000183DC720E080143
:10E0E000E36F0A0EE46F010EE56F00017ADC720E39
:10E0F0000801E36F9D0EE46F610EE56F000171DCB6
:10E10000720E0801E36FBA0EE46F600EE56F000156
:10E1100068DC720E0801E36F560EE46F080EE56FBF
:10E1200000015FDC720E0801E36F150EE46F040E50
:10E13000E56F000156DC720E0801E36F160EE46F06
:10E14000300EE56F00014DDC720E0801E36FD00E5A
:10E15000E46F300EE56F000144DC720E0801E36FDE
:10E16000D60EE46F800EE56F00013BDC720E0801F5
:10E17000E36F0A0EE46F010EE56F000132DC720EF0
:10E180000801E36F150EE46F240EE56F000129DC32
:10E19000720E0801E36F730EE46F010EE56F00016C
:10E1A00020DC720E0801E36F160EE46FB00EE56F0F
:10E1B000000117DC720E0801E36F180EE46F460EC3
:10E1C000E56F00010EDC720E0801E36F550EE46F7F
:10E1D000200EE56F000105DC720E0801E36F170EDB
:10E1E000E46F020EE56F0001F1EC6CF0720E0801B5
:10E1F000E36F560EE46F280EE56F0001F1EC6CF052
:10E20000720E0801E36FAF0EE46F160EE56F0001AA
:10E21000F1EC6CF04AAE08D0F80EF66E090EF76E0F
:10E22000000EF86E01EC6DF008018C6B8B6B8C535B
:10E2300031E18B5109082EE3D8908B35E36F8C3593
:10E24000E46F8F0EE325E96E080EE421EA6EEFCF4E
:10E250008DF8D8908B35E36F8C35E46F010EE32594
:10E26000016E000EE421036E01508F0FE96E080E5F
:10E270000320EA6EEFCF8EF8720EE36F8DC8E4F8DC
:10E280008EC8E5F80001F1EC6CF008018B2BD8B4D6
:10E290008C2BCDD75450F80FD8B01DD2080F0001E9
:10E2A00033EF74F008018C6B8B6B8C5331E18B5125
:10E2B00003082EE3D8908B35E36F8C35E46FA30E03
:10E2C000E325E96E080EE421EA6EEFCF8DF8D890D1
:10E2D0008B35E36F8C35E46F010EE325016E000E84
:10E2E000E421036E0150A30FE96E080E0320EA6ECD
:10E2F000EFCF8EF8720EE36F8DC8E4F88EC8E5F8A4
:10E300000001F1EC6CF008018B2BD8B48C2BCDD72D
:10E310004AAE0AD0040EF66E0A0EF76E000EF86EC4
:10E32000000101EC6DF00801D6D108018C6B8B6BFC
:10E330008C5331E18B5103082EE3D8908B35E36F7A
:10E340008C35E46FAB0EE325E96E080EE421EA6E2E
:10E35000EFCF8DF8D8908B35E36F8C35E46F010EDD
:10E36000E325016E000EE421036E0150AB0FE96E50
:10E37000080E0320EA6EEFCF8EF8720EE36F8DC8A1
:10E38000E4F88EC8E5F80001F1EC6CF008018B2B85
:10E39000D8B48C2BCDD74AAE0AD01C0EF66E0A0E1E
:10E3A000F76E000EF86E000101EC6DF0080193D1DC
:10E3B00008018C6B8B6B8C5331E18B5103082EE37E
:10E3C000D8908B35E36F8C35E46FB30EE325E96E9F
:10E3D000080EE421EA6EEFCF8DF8D8908B35E36F0D
:10E3E0008C35E46F010EE325016E000EE421036E0F
:10E3F0000150B30FE96E080E0320EA6EEFCF8EF8DE
:10E40000720EE36F8DC8E4F88EC8E5F80001F1ECF8
:10E410006CF008018B2BD8B48C2BCDD74AAE0AD028
:10E42000360EF66E0A0EF76E000EF86E000101EC65
:10E430006DF0080150D108018C6B8B6B8C5331E16E
:10E440008B5103082EE3D8908B35E36F8C35E46F46
:10E45000BB0EE325E96E080EE421EA6EEFCF8DF8DE
:10E46000D8908B35E36F8C35E46F010EE325016E98
:10E47000000EE421036E0150BB0FE96E080E03206D
:10E48000EA6EEFCF8EF8720EE36F8DC8E4F88EC897
:10E49000E5F80001F1EC6CF008018B2BD8B48C2B63
:10E4A000CDD74AAE0AD04C0EF66E0A0EF76E000EAD
:10E4B000F86E000101EC6DF008010DD108018C6BC4
:10E4C0008B6B8C5331E18B5103082EE3D8908B3545
:10E4D000E36F8C35E46FC30EE325E96E080EE4218B
:10E4E000EA6EEFCF8DF8D8908B35E36F8C35E46F03
:10E4F000010EE325016E000EE421036E0150C30FEF
:10E50000E96E080E0320EA6EEFCF8EF8720EE36F0D
:10E510008DC8E4F88EC8E5F80001F1EC6CF0080154
:10E520008B2BD8B48C2BCDD74AAE0AD0620EF66EA8
:10E530000A0EF76E000EF86E000101EC6DF0080196
:10E54000CAD008018C6B8B6B8C5331E18B51030863
:10E550002EE3D8908B35E36F8C35E46FCB0EE3253B
:10E56000E96E080EE421EA6EEFCF8DF8D8908B3576
:10E57000E36F8C35E46F010EE325016E000EE4219C
:10E58000036E0150CB0FE96E080E0320EA6EEFCF49
:10E590008EF8720EE36F8DC8E4F88EC8E5F80001BE
:10E5A000F1EC6CF008018B2BD8B48C2BCDD74AAE94
:10E5B0000AD0780EF66E0A0EF76E000EF86E0001A5
:10E5C00001EC6DF0080187D008018C6B8B6B8C53CC
:10E5D00031E18B5103082EE3D8908B35E36F8C35F6
:10E5E000E46FD30EE325E96E080EE421EA6EEFCF67
:10E5F0008DF8D8908B35E36F8C35E46F010EE325F1
:10E60000016E000EE421036E0150D30FE96E080E77
:10E610000320EA6EEFCF8EF8720EE36F8DC8E4F838
:10E620008EC8E5F80001F1EC6CF008018B2BD8B432
:10E630008C2BCDD74AAE0AD08E0EF66E0A0EF76E30
:10E64000000EF86E000101EC6DF0080144D00801E5
:10E650008C6B8B6B8C5331E18B5103082EE3D8907C
:10E660008B35E36F8C35E46FDB0EE325E96E080E26
:10E67000E421EA6EEFCF8DF8D8908B35E36F8C35BF
:10E68000E46F010EE325016E000EE421036E0150DC
:10E69000DB0FE96E080E0320EA6EEFCF8EF8720EE4
:10E6A000E36F8DC8E4F88EC8E5F80001F1EC6CF07A
:10E6B00008018B2BD8B48C2BCDD74AAE0AD0A40E30
:10E6C000F66E0A0EF76E000EF86E000101EC6DF0AA
:10E6D000080101D00801720EE36F340EE46F050EDD
:10E6E000E56F0001F1EC6CF0720E0801E36F170E9C
:10E6F000E46F020EE56F0001F1EC6CF0720E0801A0
:10E70000E36FBA0EE46F200EE56F0001F1EC6CF0E0
:10E71000720E0801E36FD50EE46F100EE56F000175
:10E72000F1EC6CF0720E0801E36FD60EE46F880E08
:10E73000E56F0001F1EC6CF0720E0801E36FA10EC1
:10E74000E46F1C0EE56F0001F1EC6CF0010E0C01A2
:10E75000B66F00016BEC07F0720E0801E36FA10EBB
:10E76000E46F0C0EE56F0001F1EC6CF0010E0C0192
:10E77000B66F00016BEC07F0720E0801E36FA10E9B
:10E78000E46F040EE56F0001F1EC6CF0010E0C017A
:10E79000B66F00016BEC07F0720E0801E36FA10E7B
:10E7A000E46FE56B0001F1EC6CF0010E0C01B66F4B
:10E7B00000016BEC07F0720E0801E36FD50EE46FF9
:10E7C000E56B0001F1EC6CF0720E0801E36FD60E00
:10E7D000E46F800EE56F0001F1EC6CF04BA028D0E7
:10E7E000720E0801E36F160EE46F300EE56F000144
:10E7F000F1EC6CF0720E0801E36F180EE46FC60EB8
:10E80000E56F0001F1EC6CF0720E0801E36F550E3C
:10E81000E46FE56B0001F1EC6CF0720E0801E36F40
:10E82000AF0EE46F040EE56F0001F1EC6CF00AD05E
:10E83000720E0801E36FAF0EE46F060EE56F000184
:10E84000F1EC6CF008014B914B834AAE0AD0BA0E42
:10E85000F66E0A0EF76E000EF86E000101EC6DF018
:10E86000080100011200E824F76AF736870FF66EF8
:10E87000E80EF722000EF86EFB6E0A00F550FA6EF5
:10E880000800F550F96EA4E22AE3B0E336E4BCE4F4
:10E8900042E5C8E54EE60801926B936B00015FEC20
:10E8A0006CF06CEC6CF00801926B925107082FE34E
:10E8B000000178EC6CF0958E83AE12D0070ED880F4
:10E8C00008019255946F010E006E9451016E04E0A0
:10E8D000D8900036012EFCD70050931312D00001BF
:10E8E000070ED88008019255946F010E006E945166
:10E8F000016E04E0D8900036012EFCD70050FF0ACC
:10E90000931700015FEC6CF00801922BCED7915366
:10E9100003E0000184EC6CF0000178EC6CF008017D
:10E9200093C801F00001B7EF74F091EC6CF00801AE
:10E930008B51FE0B8F6FE76F0001B3EC6CF08CC84E
:10E94000E7F8B3EC6CF091EC6CF008018B51010925
:10E950008F6FE76F0001B3EC6CF08EC803F0080115
:10E960008DC88FF88EC890F8916B000194D790C82D
:10E97000EAFF8FC8E9FF01C0EFFFE7EC6CF08EC83B
:10E9800003F008018DC8E9FF8EC8EAFFEFCF01F060
:10E990000001E8EF74F008018A6B892D06D00001B0
:10E9A0002CEC6FF008014A6B1CD0938081B018D01A
:10E9B0004A2B4A51050813E24A6B8A6B720E8B6F21
:10E9C000420E8C6F080E8E6F8A0E8D6F0001ADD7D0
:10E9D00008018AAD04D000012CEC6FF0080101D0D1
:10E9E0004A6B0001120084B408D0080138510308B2
:10E9F00002E0030E386F18D0000184B208D008017D
:10EA00003851020802E0020E386F0ED0000184B0C7
:10EA100008D00801382D01D002D0010E386F04D083
:10EA20000001010E0801386F84A618D04EBA02D03A
:10EA3000882D13D04E9C4E9AF29CF29EF2BEFDD7CA
:10EA4000F0908B9A949AF086C00EF212010E0C018F
:10EA5000B66F00016BEC07F0080119D04EAA02D086
:10EA6000882D15D04E8C4E8AF29CF29EF2BEFDD7B8
:10EA7000F0908B8A949AF096C00EF212010E0C015F
:10EA8000B66F00016BEC07F008012E6B2F6B84A8AA
:10EA90000BD04EAE08D04E9E7C86400E6F6E030E9D
:10EAA0007D6EA60E6C6E08D04EBE06D04E8E7C9645
:10EAB0000C0E6F6EA20E6C6E84BA0CD04FA402D0F6
:10EAC000882D06D0020E896F0001F7EC6EF0080168
:10EAD0004A820BD04FB402D0882D06D0030E896F26
:10EAE0000001F7EC6EF008014A9284BC0BD04BA0F9
:10EAF00002D0882D06D04B80010E896F00014BDFBC
:10EB000008010AD04BB002D0882D06D04B90010EE0
:10EB1000896F000140DF080100011200C582C5B203
:10EB2000FED70C01B651FE0BB96FBB6F0001E6ECCE
:10EB30000FF0B7CCBBFCE6EC0FF0B8CCBBFCE6ECBE
:10EB40000FF0C584C5B4FED71200C582C5B2FED78A
:10EB50000C01B651FE0BBA6FBB6F0001E6EC0FF073
:10EB6000B7CCBBFCE6EC0FF0C582C5B2FED70C01FA
:10EB7000B6510109BA6FBB6F0001E6EC0FF0B9CCDA
:10EB800003F00C01B8CCE9FFB9CCEAFF006A000140
:10EB90001BEC10F001C0EFFFC584C5B4FED7B9CCA3
:10EBA00003F00C01B8CCE9FFB9CCEAFFEFCF01F0DC
:10EBB0000001CDEF7AF00B014F6B4E6B506B516B38
:10EBC000526B546B536B5591566BF30E576F010E8E
:10EBD000586F080E596F020E5A6F5B6B030E5C6F15
:10EBE000020E5D6F040E5E6FBB0E5F6F050E606FF1
:10EBF0000B0E616F060E626F636B070E646F656BC1
:10EC0000080E666F060E676F090E686F010E696F5A
:10EC10000A0E6A6F6B6B0B0E6C6F010E6D6F0C0E34
:10EC20006E6F200E6F6F0D0E706F010E716F0E0EF6
:10EC3000726F736B0F0E746FEE0E756F100E766F32
:10EC4000020E776F110E786F796B120E7A6F7B6BF5
:10EC5000130E7C6F9F0E7D6F140E7E6F880E7F6F7C
:10EC6000806B816B826BB30E836F010E846F080E15
:10EC7000856F020E866F876B060E886F896B070E95
:10EC80008A6F8B6B130E8C6F9F0E8D6F140E8E6FB1
:10EC9000880E8F6F080E906F060E916F090E926F9F
:10ECA000010E936F0A0E946F956B0B0E966F010E0B
:10ECB000976F0C0E986F200E996F0D0E9A6F010EC4
:10ECC0009B6F0E0E9C6F9D6B0F0E9E6F650E9F6F60
:10ECD000100EA06F040EA16F110EA26FA36B120E87
:10ECE000A46FA56B030EA66F020EA76F040EA86F8C
:10ECF000A40EA96F050EAA6F0F0EAB6FAC6BF30ECF
:10ED0000AD6FAE6BAF6F010EB06F870EB16F020EBD
:10ED1000B26FB36B030EB46F010EB56F040EB66F16
:10ED2000200EB76F050EB86F030EB96F060EBA6FDF
:10ED3000BB6B070EBC6FBD6B080EBE6F020EBF6FC4
:10ED4000090EC06F010EC16F0A0EC26FC36B0B0EAE
:10ED5000C46F010EC56F0C0EC66F200EC76F0D0E6F
:10ED6000C86F010EC96F0E0ECA6FCB6B0F0ECC6F42
:10ED7000650ECD6F100ECE6F040ECF6F110ED06FDB
:10ED8000D16B120ED26FD36B130ED46F880ED56F6A
:10ED9000140ED66F880ED76FD86BD96BDA6BF30E63
:10EDA000DB6F010EDC6F080EDD6F020EDE6FDF6BB6
:10EDB000030EE06F010EE16F040EE26FD00EE36F01
:10EDC000050EE46F020EE56F060EE66FE76B070EA9
:10EDD000E86FE96B080EEA6F020EEB6F090EEC6F3D
:10EDE000010EED6F0A0EEE6FEF6B0B0EF06F010E62
:10EDF000F16F0C0EF26F200EF36F0D0EF46F010E1B
:10EE0000F56F0E0EF66FF76B0F0EF86FEE0EF96FD3
:10EE1000100EFA6F020EFB6F110EFC6FFD6B120EDF
:10EE2000FE6FFF6B130E0C01006F880E016F140E46
:10EE3000026F880E036F046B056B066BF30E076F92
:10EE4000010E086F080E096F020E0A6F0B6B030E9E
:10EE50000C6F010E0D6F040E0E6FC00E0F6F050EBE
:10EE6000106F030E116F060E126F136B070E146FE7
:10EE7000156B080E166F020E176F090E186F010E34
:10EE8000196F0A0E1A6F1B6B0B0E1C6F010E1D6F94
:10EE90000C0E1E6F200E1F6F0D0E206F010E216FC6
:10EEA0000E0E226F236B0F0E246F650E256F100E52
:10EEB000266F040E276F110E286F296B120E2A6F12
:10EEC0002B6B130E2C6F880E2D6F140E2E6F880E69
:10EED0002F6F306B316B326BF30E336F010E346F6B
:10EEE000170E356F020E366F376B030E386F010E3B
:10EEF000396F040E3A6FC00E3B6F050E3C6F030E68
:10EF00003D6F060E3E6F3F6B070E406F416B080E64
:10EF1000426F020E436F090E446F010E456F0A0ED9
:10EF2000466F476B0B0E486F010E496F0C0E4A6F10
:10EF3000200E4B6F0D0E4C6F010E4D6F0E0E4E6F6F
:10EF40004F6B0F0E506F650E516F100E526F040E07
:10EF5000536F110E546F556B120E566F576B130E85
:10EF6000586F880E596F140E5A6F880E5B6F5C6B6A
:10EF70005D6B5E6BF30E5F6F010E606F870E616FEE
:10EF8000020E626F636B030E646F010E656F040EF9
:10EF9000666F580E676F050E686F020E696F060E7A
:10EFA0006A6F6B6B070E6C6F6D6B080E6E6F020EE7
:10EFB0006F6F090E706F010E716F0A0E726F736BB7
:10EFC0000B0E746F010E756F0C0E766F200E776F3F
:10EFD0000D0E786F010E796F0E0E7A6F7B6B0F0E30
:10EFE0007C6FEE0E7D6F100E7E6F010E7F6F110E27
:10EFF000806F816B120E826F836B130E846F880E8D
:10F00000856F140E866F880E876F886B896B8A6B8D
:10F01000F30E8B6F010E8C6F080E8D6F020E8E6FCC
:10F020008F6B030E906F010E916F040E926F200E86
:10F03000936F050E946F030E956F060E966F976B88
:10F04000070E986F996B080E9A6F020E9B6F090E50
:10F050009C6F010E9D6F0A0E9E6F9F6B0B0EA06F33
:10F06000010EA16F0C0EA26F200EA36F0D0EA46FE8
:10F07000010EA56F0E0EA66FA76B0F0EA86F650E83
:10F08000A96F100EAA6F040EAB6F110EAC6FAD6BB3
:10F09000120EAE6FAF6B130EB06F880EB16F140E01
:10F0A000B26F880EB36FB46BB56B0B014D51000A94
:10F0B000000115E0010A5CE0030AD8B4A2D0010AFD
:10F0C000D8B4E8D0070AD8B42ED1010AD8B475D183
:10F0D000030AD8B4BCD1010AD8B403D24DD24AAE87
:10F0E00008D0160EF66E080EF76E000EF86E01ECE4
:10F0F0006DF00B014F6B4E6B4F5339E14E511408BD
:10F1000036E3D8904E350C01B66F0B014F350C012C
:10F11000B76F560EB625E96E0B0EB721EA6EEFCF2C
:10F1200050FB0B01D8904E350C01B66F0B014F35DB
:10F130000C01B76F010EB625016E000EB721036EEC
:10F140000150560FE96E0B0E0320EA6EEFCF51FB14
:10F150000B01DC0E0C01B66F50CBB7FC51CBB8FCE9
:10F160000001DCDC0B014E2BD8B44F2BC5D707D2E6
:10F170004AAE08D02C0EF66E080EF76E000EF86E32
:10F1800001EC6DF00B014F6B4E6B4F5339E14E515B
:10F19000150836E3D8904E350C01B66F0B014F358C
:10F1A0000C01B76F820EB625E96E0B0EB721EA6E21
:10F1B000EFCF50FB0B01D8904E350C01B66F0B0111
:10F1C0004F350C01B76F010EB625016E000EB72149
:10F1D000036E0150820FE96E0B0E0320EA6EEFCF33
:10F1E00051FB0B01DC0E0C01B66F50CBB7FC51CBC1
:10F1F000B8FC000193DC0B014E2BD8B44F2BC5D7C4
:10F20000BED14AAE08D0400EF66E080EF76E000E64
:10F21000F86E01EC6DF00B014F6B4E6B4F5339E103
:10F220004E51140836E3D8904E350C01B66F0B01E1
:10F230004F350C01B76FAE0EB625E96E0B0EB72138
:10F24000EA6EEFCF50FB0B01D8904E350C01B66F34
:10F250000B014F350C01B76F010EB625016E000E84
:10F26000B721036E0150AE0FE96E0B0E0320EA6E5C
:10F27000EFCF51FB0B01DC0E0C01B66F50CBB7FC8E
:10F2800051CBB8FC00014ADC0B014E2BD8B44F2BFC
:10F29000C5D775D14AAE08D0580EF66E080EF76E77
:10F2A000000EF86E01EC6DF00B014F6B4E6B4F537F
:10F2B00039E14E51140836E3D8904E350C01B66F43
:10F2C0000B014F350C01B76FDA0EB625E96E0B0E48
:10F2D000B721EA6EEFCF50FB0B01D8904E350C01F1
:10F2E000B66F0B014F350C01B76F010EB625016EDD
:10F2F000000EB721036E0150DA0FE96E0B0E0320EA
:10F30000EA6EEFCF51FB0B01DC0E0C01B66F50CB58
:10F31000B7FC51CBB8FC000101DC0B014E2BD8B47B
:10F320004F2BC5D72CD14AAE08D06E0EF66E080E04
:10F33000F76E000EF86E01EC6DF00B014F6B4E6B2B
:10F340004F533AE14E51140837E3D8904E350C0133
:10F35000B66F0B014F350C01B76F060EB625E96E7F
:10F360000C0EB721EA6EEFCF50FB0B01D8904E3553
:10F370000C01B66F0B014F350C01B76F010EB625AE
:10F38000016E000EB721036E0150060FE96E0C0EE0
:10F390000320EA6EEFCF51FB0B01DC0E0C01B66FC0
:10F3A00050CBB7FC51CBB8FC00018EEC75F00B01D3
:10F3B0004E2BD8B44F2BC4D7E2D04AAE08D0860E1D
:10F3C000F66E080EF76E000EF86E01EC6DF00B0194
:10F3D0004F6B4E6B4F533AE14E51140837E3D890C0
:10F3E0004E350C01B66F0B014F350C01B76F320E65
:10F3F000B625E96E0C0EB721EA6EEFCF50FB0B017C
:10F40000D8904E350C01B66F0B014F350C01B76F1C
:10F41000010EB625016E000EB721036E0150320FAA
:10F42000E96E0C0E0320EA6EEFCF51FB0B01DC0EF0
:10F430000C01B66F50CBB7FC51CBB8FC00018EEC81
:10F4400075F00B014E2BD8B44F2BC4D798D04AAED1
:10F4500008D09E0EF66E080EF76E000EF86E01ECE8
:10F460006DF00B014F6B4E6B4F533AE14E51140848
:10F4700037E3D8904E350C01B66F0B014F350C01B8
:10F48000B76F5E0EB625E96E0C0EB721EA6EEFCFB0
:10F4900050FB0B01D8904E350C01B66F0B014F3568
:10F4A0000C01B76F010EB625016E000EB721036E79
:10F4B00001505E0FE96E0C0E0320EA6EEFCF51FB98
:10F4C0000B01DC0E0C01B66F50CBB7FC51CBB8FC76
:10F4D00000018EEC75F00B014E2BD8B44F2BC4D726
:10F4E0004ED04AAE08D0B40EF66E080EF76E000E7F
:10F4F000F86E01EC6DF00B014F6B4E6B4F533AE120
:10F500004E51140837E3D8904E350C01B66F0B01FD
:10F510004F350C01B76F8A0EB625E96E0C0EB72178
:10F52000EA6EEFCF50FB0B01D8904E350C01B66F51
:10F530000B014F350C01B76F010EB625016E000EA1
:10F54000B721036E01508A0FE96E0C0E0320EA6E9C
:10F55000EFCF51FB0B01DC0E0C01B66F50CBB7FCAB
:10F5600051CBB8FC00018EEC75F00B014E2BD8B4DA
:10F570004F2BC4D704D0000129D00B0100D055B1C6
:10F5800025D0DC0E0C01B66F010EB76F0B0EB96FF4
:10F59000520EB86F0001A5EF75F0780E0C01B66F32
:10F5A00000016BEC07F00B015251060B060808E056
:10F5B0005451000806E2FF0A03E15351F40801E246
:10F5C0005581526B532BD8B4542BD9D7000120EF5F
:10F5D00085F00801B66B979A8E9A00D0929689961C
:10F5E00000D0080EB66FB6531BE0929689960000C5
:10F5F000010EB65DB76FB1C800F0B751016E04E0FF
:10F60000D8900032012EFCD700B002D0899201D0F0
:10F610008982929200009296898600D0B607E3D73D
:10F62000200EB66FB65324E0929689960000010E24
:10F63000B65DB76FB5C803F0B4C802F0B3C801F047
:10F64000B2C800F0B751B86F07E0D8900332023269
:10F6500001320032B82FF9D700B002D0899201D020
:10F660008982929200009296898600D0B607DAD7F6
:10F6700000D092968996978AB66B85BAB62B030E00
:10F68000006E002EFED7000112000A0E08018C6FDA
:10F69000E10E8B6FE40E8A6F8969070E906F210E61
:10F6A0008F6F670E8E6F7F0E8D6F080E946F220E18
:10F6B000936FD70E926F7F0E916F0A0E986FC10EE7
:10F6C000976FE40E966F9569070E9C6F010E9B6F06
:10F6D000670E9A6F7F0E996F070EA06F220E9F6FB5
:10F6E000D70E9E6F7F0E9D6F0A0EA46FE10EA36F63
:10F6F000E40EA26FA169070EA86F210EA76F670E17
:10F70000A66F7F0EA56FA96BAA6BAB6BAC6BAD6BD5
:10F71000AE6BAF6BB06B8851000A000112E0010ABA
:10F7200026E0030A3AE0010A4EE0070A62E0010A15
:10F73000D8B475D0030AD8B488D0010AD8B49BD005
:10F74000B0D04AAE08D0C80EF66E080EF76E000EA6
:10F75000F86E01EC6DF0A9C8B1F88CC8B5F88BC88B
:10F76000B4F88AC8B3F889C8B2F833DF9BD04AAE80
:10F7700008D0F00EF66E080EF76E000EF86E01EC73
:10F780006DF0AAC8B1F890C8B5F88FC8B4F88EC8A3
:10F79000B3F88DC8B2F81DDF85D04AAE08D0180E78
:10F7A000F66E090EF76E000EF86E01EC6DF0ABC848
:10F7B000B1F894C8B5F893C8B4F892C8B3F891C832
:10F7C000B2F807DF6FD04AAE08D03E0EF66E090ED3
:10F7D000F76E000EF86E01EC6DF0ACC8B1F898C889
:10F7E000B5F897C8B4F896C8B3F895C8B2F8F1DE82
:10F7F00059D04AAE08D0620EF66E090EF76E000EB2
:10F80000F86E01EC6DF0ADC8B1F89CC8B5F89BC8B6
:10F81000B4F89AC8B3F899C8B2F8DBDE43D04AAE60
:10F8200008D0880EF66E090EF76E000EF86E01EC29
:10F830006DF0AEC8B1F8A0C8B5F89FC8B4F89EC8BE
:10F84000B3F89DC8B2F8C5DE2DD04AAE08D0AE0ED2
:10F85000F66E090EF76E000EF86E01EC6DF0AFC893
:10F86000B1F8A4C8B5F8A3C8B4F8A2C8B3F8A1C841
:10F87000B2F8AFDE17D04AAE08D0D20EF66E090E3F
:10F88000F76E000EF86E01EC6DF0B0C8B1F8A8C8C4
:10F89000B5F8A7C8B4F8A6C8B3F8A5C8B2F899DEF9
:10F8A00001D000D00FEF7EF00801856B876B866B6F
:10F8B000936881CF52F05230006E00323F0E001636
:10F8C00000500F0B526E0F0E521A52165150525CCE
:10F8D00002E16B2DAFD10A0E0C01B66F00016BEC8B
:10F8E00007F0936881CF85F808018531006E0032FA
:10F8F0003F0E001600500F0B856F0F0E851B8517EE
:10F900005150855D02E16B2D95D185C851F04AAE0D
:10F910001CD0200EF66E0E0EF76E000EF86E0C0E5A
:10F92000886F000121EF6CF085C888F8570E080138
:10F93000896F00013BEF6CF00A0EA4A8FED76D6E34
:10F940000D0EA4A8FED76D6E08015150070801E204
:10F9500071D1030E0901306F0001F8EC1BF016EFB6
:10F960006DF00801876B866B87C867F986C866F9F2
:10F970000901696B320E686F000135EC14F002C0AA
:10F9800089F801C088F80801895323E18851F908F2
:10F9900020E3080EF86F6C0EF76F180EF96F000178
:10F9A0006CEC0FF0012C0AD0080E0801F86F6C0EF9
:10F9B000F76F000178EC69F00801EBD7320E0C010B
:10F9C000B66F00016BEC07F00801862BD8B4872BCB
:10F9D000CBD7010E886F0001F3EC74F05150545CEA
:10F9E00004E051C054F02CEC6FF00801876B866B7B
:10F9F00087C867F986C866F90901696B320E686FB6
:10FA0000000135EC14F002C089F801C088F8080143
:10FA1000895323E18851F90820E3080EF86F6C0E32
:10FA2000F76F180EF96F00016CEC0FF0012C0AD083
:10FA3000080E0801F86F6C0EF76F000178EC69F0A2
:10FA40000801EBD7320E0C01B66F00016BEC07F02A
:10FA50000801862BD8B4872BCBD7978E85BEE1D0F3
:10FA60004AAE0AD0320EF66E0E0EF76E000EF86E2B
:10FA7000000101EC6DF00801876B866B87C867F9A0
:10FA800086C866F90901696B320E686F000135ECB2
:10FA900014F002C089F801C088F80801895323E1F5
:10FAA0008851F90820E3080EF86F6C0EF76F180EF6
:10FAB000F96F00016CEC0FF0012C0AD0080E080160
:10FAC000F86F6C0EF76F000178EC69F00801EBD766
:10FAD000320E0C01B66F00016BEC07F00801862BAB
:10FAE000D8B4872BCBD751C053F053C088F800014E
:10FAF00087D2020E0901306F0001F8EC1BF00801FB
:10FB0000876B866B87C867F986C866F90901696BD8
:10FB1000320E686F000135EC14F002C089F801C0A4
:10FB200088F808010250030824E303E18851E7083C
:10FB300020E3080EF86F6C0EF76F180EF96F0001D6
:10FB40006CEC0FF0012C0AD0080E0801F86F6C0E57
:10FB5000F76F000178EC69F00801EBD7320E0C0169
:10FB6000B66F00016BEC07F00801862BD8B4872B29
:10FB7000C9D7DC0E0C01B66F0A0EB76FA00EB86FB6
:10FB800000018EEC75F00801876B866B87C867F9FA
:10FB900086C866F90901696B320E686F000135ECA1
:10FBA00014F002C089F801C088F8080102501B084F
:10FBB00024E303E18851570820E3080EF86F6C0E28
:10FBC000F76F180EF96F00016CEC0FF0012C0AD0E2
:10FBD000080E0801F86F6C0EF76F000178EC69F001
:10FBE0000801EBD7320E0C01B66F00016BEC07F089
:10FBF0000801862BD8B4872BC9D7DC0E0C01B66F51
:10FC00000A0EB76FB86B00018EEC75F0640E0C0134
:10FC1000B66F00016BEC07F053C088F836D509D0F9
:10FC200008016B5307E1020E0901306F0001F8EC87
:10FC30001BF008010001120008016B6B010E6C6FD4
:10FC4000040E6D6F3F0E6E6F020E6F6F706B7169F9
:10FC5000726B736B746B080E0901306F6B0E2F6F34
:10FC60000001A8EC35F0A8EF90F008016E6B6D6B09
:10FC7000036A2FC802F0D890023603360250C60F2E
:10FC8000E96E060E0320EA6EECCF03F0ED52EFCFE3
:10FC90006DF803C06EF82F51B30802E32F2B01D08B
:10FCA0002F6B6DC801F06EC802F00001AAEF8DF055
:10FCB0000801736B726B716B706B756B746B766B29
:10FCC000776B030E786F6E51050828E2FF0A03E197
:10FCD0006D51A30823E26E51070820E303E16D5143
:10FCE00039081CE3036A026A016A010E006E6F5153
:10FCF000796F07E0D8900036013602360336792F47
:10FD0000F9D700500601C2130150C3130250C413A7
:10FD10000350C513010E0801786F9ED06E51020882
:10FD20002CE2FF0A03E16D51E70827E26E51050856
:10FD300024E303E16D51140820E3036A026A016AB7
:10FD4000010E006E6F51796F07E0D89000360136D2
:10FD500002360336792FF9D7FF0E001A011A021A5C
:10FD6000031A00500601C2170150C3170250C417EE
:10FD70000350C5170801786B6FD06E5106086CE20E
:10FD8000FF0A03E16D51390867E26F510E083EE149
:10FD90000601C251800B0801706F0601C351020BAE
:10FDA0000801716F726B736B0601C53108017D6FBD
:10FDB0000601C43108017C6F0601C33108017B6F65
:10FDC0000601C23108017A6F7D337C337B337A338D
:10FDD0007D337C337B337A337D337C337B337A33AF
:10FDE0007D337C337B337A337D337C337B337A339F
:10FDF000030E7D177A510F0B776F0601C2517F0BEF
:10FE0000E8CF76F8020E0801786F26D06F511308FC
:10FE100021E1706B0601C351800B0801716F06016F
:10FE2000C451010B0801726F736BD8900601C53184
:10FE30000601C4310601C33108011F0B776F0601AB
:10FE4000C351010BE8CF75F8C2C674F8020E080161
:10FE5000786F02D0030E786F78C801F00001BDEF13
:10FE60008DF00801826B81C882F882512A0804E172
:10FE7000010E016E12D011D082512C0804E1020E45
:10FE8000016E0BD00AD082512D0804E1030E016EE1
:10FE900004D003D0000E016E00D000011200080152
:10FEA000846B8331886F8231876F8131866F8833AD
:10FEB0008733863388338733863388338733863373
:10FEC0000F0E881786C884F88451510804E1010E8A
:10FED000016E11D010D0842D04D0020E016E0BD013
:10FEE0000AD08451090804E1030E016E04D003D046
:10FEF000000E016E00D000011200010E0801816F9A
:10FF00008051000A000109E0010A0FE0030A17E02E
:10FF1000010A1EE0070A26E030D0010E0801826FB8
:10FF2000836F030E846F856F2BD00E0E0801826FD6
:10FF3000010E836F020E846F030E856F21D00E0EAB
:10FF40000801826F010E836F846F030E856F18D0D6
:10FF5000010E0801826F0A0E836F030E846F010E7B
:10FF6000856F0ED0010E0801826F0A0E836F030E9B
:10FF7000846F020E856F04D0000121D0080100D0EB
:10FF8000802D01D003D0805102080EE13B510408BE
:10FF900006E23B51080803E3070E826F05D03B5190
:10FFA000080802E2010E826F866B080E0901E36FFA
:10FFB000810EE26F050EE46F0001F4EC0FF0120009
:10FFC000900E08016C6F600E6D6F030E6E6F6F699F
:10FFD0006B39006EF00E0016005080096C6F080E31
:10FFE0000901E36F6C0EE26FE46BE569000128EC38
:06FFF0000FF0FBEF90F0A2
:020000040001F9
:1000000008018A6B896B8B6B8C6B010E8D6F8E6B0D
:10001000020E8F6F906B030E916F9C0E926F040E09
:10002000936F200E946F050E956F550E966F060E0A
:10003000976F986B070E996F5D0E9A6F080E9B6F06
:100040009C6B090E9D6F550E9E6F0A0E9F6FA06BE5
:100050000B0EA16F400EA26F0C0EA36FA46B0D0EC2
:10006000A56F030EA66F0E0EA76FA86B0F0EA96FDC
:10007000400EAA6F100EAB6FAC6B110EAD6F200E61
:10008000AE6F120EAF6F100EB06F130EB16F800E09
:10009000B26F140EB36F1A0EB46F150EB56F1F0E3C
:1000A000B66F160EB76F040EB86F170EB96F040E49
:1000B000BA6F180EBB6F2A0EBC6F190EBD6F200EE3
:1000C000BE6F1A0EBF6F800EC06F1B0EC16F3B0E4E
:1000D000C26F1C0EC36FC4691D0EC56F800EC66F44
:1000E0001E0EC76FA40EC86F1F0EC96FB50ECA6F64
:1000F000200ECB6F0F0ECC6F210ECD6F200ECE6F6A
:10010000220ECF6F320ED06F230ED16F140ED26F2E
:10011000280ED36FBF0ED46F290ED56F020ED66F87
:100120002A0ED76F800ED86F2B0ED96FDA6B2C0E7C
:10013000DB6FDC6B2D0EDD6FE80EDE6F2E0EDF6FDA
:10014000E00EE06F3C0EE16FE26BE36BE46B010EDF
:10015000E56FE66B020EE76FE86B030EE96F9C0E2E
:10016000EA6F040EEB6F600EEC6F050EED6F550E2F
:10017000EE6F060EEF6FF06B070EF16F5D0EF26F14
:10018000080EF36FF46B090EF56F550EF66F0A0E3D
:10019000F76FF86B0B0EF96F400EFA6F0C0EFB6FDA
:1001A000FC6B0D0EFD6F030EFE6F0E0EFF6F09014F
:1001B000006B0F0E016F400E026F100E036F046B89
:1001C000110E056F200E066F120E076F100E086FCE
:1001D000130E096F800E0A6F140E0B6F1A0E0C6F40
:1001E000150E0D6F180E0E6F160E0F6F040E106F9A
:1001F000170E116F040E126F180E136F2A0E146F64
:10020000190E156F200E166F1A0E176F800E186FCD
:100210001B0E196F3B0E1A6F1C0E1B6F1C691D0EF7
:100220001D6F800E1E6F1E0E1F6FA40E206F1F0EFF
:10023000216FB50E226F200E236F0F0E246F210E3B
:10024000256F200E266F220E276F320E286F230E89
:10025000296F140E2A6F280E2B6FBF0E2C6F290EDC
:100260002D6F020E2E6F2A0E2F6F800E306F2B0E09
:10027000316F326B2C0E336F346B2D0E356FE80EF1
:10028000366F2E0E376FE00E386F3C0E396F3A6BBB
:100290003B6B3C6B010E3D6F890E3E6F020E3F6F54
:1002A000800E406F030E416FE40E426F040E436FE9
:1002B000800E446F050E456F550E466F060E476F54
:1002C000486B070E496F5D0E4A6F080E4B6F4C6B03
:1002D000090E4D6F550E4E6F0A0E4F6F506B0B0E81
:1002E000516F400E526F0C0E536F546B0D0E556FC5
:1002F000030E566F0E0E576F586B0F0E596F400E50
:100300005A6F100E5B6F5C6B110E5D6F200E5E6F8F
:10031000120E5F6F100E606F130E616F6E0E626FC4
:10032000140E636F1A0E646F150E656F190E666FEB
:10033000160E676F040E686F170E696F040E6A6FF2
:10034000180E6B6F2A0E6C6F190E6D6F200E6E6F8C
:100350001A0E6F6F800E706F1B0E716F3B0E726FF7
:100360001C0E736F74691D0E756F780E766F1E0EFE
:10037000776FA40E786F1F0E796FB50E7A6F200E0F
:100380007B6F0F0E7C6F210E7D6F200E7E6F220E15
:100390007F6F320E806F230E816F140E826F280ED6
:1003A000836FBF0E846F290E856F020E866F2A0E33
:1003B000876F800E886F2B0E896F8A6B2C0E8B6F68
:1003C0008C6B2D0E8D6FE80E8E6F2E0E8F6FE00EE4
:1003D000906F3C0E916F926B936B946B010E956FC7
:1003E000966B020E976F986B030E996F9C0E9A6F27
:1003F000040E9B6F800E9C6F050E9D6F550E9E6FB9
:10040000060E9F6FA06B070EA16F5D0EA26F080E08
:10041000A36FA46B090EA56F550EA66F0A0EA76FEA
:10042000A86B0B0EA96F400EAA6F0C0EAB6FAC6BD6
:100430000D0EAD6F030EAE6F0E0EAF6FB06B0F0EE5
:10044000B16F400EB26F100EB36FB46B110EB56F7B
:10045000200EB66F120EB76F100EB86F130EB96F75
:10046000800EBA6F140EBB6F1A0EBC6F150EBD6FE7
:100470000A0EBE6F160EBF6F040EC06F170EC16F4F
:10048000040EC26F180EC36F2A0EC46F190EC56F0B
:10049000200EC66F1A0EC76F800EC86F1B0EC96F75
:1004A0003B0ECA6F1C0ECB6FCC691D0ECD6F800E3C
:1004B000CE6F1E0ECF6FA40ED06F1F0ED16FB50E74
:1004C000D26F200ED36F0F0ED46F210ED56F200E7A
:1004D000D66F220ED76F320ED86F230ED96F140E3F
:1004E000DA6F280EDB6FBF0EDC6F290EDD6F020E98
:1004F000DE6F2A0EDF6F800EE06F2B0EE16FE26B76
:100500002C0EE36FE46B2D0EE56FE80EE66F2E0EFA
:10051000E76FE00EE86F3C0EE96FEA6BEB6BEC6B9C
:10052000010EED6FEE6B020EEF6FF06B030EF16FCD
:100530009C0EF26F040EF36F800EF46F050EF56FD4
:10054000550EF66F060EF76FF86B070EF96F5D0E1E
:10055000FA6F080EFB6FFC6B090EFD6F550EFE6FF8
:100560000A0EFF6F0A01006B0B0E016F400E026F47
:100570000C0E036F046B0D0E056F030E066F0E0E4F
:10058000076F086B0F0E096F400E0A6F100E0B6F8E
:100590000C6B110E0D6F200E0E6F120E0F6F100EE2
:1005A000106F130E116F800E126F140E136F1A0E50
:1005B000146F150E156F190E166F160E176F040EA9
:1005C000186F170E196F040E1A6F180E1B6F2A0E74
:1005D0001C6F190E1D6F200E1E6F1A0E1F6F800EDE
:1005E000206F1B0E216F3B0E226F1C0E236F2469A0
:1005F0001D0E256F800E266F1E0E276FA40E286F0E
:100600001F0E296FB50E2A6F200E2B6F0F0E2C6F49
:10061000210E2D6F200E2E6F220E2F6F320E306F97
:10062000230E316F140E326F280E336FBF0E346FEE
:10063000290E356F020E366F2A0E376F800E386F17
:100640002B0E396F3A6B2C0E3B6F3C6B2D0E3D6FB2
:10065000E80E3E6F2E0E3F6FE00E406F3C0E416F76
:10066000426B436B446B010E456FA50E466F020E45
:10067000476F486B030E496FE40E4A6F040E4B6FD1
:10068000800E4C6F050E4D6F550E4E6F060E4F6F60
:10069000506B070E516F5D0E526F080E536F546B07
:1006A000090E556F550E566F0A0E576F586B0B0E8D
:1006B000596F400E5A6F0C0E5B6F5C6B0D0E5D6FC9
:1006C000030E5E6F0E0E5F6F606B0F0E616F400E5C
:1006D000626F100E636F646B110E656F200E666F94
:1006E000120E676F100E686F130E696F800E6A6FBF
:1006F000140E6B6F1A0E6C6F150E6D6F190E6E6FF8
:10070000160E6F6F040E706F170E716F040E726FFE
:10071000180E736F2A0E746F190E756F200E766F98
:100720001A0E776F800E786F1B0E796F3B0E7A6F03
:100730001C0E7B6F7C691D0E7D6F780E7E6F1E0E0A
:100740007F6FA40E806F1F0E816FB50E826F200E1B
:10075000836F0F0E846F210E856F200E866F220E21
:10076000876F320E886F230E896F140E8A6F280EE2
:100770008B6FBF0E8C6F290E8D6F020E8E6F2A0E3F
:100780008F6F800E906F2B0E916F926B2C0E936F6C
:10079000946B2D0E956FE80E966F2E0E976FE00EF0
:1007A000986F3C0E996F9A6B9B6B9C6B010E9D6FC3
:1007B0009E6B020E9F6FA06B030EA16F9C0EA26F2B
:1007C000040EA36F800EA46F050EA56F550EA66FC5
:1007D000060EA76FA86B070EA96F5D0EAA6F080E15
:1007E000AB6FAC6B090EAD6F550EAE6F0A0EAF6FEF
:1007F000B06B0B0EB16F400EB26F0C0EB36FB46BDB
:100800000D0EB56F030EB66F0E0EB76FB86B0F0EF1
:10081000B96F400EBA6F100EBB6FBC6B110EBD6F7F
:10082000200EBE6F120EBF6FC00EC06F130EC16FD1
:10083000800EC26F140EC36F1A0EC46F150EC56FF3
:100840001F0EC66F160EC76F040EC86F170EC96F46
:10085000040ECA6F180ECB6F2A0ECC6F190ECD6F17
:10086000200ECE6F1A0ECF6F800ED06F1B0ED16F81
:100870003B0ED26F1C0ED36FD4691D0ED56F800E48
:10088000D66F1E0ED76FA40ED86F1F0ED96FB50E80
:10089000DA6F200EDB6F0F0EDC6F210EDD6F200E86
:1008A000DE6F220EDF6F320EE06F230EE16F140E4B
:1008B000E26F280EE36FBF0EE46F290EE56F020EA4
:1008C000E66F2A0EE76F800EE86F2B0EE96FEA6B7A
:1008D0002C0EEB6FEC6B2D0EED6FE80EEE6F2E0E07
:1008E000EF6FE00EF06F3C0EF16FF26BF36BF46B99
:1008F000010EF56FF66B020EF76FF86B030EF96FD2
:100900009C0EFA6F040EFB6F800EFC6F050EFD6FE0
:10091000550EFE6F060EFF6F0B01006B070E016F89
:100920005D0E026F080E036F046B090E056F550E06
:10093000066F0A0E076F086B0B0E096F400E0A6FE9
:100940000C0E0B6F0C6B0D0E0D6F030E0E6F0E0E5B
:100950000F6F106B0F0E116F400E126F100E136F92
:10096000146B110E156F200E166F120E176FC00E3E
:10097000186F130E196F800E1A6F140E1B6F1A0E5C
:100980001C6F150E1D6F180E1E6F160E1F6F040EB6
:10099000206F170E216F040E226F180E236F2A0E80
:1009A000246F190E256F200E266F1A0E276F800EEA
:1009B000286F1B0E296F3B0E2A6F1C0E2B6F2C69A4
:1009C0001D0E2D6F800E2E6F1E0E2F6FA40E306F1A
:1009D0001F0E316FB50E326F200E336F0F0E346F56
:1009E000210E356F200E366F220E376F320E386FA4
:1009F000230E396F140E3A6F280E3B6FBF0E3C6FFB
:100A0000290E3D6F020E3E6F2A0E3F6F800E406F23
:100A10002B0E416F426B2C0E436F446B2D0E456FB6
:100A2000E80E466F2E0E476FE00E486F3C0E496F82
:100A30004A6B4B6B4C6B88C84DFB0001DBEF75F0CC
:100A400008018851000A0001D8B445EF85F0010A79
:100A5000D8B496EF85F0030AD8B4E7EF85F0010A21
:100A6000D8B438EF86F0070AD8B489EF86F0010AC7
:100A7000D8B4DAEF86F0030AD8B42BEF87F0010A76
:100A8000D8B47CEF87F0CDEF87F04AAE50EF85F019
:100A9000500EF66E070EF76E000EF86E01EC6DF05C
:100AA00008018A6B896B8A53D8A494EF85F0895129
:100AB0002A08D8A094EF85F0D89089350B014D6FA6
:100AC00008018A350B014E6F8D0E4D25E96E080E1B
:100AD0004E21EA6EEFCF8BF80801D89089350B01D3
:100AE0004D6F08018A350B014E6F010E4D25016EC9
:100AF000000E4E21036E01508D0FE96E080E03208B
:100B0000EA6EEFCF8CF808019A0E0C01B66F8BC815
:100B1000B7FC8CC8B8FC00018EEC75F00801892B7D
:100B2000D8B48A2B53EF85F0D0EF87F04AAEA1EF0F
:100B300085F06A0EF66E070EF76E000EF86E01EC89
:100B40006DF008018A6B896B8A53D8A4E5EF85F0B4
:100B500089512A08D8A0E5EF85F0D89089350B0196
:100B60004D6F08018A350B014E6FE50E4D25E96E7C
:100B7000080E4E21EA6EEFCF8BF80801D890893528
:100B80000B014D6F08018A350B014E6F010E4D258B
:100B9000016E000E4E21036E0150E50FE96E080E46
:100BA0000320EA6EEFCF8CF808019A0E0C01B66FA5
:100BB0008BC8B7FC8CC8B8FC00018EEC75F008013E
:100BC000892BD8B48A2BA4EF85F0D0EF87F04AAEFA
:100BD000F2EF85F0860EF66E070EF76E000EF86ED9
:100BE00001EC6DF008018A6B896B8A53D8A436EF4B
:100BF00086F089512A08D8A036EF86F0D89089353A
:100C00000B014D6F08018A350B014E6F3D0E4D25CE
:100C1000E96E090E4E21EA6EEFCF8BF80801D890ED
:100C200089350B014D6F08018A350B014E6F010E9E
:100C30004D25016E000E4E21036E01503D0FE96EF1
:100C4000090E0320EA6EEFCF8CF808019A0E0C0112
:100C5000B66F8BC8B7FC8CC8B8FC00018EEC75F081
:100C60000801892BD8B48A2BF5EF85F0D0EF87F0F7
:100C70004AAE43EF86F09E0EF66E070EF76E000E3C
:100C8000F86E01EC6DF008018A6B896B8A53D8A469
:100C900087EF86F089512A08D8A087EF86F0D89090
:100CA00089350B014D6F08018A350B014E6F950E8A
:100CB0004D25E96E090E4E21EA6EEFCF8BF8080143
:100CC000D89089350B014D6F08018A350B014E6FA5
:100CD000010E4D25016E000E4E21036E0150950F41
:100CE000E96E090E0320EA6EEFCF8CF808019A0E28
:100CF0000C01B66F8BC8B7FC8CC8B8FC00018EEC39
:100D000075F00801892BD8B48A2B46EF86F0D0EF16
:100D100087F04AAE94EF86F0B60EF66E070EF76EC9
:100D2000000EF86E01EC6DF008018A6B896B8A5336
:100D3000D8A4D8EF86F089512A08D8A0D8EF86F039
:100D4000D89089350B014D6F08018A350B014E6F24
:100D5000ED0E4D25E96E090E4E21EA6EEFCF8BF8B0
:100D60000801D89089350B014D6F08018A350B01B8
:100D70004E6F010E4D25016E000E4E21036E015087
:100D8000ED0FE96E090E0320EA6EEFCF8CF8080133
:100D90009A0E0C01B66F8BC8B7FC8CC8B8FC00016A
:100DA0008EEC75F00801892BD8B48A2B97EF86F06A
:100DB000D0EF87F04AAEE5EF86F0CE0EF66E070E66
:100DC000F76E000EF86E01EC6DF008018A6B896B0E
:100DD0008A53D8A429EF87F089512A08D8A029EF8F
:100DE00087F0D89089350B014D6F08018A350B01CA
:100DF0004E6F450E4D25E96E0A0E4E21EA6EEFCF7D
:100E00008BF80801D89089350B014D6F08018A35A0
:100E10000B014E6F010E4D25016E000E4E21036E2B
:100E20000150450FE96E0A0E0320EA6EEFCF8CF8F1
:100E300008019A0E0C01B66F8BC8B7FC8CC8B8FCC1
:100E400000018EEC75F00801892BD8B48A2BE8EFED
:100E500086F0D0EF87F04AAE36EF87F0E60EF66EFA
:100E6000070EF76E000EF86E01EC6DF008018A6B4C
:100E7000896B8A53D8A47AEF87F089512A08D8A0C1
:100E80007AEF87F0D89089350B014D6F08018A35CC
:100E90000B014E6F9D0E4D25E96E0A0E4E21EA6E36
:100EA000EFCF8BF80801D89089350B014D6F080101
:100EB0008A350B014E6F010E4D25016E000E4E213D
:100EC000036E01509D0FE96E0A0E0320EA6EEFCF0C
:100ED0008CF808019A0E0C01B66F8BC8B7FC8CC851
:100EE000B8FC00018EEC75F00801892BD8B48A2B70
:100EF00039EF87F0D0EF87F04AAE87EF87F0FE0E2C
:100F0000F66E070EF76E000EF86E01EC6DF008013C
:100F10008A6B896B8A53D8A4CBEF87F089512A0852
:100F2000D8A0CBEF87F0D89089350B014D6F080121
:100F30008A350B014E6FF50E4D25E96E0A0E4E21D6
:100F4000EA6EEFCF8BF80801D89089350B014D6F11
:100F500008018A350B014E6F010E4D25016E000E02
:100F60004E21036E0150F50FE96E0A0E0320EA6E62
:100F7000EFCF8CF808019A0E0C01B66F8BC8B7FC46
:100F80008CC8B8FC00018EEC75F00801892BD8B430
:100F90008A2B8AEF87F0D0EF87F00801D0EF87F037
:100FA000000179EF7DF00801736B726B7E6B7F6BD4
:100FB0006DC87FF86EC87EF86EC873F86DC872F899
:100FC0004DBE03EF88F072511508D8A4EDEF87F0FD
:100FD00073512A08D8B403EF88F072519508D8A449
:100FE000F7EF87F073512C08D8B403EF88F07251F3
:100FF0001508D8A401EF88F073512D08D8B403EF79
:1010000088F0A2EF8DF03553D8A411EF88F072511B
:101010000308D8A413EF89F073511208D8A413EF72
:1010200089F03551000A0001D8B435EF88F0010A83
:10103000D8B435EF88F0030AD8B435EF88F0010A48
:10104000D8B446EF88F0070AD8B465EF88F0010AF3
:10105000D8B474EF88F0030AD8B491EF88F0010A8D
:10106000D8B4E4EF88F00FEF89F00801725103085B
:10107000D8A443EF88F073511208D8A443EF88F046
:10108000352B13EF89F0356B13EF89F008017331BD
:10109000816F7231806F813380338133803381334C
:1010A00080330F0E81178017816B010E385D805DD4
:1010B000D8A462EF88F08153D8A462EF88F0352B72
:1010C00013EF89F0356B13EF89F00801722D71EF82
:1010D00088F073510A08D8A471EF88F0352B13EF0C
:1010E00089F0356B13EF89F008017251F00B806FB6
:1010F00073C881F88053D8A48EEF88F081510A0814
:10110000D8A48EEF88F072510F0B376F3751050856
:10111000D8A08EEF88F0352B13EF89F0356B13EFE5
:1011200089F008017251F00B806F73C881F8805309
:10113000D8A4E1EF88F081510A08D8A4E1EF88F043
:1011400072510F0B006E036A0050006E0350D8A45A
:10115000B1EF88F0010E005C0001D8B4C9EF88F04F
:1011600008010350D8A4BCEF88F0020E005C000117
:10117000D8B4CFEF88F008010350D8A4C7EF88F0A7
:10118000030E005C0001D8B4D5EF88F00801DAEF57
:1011900088F0020E0801366F352BDDEF88F0010E66
:1011A0000801366F352BDDEF88F00801366B352BE3
:1011B000DDEF88F0356BDDEF88F013EF89F0E2EFBB
:1011C00088F0356B13EF89F00801806B73C881F8E4
:1011D0008053D8A40CEF89F081510A08D8A40CEFF1
:1011E00089F03939006EF00E001600508009746FD6
:1011F000010E756F040E766F3F0E776F36C878F864
:1012000037C879F87A69080E0901306F740E2F6FAC
:101210000001A8EC35F00801356B13EF89F00801E7
:10122000356B13EF89F07251006E7351036E2A0E05
:10123000035CD8A423EF89F0150E005C0001D8B43C
:1012400029EF8BF008012C0E035CD8A42FEF89F056
:10125000950E005C0001D8B429EF8BF008012D0E2B
:10126000035CD8A43BEF89F0150E005C0001D8B4F4
:1012700029EF8BF008011D0E035CD8A447EF89F01D
:10128000680E005C0001D8B453EF8BF008019D0E8E
:10129000035CD8A453EF89F0680E005C0001D8B459
:1012A00053EF8BF008012A0E035CD8A45FEF89F09E
:1012B000280E005C0001D8B469EF8BF008012C0EF9
:1012C000035CD8A46BEF89F0A80E005C0001D8B4D1
:1012D00069EF8BF008012D0E035CD8A477EF89F03D
:1012E000280E005C0001D8B469EF8BF008011D0ED8
:1012F000035CD8A483EF89F01A0E005C0001D8B417
:101300009BEF8BF008019D0E035CD8A48FEF89F052
:101310001A0E005C0001D8B49BEF8BF008011D0E83
:10132000035CD8A49BEF89F01B0E005C0001D8B4CD
:10133000CAEF8BF008019D0E035CD8A4A7EF89F0DB
:101340001B0E005C0001D8B4CAEF8BF008011D0E23
:10135000035CD8A4B3EF89F01D0E005C0001D8B483
:10136000F9EF8BF008019D0E035CD8A4BFEF89F064
:101370001D0E005C0001D8B4F9EF8BF008011D0EC2
:10138000035CD8A4CBEF89F01C0E005C0001D8B43C
:1013900028EF8CF008019D0E035CD8A4D7EF89F0EC
:1013A0001C0E005C0001D8B428EF8CF008011D0E63
:1013B000035CD8A4E3EF89F0190E005C0001D8B4F7
:1013C00057EF8CF008019D0E035CD8A4EFEF89F075
:1013D000190E005C0001D8B457EF8CF008011D0E07
:1013E000035CD8A4FBEF89F0180E005C0001D8B4B0
:1013F00078EF8CF008019D0E035CD8A407EF8AF00B
:10140000180E005C0001D8B478EF8CF008012A0EA9
:10141000035CD8A413EF8AF01C0E005C0001D8B462
:101420009CEF8CF008012C0E035CD8A41FEF8AF00F
:101430009C0E005C0001D8B49CEF8CF008012D0ECE
:10144000035CD8A42BEF8AF01C0E005C0001D8B41A
:101450009CEF8CF008012A0E035CD8A437EF8AF0C9
:101460001D0E005C0001D8B4BDEF8CF008012C0EFD
:10147000035CD8A443EF8AF09D0E005C0001D8B451
:10148000BDEF8CF008012D0E035CD8A44FEF8AF05D
:101490001D0E005C0001D8B4BDEF8CF008012A0ECF
:1014A000035CD8A45BEF8AF01A0E005C0001D8B48C
:1014B000DEEF8CF008012C0E035CD8A467EF8AF0F5
:1014C0009A0E005C0001D8B4DEEF8CF008012D0EFE
:1014D000035CD8A473EF8AF01A0E005C0001D8B444
:1014E000DEEF8CF008012A0E035CD8A47FEF8AF0AF
:1014F0001B0E005C0001D8B4FFEF8CF008012C0E2D
:10150000035CD8A48BEF8AF09B0E005C0001D8B47A
:10151000FFEF8CF008012D0E035CD8A497EF8AF042
:101520001B0E005C0001D8B4FFEF8CF008012A0EFE
:10153000035CD8A4A3EF8AF0230E005C0001D8B4AA
:1015400020EF8DF008012C0E035CD8A4AFEF8AF0D9
:10155000A30E005C0001D8B420EF8DF008012D0E21
:10156000035CD8A4BBEF8AF0230E005C0001D8B462
:1015700020EF8DF008012A0E035CD8A4C7EF8AF093
:101580001F0E005C0001D8B444EF8DF008012C0E52
:10159000035CD8A4D3EF8AF09F0E005C0001D8B49E
:1015A00044EF8DF008012D0E035CD8A4DFEF8AF024
:1015B0001F0E005C0001D8B444EF8DF008012A0E24
:1015C000035CD8A4EBEF8AF01E0E005C0001D8B4D7
:1015D00061EF8DF008012C0E035CD8A4F7EF8AF0C0
:1015E0009E0E005C0001D8B461EF8DF008012D0E55
:1015F000035CD8A403EF8BF01E0E005C0001D8B48E
:1016000061EF8DF008012A0E035CD8A40FEF8BF078
:10161000220E005C0001D8B47EEF8DF008012C0E84
:10162000035CD8A41BEF8BF0A20E005C0001D8B4C1
:101630007EEF8DF008012D0E035CD8A427EF8BF010
:10164000220E005C0001D8B47EEF8DF00801A2EFFD
:101650008DF073C881F872C880F831EC7FF0080112
:101660003851015CD8A451EF8BF03853D8B451EF06
:101670008BF031510908D8B451EF8BF0090E316F5E
:101680004DAE4BEF8BF0010E09012F6F00014DECB9
:101690001CF050EF8BF009012F6B00014DEC1CF09A
:1016A0000801A2EF8DF070C883F86FC882F86EC889
:1016B00081F86DC880F84FEC7FF008013851015C6B
:1016C000D8A467EF8BF03853D8B467EF8BF0A2EF54
:1016D0008DF073C881F872C880F831EC7FF0080192
:1016E0003851015CD8A499EF8BF03853D8B499EFF6
:1016F0008BF031510A08D8B499EF8BF00A0E316F94
:101700004DA686EF8BF04D9687EF8BF04D864DA65C
:1017100092EF8BF0020E09016A6F0001F3EC30F0DA
:1017200098EF8BF0030E09016A6F0001F3EC30F0C3
:101730000801A2EF8DF070C883F86FC882F86EC8F8
:1017400081F86DC880F84FEC7FF008013851015CDA
:10175000D8A4C8EF8BF03853D8B4C8EF8BF0315110
:101760000308D8B4C8EF8BF0030E316F4AB2C1EF53
:101770008BF0030E806F00017DEC7FF0C6EF8BF0E5
:101780000801040E806F00017DEC7FF008013487B2
:10179000A2EF8DF070C883F86FC882F86EC881F828
:1017A0006DC880F84FEC7FF008013851015CD8A477
:1017B000F7EF8BF03853D8B4F7EF8BF031510408C2
:1017C000D8B4F7EF8BF0040E316F4AB2F0EF8BF024
:1017D000040E806F00017DEC7FF0F5EF8BF00801C7
:1017E000030E806F00017DEC7FF008013487A2EFCB
:1017F0008DF070C883F86FC882F86EC881F86DC824
:1018000080F84FEC7FF008013851015CD8A426EF36
:101810008CF03853D8B426EF8CF031510208D8B48C
:1018200026EF8CF0020E316F4AB21FEF8CF0020EE1
:10183000806F00017DEC7FF024EF8CF00801010E39
:10184000806F00017DEC7FF008013487A2EF8DF0FE
:1018500070C883F86FC882F86EC881F86DC880F8C8
:101860004FEC7FF008013851015CD8A455EF8CF0A3
:101870003853D8B455EF8CF0312D41EF8CF055EF43
:101880008CF0010E316F4AB24EEF8CF0010E806F7A
:1018900000017DEC7FF053EF8CF00801020E806FA9
:1018A00000017DEC7FF008013487A2EF8DF070C855
:1018B00083F86FC882F86EC881F86DC880F84FEC65
:1018C0007FF008013851015CD8A476EF8CF03853D2
:1018D000D8B476EF8CF031510808D8B476EF8CF09C
:1018E000080E316F000175EC14F00801A2EF8DF0C5
:1018F00070C883F86FC882F86EC881F86DC880F828
:101900004FEC7FF008013851015CD8A49AEF8CF0BD
:101910003853D8B49AEF8CF031510708D8B49AEF05
:101920008CF0070E316F4D9E09012F6B00014DECBD
:101930001CF00801A2EF8DF073C881F872C880F81E
:1019400031EC7FF008013851015CD8A4BBEF8CF07A
:101950003853D8B4BBEF8CF033510508D8B4BBEF83
:101960008CF0050E336F270E0901306F000198ECE3
:1019700019F008013483A2EF8DF073C881F872C8A2
:1019800080F831EC7FF008013851015CD8A4DCEF1D
:101990008CF03853D8B4DCEF8CF033510608D8B44F
:1019A000DCEF8CF0060E336F370E0901306F00014B
:1019B00098EC19F008013483A2EF8DF073C881F818
:1019C00072C880F831EC7FF008013851015CD8A46E
:1019D000FDEF8CF03853D8B4FDEF8CF0335105088F
:1019E000D8B4FDEF8CF0050E336F210E0901306F76
:1019F000000198EC19F008013483A2EF8DF073C850
:101A000081F872C880F831EC7FF008013851015C30
:101A1000D8A41EEF8DF03853D8B41EEF8DF033519B
:101A20000608D8B41EEF8DF0060E336F310E090193
:101A3000306F000198EC19F008013483A2EF8DF0AB
:101A400073C881F872C880F831EC7FF00801385112
:101A5000015CD8A442EF8DF03853D8B442EF8DF03A
:101A60004DA042EF8DF032510508D8B442EF8DF011
:101A7000050E326F3485030E0901306F00012BEC27
:101A800038F00801A2EF8DF073C881F872C880F8B1
:101A900031EC7FF008013851015CD8A45FEF8DF084
:101AA0003853D8B45FEF8DF04DB05FEF8DF04D80BF
:101AB000030E09016A6F000189EC1DF00801A2EF15
:101AC0008DF073C881F872C880F831EC7FF008019E
:101AD0003851015CD8A47CEF8DF03853D8B47CEF3A
:101AE0008DF04DA07CEF8DF04D90020E09016A6FD4
:101AF000000189EC1DF00801A2EF8DF073C881F898
:101B000072C880F831EC7FF008013851015CD8A42C
:101B1000A0EF8DF03853D8B4A0EF8DF04DA0A0EF1A
:101B20008DF032510608D8B4A0EF8DF0060E326F5A
:101B30003485020E0901306F00012BEC38F00801EA
:101B4000A2EF8DF00001120008016C6B6B6B0001BD
:101B500035EF7EF002C06CF801C06BF8080130511F
:101B60001308D8A0F8EF8DF06CC86EF86BC86DF84C
:101B700030C86FF8000158EF7EF00150FC0FD8B06C
:101B8000F5EF8DF0040F0EEF8EF0080130511108C3
:101B9000D8A0CFEF8DF0302B0001F5EF8DF0C5C64A
:101BA00070F8C4C66FF8C3C66EF8C2C66DF830C808
:101BB00071F80001D3EC87F00801306B0001C5C655
:101BC00070F8C4C66FF8C3C66EF8C2C66DF830C8E8
:101BD00071F8D3EC87F00801306B0601C56BC46B5C
:101BE000C36BC26B0001F5EF8DF0FEEF8DF00801C5
:101BF000306B0601C56BC46BC36BC26B08012F5100
:101C00002E5DD8A40BEF8EF0960E0C01B66F00017E
:101C10006BEC07F00801000132EF8EF0E824F76A60
:101C2000F7363D0FF66E1C0EF722010EF86EFB6EB6
:101C30000A00F550FA6E0800F550F96E8A1B8A1BEF
:101C4000BE1BD61B4EBC7AEF8EF008012F512E5DC5
:101C5000D8B43FEF8EF02F512E5DD8B435EF8EF013
:101C6000000172D708012BEF8EF04C9A306B060101
:101C7000C56BC46BC36BC26B77EF8EF008012F6B23
:101C80002FC82EF8B250B3CF03F06B6FB3506C6F08
:101C90000608D8B076EF8EF0FF0AD8A455EF8EF084
:101CA0006B513A08D8B076EF8EF034A35FEF8EF028
:101CB00034930901306B000198EC19F0080134A548
:101CC00069EF8EF034950901306B00012BEC38F090
:101CD000080134A772EF8EF03497806B00017DEC21
:101CE0007FF00801346B316B326B336B06017FEF91
:101CF0008EF0000108012F6B2FC82EF8060100019D
:101D0000D1EF90F0F86AD09E078E0C0E1D6ECC0EAF
:101D10001C6E020E0C01CD6F900ECC6FCF6BCE6B94
:101D20000001EA6AE96A700ED36E400E9B6ED350D2
:101D30007E86820EAF6E060E7F6EE60EAC6ED00E05
:101D4000AB6E7C86400E6F6E030E7D6EA60E6C6EC3
:101D5000900E6B6E948694884F0EC86E280EC66ED9
:101D6000C78EC79C456A446A436A426A476A466AA4
:101D7000496A486A4B6A4A6A4C904C925168FE0E16
:101D8000526E536A5468566A556A586A576A596A55
:101D90000101006B016B4C944C9606017B6B7A6BD6
:101DA0007D6B7C6B7E6B4C98BF6BC06BC16BC56BE6
:101DB000C46BC36BC26B08012E6B2F6B306B316B26
:101DC000326B336B346B356B366B376B010E386FA0
:101DD0004C9A810E396F870E3A6F3B6B4C9C4C9E30
:101DE000476B070E486F49694A6B4B6B4D6B4C6BE9
:101DF000C150C00B0F09C16E070EB46E1E6A1F6A78
:101E0000560E246E300E256E310E266E2E0E276E67
:101E1000300E286E310E296E2E0E2A6E300E2B6E6D
:101E2000330E2C6E2D6A200E2E6E480E2F6E440E31
:101E3000306E320E316E300E326E200E336E200E4A
:101E4000346E200E356E200E366E376A310E386EC7
:101E5000330E396E2D0E3A6E530E3B6E650E3C6E90
:101E6000700E3D6E2D0E3E6E310E3F6E310E406E89
:101E7000416A900E3C6F500E3D6F3E6B010E3F6FFE
:101E8000050E406F040E416F0E0E426F0E0E436F33
:101E9000020E446F4569466B686B676B6A6B696BD2
:101EA000210EC86E7D6A400E7C6E330E6F6EA00EE2
:101EB0006C6E900E6B6E8E8097908C9895988C8A35
:101EC000959A8C8695968C84959497988E88938015
:101ED000676B81B0672B686B958E676B83BE672BD2
:101EE000686B958C676B83BC672B686B9786676B99
:101EF00085B6672B686B9784676B85B4672B686BB7
:101F0000968C676B84BC672B686B97928E82700E81
:101F1000D36E400E9B6ED350F19E978A676B85BA45
:101F2000672B686B978C676B85BC672B686BB50EEE
:101F3000B16E850ECD6E800ED56E9D809D8AA38A72
:101F400000011FEC07F0F19A84A6B4EF8FF04E9CCD
:101F50004E9AF29CF29EF2BEAAEF8FF0F0908B9A0E
:101F6000949AF086C3EF8FF04E8C4E8AF29CF29ECC
:101F7000F2BEB7EF8FF0F0908B8A949AF09608013A
:101F80002E6B2F6B00014C92C00EF21248EF07F03F
:101F9000CAEF07F0012CCFEF8FF0D1EF8FF0A1EF58
:101FA00008F04FEF0AF04A9E4D9E0BEF0BF0C7EC86
:101FB0006AF039C86BF807EF6CF0080EEA6E4E0E47
:101FC000E96E006A026A190E016E3BEC07F0080E1A
:101FD0000801F86F4E0EF76F180EF96F00016CECE8
:101FE0000FF0012CFEEF8FF0080E0801F86F4E0E77
:101FF000F76F000178EC69F0E7EF8FF085A612EF3C
:1020000090F085A60CEF90F0020E0C01B66F000167
:102010006BEC07F001EF90F00A0E0C01B66F0001B7
:102020006BEC07F0010E08016B6F000154EC7CF0C3
:10203000080EEA6E4E0EE96E006A026A190E016E13
:102040003BEC07F0080E0801F86F4E0EF76F180E04
:10205000F96F00016CEC0FF0012C39EF90F0080ED5
:102060000801F86F4E0EF76F000178EC69F022EF6F
:1020700090F01FEC07F008016A6B696B6AC867F99A
:1020800069C866F90901696B320E686F000135ECA9
:1020900014F002C06CF801C06BF808016C53D8A4AE
:1020A0007AEF90F06B51F908D8A07AEF90F0080E13
:1020B000F86F4E0EF76F180EF96F00016CEC0FF011
:1020C000012C6EEF90F0080E0801F86F4E0EF76FBE
:1020D000000178EC69F0080157EF90F0320E0C0126
:1020E000B66F00016BEC07F00801692BD8B46A2BBE
:1020F0003EEF90F0020E0901306F0001F8EC1BF08A
:10210000080EEA6E4E0EE96E006A026A190E016E42
